:020000040000FA
:1000000000F80202E1360000B911000025120000DC
:1000100000000000000000000000000000000000E0
:100020000000000080E30000C8E30000B9110000F8
:100030000000000000000000B9110000E1370000DE
:1000400045110000B9110000B9110000053700008A
:10005000D91400003534000049110000E9110000F6
:10006000A10E0000BD0D0000B9110000BD1100007F
:10007000AD140000C53C000081360000AD36000024
:10008000B9110000B9110000B911000009380000D1
:1000900029380000B9110000B9110000B9110000A1
:1000A0004D38000057380000471100009D35000012
:1000B000B91100009D3400000000000000000000A5
:1000C0000348854600F094FC004800470178000092
:1000D00000F8020230B50B46014600202022012420
:1000E00009E00D46D5409D4205D31D469540491B6C
:1000F0002546954040191546521E002DF1DC30BDB5
:1001000070B500242546002801DA01244042002968
:1001100001DA01254942FFF7DDFFAC4200D0404241
:10012000002C00D0494270BD03460B439B0703D00F
:1001300009E008C9121F08C0042AFAD203E00B78AC
:100140000370401C491C521EF9D27047D2B201E024
:100150000270401C491EFBD270470022F6E710B522
:1001600013460A4604461946FFF7F0FF204610BD25
:100170000FB400B58DB009900B9010A9002000912C
:10018000C0430A9000200C9006480690064807904D
:100190006A4609A80F9900F059FB0DB008BC04B0DD
:1001A000184700006D0800008D080000FFB5002012
:1001B00083B00090506801909169144600269768BA
:1001C0000498884705460C990698084305D009E02D
:1001D000A169761C049888470546216A2846884705
:1001E0000028F5D1681C03D00198C00704D017E09F
:1001F0000020C04307B0F0BD2068011D21600068E9
:1002000000900DE00198C00704D100980570009897
:10021000401C0090A169761C7F1E04988847054603
:10022000002F1CDD681C1AD0069800280FD0E81794
:10023000C00E401941118A00069940095118400129
:100240002A1A0968012090400142DBD107E00C988E
:100250000028D7D1216A284688470028D2D0E169F2
:10026000049888470C98002807D1002E05DD0198D6
:10027000C00702D1009800210170A068B84204DDD7
:100280000C98002804D0002F02D00120C043B1E711
:100290003046AFE7F8B502464A40D40F42004B0063
:1002A00052085B089A4202D20246084611464A00AA
:1002B00023D0C30D4A00DDB2120EAD1A202D35DA5F
:1002C00049020126490AF6058A19002C00D052423B
:1002D00020214F1B1146B9402A411018C20D9A42E5
:1002E00021D0002C17D0012D08DCDA05801AD20F9E
:1002F0008019D207DBB200F0E3FAF8BDDA05801A04
:10030000012340001B06C01880185A428018CA0FEB
:100310001043490007E04908C2071143DA05801A73
:1003200080194008801800F0C3FAF8BD610001226E
:10033000511A001BF7E70122D2075140AAE7012218
:10034000D2075040A6E7024670B54A40D30FDB07FC
:1003500040002DD04A002AD0010E140E00021202D5
:100360000919400A520A8418E50104465443000A58
:10037000120A2E045043A4194219200CC543AA188E
:10038000120C0125AD03521C521912047F392404AA
:1003900000D0521C104301D44000491EC2B20C06CA
:1003A000C0092018401C4008802A02D003E0002029
:1003B00070BD40084000002900DA0020184370BDDD
:1003C00070B502464A40D50F40004A00ED0740088C
:1003D0005208002814D0002A12D0C40DD30D4102B7
:1003E0000120C0055202490A520AE41A09181218DB
:1003F0007D34914201D3641C00E04900002C01DAF5
:10040000002070BD0023914201D3891A03434008A4
:1004100049000028F7D100290AD0914202D10121D8
:10042000C90705E0914201D2012101E00121C94340
:10043000E005C018401900F03BFA70BDF0B51FB4DC
:1004400088B00B990998002448400999C00F4900C9
:1004500049080991C0070B990090490049080B9180
:1004600009990898A64608431CD00B990A98084396
:1004700018D0099801244000420D4800410D099808
:1004800024050003000B204309900B980003000B88
:1004900020430B9050181C4940180022019014462C
:1004A000104605E0002001460DB0F0BD032801DA3A
:1004B000034600E003239C46C11A0AAE0AE05F002F
:1004C00008ADED5B4F00F75B7D430027AA187C4128
:1004D000491C5B1E6145F2DD410004AB5A52210408
:1004E000120C0A43240C401C0828DFDB0198029000
:1004F0000099704601910090059B049A079906980F
:1005000000F024FAD0E700000DFCFFFFF0B50C4628
:100510005C4085B0E40FE40703944C0000266408B7
:1005200059009446490802460296224321D0624669
:100530000A431ED06200570D4A000E032303550DD7
:10054000012402462C492405781B1B0B360B40184E
:1005500023432643614600901C46501AB44103D3FE
:100560000098401C009002E0921800985B4100281F
:1005700003DA0020014605B0F0BD00200121090585
:100580000746864611E064461D46141BB54106D356
:100590006546521BB341744607430C43A646CD073C
:1005A00040084908284392185B4105460D43EAD1AB
:1005B0001046184313D06046194650407140084316
:1005C00006D06046101AB34106D20122002306E08D
:1005D00000220123DB0702E00122D24353100098DE
:1005E00074460105381C6141029C039D0019694154
:1005F00000F09FF9BFE70000FD0300000122D207D1
:10060000002800DB101A002900DB511A814201D8B2
:1006100001207047002070470122D207002800DB2C
:10062000101A002900DB511A814201D201207047C3
:10063000002070470122D207002800DB101A002991
:1006400000DB511A814201D301207047002070471E
:100650000122D207002800DB101A002900DB511A02
:10066000814201D901207047002070470122D20742
:10067000002800DB101A002900DB511A814201D149
:10068000012070470020704710B5002904DB0C469C
:100690000121C9074042A141002B04DB1C46012374
:1006A000DB075242A34142404B401A4301D0002095
:1006B00010BD012010BDC217C10F504010B5401829
:1006C000CA079623002100F0FBF810BD10B50022E8
:1006D0009623114600F0F4F810BD00000EB5054950
:1006E0000291002100910A460B46019100F02EF97B
:1006F00003B000BD33040000C20F410040020123DB
:10070000400ADB05D207090EC0187F2901DA002054
:100710007047962903DC9623591AC84001E09639A0
:100720008840002AF4D04042704741004002012234
:10073000400AD205090E80187F2901DA002070478F
:10074000962903DC9622511AC84070479639884092
:100750007047000070B5CD0F4A0009030123090B53
:100760001B0519430B4BED070024520D9A4201DA89
:10077000002070BD074B34339A4203DC9A1A00F014
:100780004DF802E00449511888402C43F1D0404212
:1007900070BD0000FF030000CDFBFFFFC20FD207BA
:1007A000400040080BD0C10D0723DB01C9184002EF
:1007B0000905400A1143C208400711437047002051
:1007C00001467047CB0FDB07490010B549080246C8
:1007D0000A4307D00A0D07240903E401090B121B81
:1007E000002A01DC002010BDC900440F0C43C100E9
:1007F000E018D205801800F05BF810BD10B5202A73
:1008000004DB0146203A9140002010BD9140202396
:100810009C1A0346E3401943904010BD10B5202AAE
:1008200004DB0846203AD040002110BD0B46D340DF
:10083000D0402024A21A91400843194610BD000060
:1008400002681378511801601846704710B5D160DE
:10085000044951610449116200211161114600F0FF
:10086000E1F810BD41080000150A00004268002AA6
:1008700008D001680B78491C002B03D0521E06C01B
:10088000184670470121C160881E70474268002ADF
:100890000BD0C3680168002B07D183688B4204D05A
:1008A000491E521C06C0002070470020C0437047FC
:1008B000002904DA401C490001D14008400070477B
:1008C00070B40024050C05D11024000402D10029C5
:1008D00021D01124050E01D100020834050F01D1E9
:1008E0000001241D850F01D18000A41C002801DB1C
:1008F0004000641C002908D020252E1B0D46F54021
:10090000A14000D001212943084301061B1B000A16
:10091000DB1D02D5002070BC7047DB05181880185D
:100920000029F8DA401C4900F5D170BC40084000AD
:10093000704710B5002B08DA0024401C6141921862
:100940005B411A4301D14008400010BDF0B51FB40F
:1009500082B005460C0003D008460BF091FC02E083
:100960000BF08EFC20300246009021462846FFF70F
:1009700045FF049B059A04460F461843114308435C
:1009800014D0184610431BD0009840210A1A18466C
:100990000599FFF743FF05460E46009A059904980E
:1009A000FFF72CFF084305D0012004E0204639461C
:1009B00007B0F0BD0020C11705430E432C43374359
:1009C00000990E986305401A7905E40A00220C4349
:1009D000FD0A0A3002D500200146E9E70105101999
:1009E00069410C9C0D9D00196941FFF7A2FFDFE7EB
:1009F000064C0125064E05E0E36807CC2B430C3C72
:100A000098471034B442F7D3FFF75EFB40DE000096
:100A100060DE000010B50F21C0B2490200F09EF95F
:100A200010BD0000F3B58DB000200A9001200B909E
:100A3000002608460C300C4609906269012109988D
:100A40009047051E2ED0252D2DD0216A88470028DD
:100A500018D06269012109989047216A88470028C7
:100A6000F7D1411E62690998904700E0761CA169A0
:100A70000D988847216A88470028F7D1E1690D98C9
:100A80008847DAE7A1690D9888470746A84201D14F
:100A9000761CD2E7E1690D9888477F1C02D10A983D
:100AA000002877D049E1002762693D463946099818
:100AB00090472A280CD162690121099890470125A5
:100AC00006E00A214F433F18303FEBD41020054386
:100AD0006269012109989047014630390A2903D2F9
:100AE0009B498F42DEDCECE7E90600D4994F6C2885
:100AF0000AD04C2810D0682824D06A282ED0742818
:100B00000CD07A280AD00DE062690121099890473B
:100B10006C2823D004211CE02020054362690121B8
:100B200009989047A760656065284FD026DC582853
:100B300039D01ADC452849D012DC252834D0412888
:100B4000B0D143E06269012109989047682802D03A
:100B500008210D43E6E70120C002DEE70220DCE7C2
:100B6000462833D047282CD130E05B2870D061284C
:100B70002CD063286CD0642823D161E06F284FD03B
:100B800009DC662822D0672820D0692826D06E2864
:100B900017D12EE0CDE070284DD073286FD0752886
:100BA0004ED078280DD154E0A1690D9888470546AC
:100BB000252800D16CE7E1690D9888476D1C00D1AC
:100BC0006DE7BAE00A224CE00A2252E001202346F7
:100BD0006A46C0430D99C046C046A3E0284640215E
:100BE00008436060A807234601D5002239E00022AF
:100BF0003FE0E80700D020E72068011D2160006881
:100C0000290501D5067018E7290701D5068014E7E4
:100C1000A90703D5F117066041600EE706600CE7EF
:100C20002846402108436060A807234601D50822D2
:100C300017E008221DE0484928460840606016E099
:100C40002846402108436060A8072346BCD5B9E781
:100C500015E02846402108436060A80707D52346D1
:100C600010220120C0430D99C046C0465AE02346D9
:100C700010220120C0430D99C046C04652E0002119
:100C80000C910B460091632802D05B2807D043E00B
:100C9000E80601D40120A060012000903CE06269D8
:100CA0000121099890475E2805D101200C9001464A
:100CB0006269099890472169002906D10B4601AA6B
:100CC0008F00491CD3510829FADB002835D021694F
:100CD00000290ED1C117C90E09184A11930001AAA3
:100CE0009A1849094901411A0120136888400343B1
:100CF000136062690121099890475D28E5D10C983D
:100D0000002808D0002001AB81005A58401CD24373
:100D10005A500828F8DB01AB01202246C0430D9948
:100D2000FFF744FA00280ADA401C06D10B98002885
:100D300003D00020C0430FB0F0BD0A98FBE7E907DD
:100D400002D10A99491C0A91361800200B9074E6CA
:100D5000CCCCCC0CFFFFFF7FF1F7FFFF7F2801D940
:100D6000002207E0054B42089A5CC00700D1120937
:100D70001207120F0120904008407047CCC20000BB
:100D800030B58C180278401C13071B0F01D1037873
:100D9000401C120906D10278401C03E005780D7052
:100DA000401C491C5B1EF9D101E00B70491C521E0E
:100DB000FBD1A142E6D3002030BD000010B524488D
:100DC000016A8A0717D44A0717D4C90739D02249BC
:100DD0000A88002A17D0521E0A8081681F4B1C689F
:100DE00002C41C601E49096812040ED0002927D1D4
:100DF0000121016010BD022100E00421C1611548FC
:100E00008021016010BD16490968012909D10168D6
:100E1000012291430160C261FF206830993011497D
:100E200008600C48012101600F480268002A07D0C1
:100E30000A4800680D4909888B00C01A904710BD08
:100E400010BDFF2268320A480AA10EA308F0B2FFC3
:100E500008D00140A4950102B0950102A8950102B5
:100E6000A095010280E200E09C950102AC95010290
:100E700064CD00004144435F49525148616E646C47
:100E800065720000556E6578706563746564204115
:100E9000444320696E746572727570740D0A0000A7
:100EA00070B582B000230193444801688A6A4C6897
:100EB00013252540132D02D1CB689B07DB0F43611F
:100EC000930772D453070AD4D30711D1130724D53B
:100ED000048F838E1C1B102C0EDD102310E00420C9
:100EE00088620220032142A209F094FF02B070BD83
:100EF0000120886202B070BD048F1B1B1C0610D03D
:100F0000DBB20024058FC66A75192D5D0D74641C53
:100F1000A342F7D1048FE3180387D20607D4002138
:100F20002FE04B6A0824A3434B62D206F7D5CB6867
:100F3000C28E448F141B5B04DB0EA34201D3438F8C
:100F4000D31ADAB2002A16D0097D438F046BE1541C
:100F50000199012A10D001231C46890145582D7D95
:100F600041184E8F9B19096BCD54641CE3B2019953
:100F70009A42F2D800E000218B01C3185C8FA218BE
:100F80005A878A0181184B8FCC8EA3420BD3012341
:100F90000B61805800224262CA6B002A03D03A31AA
:100FA000098801A8904702B070BD022088620448F9
:100FB00004A1084A08A308F0FDFEC04610900102F3
:100FC0007DCD00004145535F49525148616E646CCC
:100FD00065720000CE02000041455320696E7075B5
:100FE00074206F766572666C6F770D0A00000000E2
:100FF000414553206F757470757420756E64657209
:10100000666C6F770D0A0000F0B581B03B4C21276C
:1010100067723B490A8862703A490B8863713A49A2
:1010200009683A4D29603A4D2D782570120AA27050
:101030001A0AA271C3221502364E327882420FD1AB
:1010400007F0F6FD7D21C900FFF744F83348018021
:10105000307845432C48006808183149401803E0AF
:1010600045432D4828180D4645192E48056007F0C0
:1010700075FD401908F0CEF906460D462A48007B5A
:1010800008F054F8294909882222A15482B2D20BCF
:10109000801802B2D0175210B2186841130EE355EF
:1010A000130C20256355224B1B68A3761D0AE57699
:1010B0001D0C25771B0E637723462233090A5970CE
:1010C000A2771C490A604860100AE07707F0B0FD7B
:1010D00019490860134803682821012220460BF0B3
:1010E00067F81649086007F0A3FD1549086005F088
:1010F000BDFF0028FBD1002001B0F0BD40A70102D8
:10110000409D010272B301020CA601027CB30102F0
:10111000F7A3010276A60102609E01003AA6010231
:1011200060DB00007CA6010252900102449D010296
:1011300018A6010290B3010280B3010284B3010238
:1011400078B3010270477047B0B582B0194C20687F
:10115000056801A90020087007E090470198401C2D
:1011600001A90870C0B2082822D2012211048140CE
:10117000294209D02268516080002018826A002A22
:10118000ECD001A80121E8E7130283402B4201D0F3
:10119000022104E082402A42E0D003211346226863
:1011A0005360800020188268002AD7D001A8D4E7B5
:1011B00002B0B0BD60920102FEE7000010B5094820
:1011C0000168CA6920231343CB610269032A08D14D
:1011D000012293050C689C430C605102C26E0A43C5
:1011E000C26610BDD0920102F0B581B00C4806462F
:1011F0000C360068876B002403E0361D641C122C3B
:101200000CD00125A5403D42F7D031680029F4D02B
:1012100020468847024800688563EEE701B0F0BDCC
:101220005093010204217046084204D0EFF3098371
:10123000EFF3088203E0EFF30883EFF309829BB03A
:1012400004A8F0C044464D4656465F4608A8F0C084
:101250001846F0C86846F0C018690C902020184461
:101260000D9058690E9098690F90D8691090EFF31F
:1012700010801190EFF314801290094908681390C0
:1012800008490868149008490868159007490868D3
:1012900016901793189270461990684608F0A2FFAE
:1012A00004ED00E00CED00E010ED00E014ED00E0D6
:1012B000B0B50446C00703D1032005F097FA02E059
:1012C000032005F0A3FA0825284605F09FFA2846D2
:1012D00005F08CFAA00703D4032005F087FA02E09A
:1012E000032005F093FA0825284605F08FFA2846D2
:1012F00005F07CFA600703D4032005F077FA02E0DA
:10130000032005F083FA0825284605F07FFA2846D1
:1013100005F06CFA200703D4032005F067FA02E019
:10132000032005F073FA0825284605F06FFA2846D1
:1013300005F05CFAE00603D4032005F057FA02E05A
:10134000032005F063FA0825284605F05FFA2846D1
:1013500005F04CFAA00603D4032005F047FA02E09A
:10136000032005F053FA0825284605F04FFA2846D1
:1013700005F03CFA600603D4032005F037FA02E0DA
:10138000032005F043FA0825284605F03FFA2846D1
:1013900005F02CFA60B2002803D4032005F026FAE9
:1013A00002E0032005F032FA0824204605F02EFA68
:1013B000204605F01BFA0724204605F027FA2046B0
:1013C00005F014FAB0BDF0B581B00327002438460B
:1013D000214605F07DFA3846214605F089FA0125B7
:1013E00038462946224605F019FA05263846294688
:1013F000324605F0A5FA08273846214605F078FA66
:1014000038462946224605F009FA3846294632462A
:1014100005F096FA07273846214605F069FA38465E
:101420002946224605F0FAF938462946324605F0A3
:1014300087FA01B0F0BD000010B50B2005F0DEF911
:1014400015490A78002802D0002A14D010BD012ABC
:101450000ED11248002202700A7011480124047053
:1014600009F01AFE0F4964220F4B20460AF034F9A6
:1014700002F0F6F910BD0948012404700C70084808
:101480000021017009F024FE06496422064B204623
:101490000AF022F910BDC046EDA70102ECA7010237
:1014A000A493010214A50102E1B8000080B5074829
:1014B00001210170064802680A430260054802687B
:1014C000002A02D000200146904780BD12A40102EC
:1014D0001C10005014A40102F0B599B0F548017B2E
:1014E000C67A427B0E92F44C221F1368F34A1268AC
:1014F000069242780C9202790592C76A04931F40C3
:1015000001200F907A0200D5BCE03A0200D5BFE07E
:10151000FA0102D50F9802062260502508968A1912
:101520001826BB0102D50F98430623604123079577
:1015300069430A96354655431426FC0210D50F9888
:10154000040538463746DC4E3460DA4CA469B4648E
:10155000D84CE4697464DA4C241D34603E46074676
:1015600090000B90D8040D90681809900E9B73435F
:101570000F988203B902D04D22D50F9841052960FA
:10158000CC480E961646024681692965C16969658F
:1015900009990D9801430898000108180B99401803
:1015A000C018C849098892794A4380180A301C46F5
:1015B00003F0EAFB234632460E9EC04988672A6044
:1015C0000F98C404380300D52C60F80302D50F9897
:1015D000000428600F984104B80300D5296038043E
:1015E00000D4E4E1039402910E9308920D980B99B4
:1015F0000C180A980C9941430C910F98C0030B905A
:10160000286006F0B9FA002801D003F09FFB0C987F
:10161000005B410B43D1099800190E9940180599B8
:10162000090140180E90E74D287B079B4343E97A58
:101630000A010D9C2243D21841188B00D2180A9B34
:101640004B43D1186A7B564389190E9E2A7910188C
:10165000DF4A12884243881816903068C000800D17
:1016600010A9C882002511957079C0077ED110A8F5
:101670000F998182069C00940020E8A2049B09F047
:10168000C9FB78E00F98820522603A0200D43FE758
:101690000F98C2052260FA0100D53BE73DE707211C
:1016A00049030840032149038842089A00D07EE19B
:1016B000069705F003FF0020169009901590C14C85
:1016C000E07A217B08180A99414380000D9A104363
:1016D0004118627B0E9672438A186178A379079E3F
:1016E0007343D718FA683F26324063789A420C97C2
:1016F0006ED105960A9A4A4380580F210A07024084
:101700000398401EC04B1B68DB09034098181090DB
:101710000F98C0020B90B868800767D42C46283C0D
:1017200008F042FA05462068000609D5C320840166
:10173000786A400704D408F037FA401BA042F7D972
:1017400005980002B96849080140B34803688268F7
:10175000B868C40C20202040DB0700D095E00023AF
:1017600010221D461C460E9E0B9FB1E010A88582DC
:10177000B0681190069C701D924B1979E20707D151
:10178000491C1971D97A1A798A4202D31D7100E075
:10179000D97001784278120251188278120489189F
:1017A00003229143017035715878401C5870D87AE3
:1017B000197B08185978884200D85D70D879401E86
:1017C000D871596B002901D010A888477E4DEDE0F3
:1017D00010A80B998182F86830406378009000204F
:1017E0007CA20F9909F016FB0E9E94E0388A874A76
:1017F000024010A8C2822022BA5C9307DB0F3C682B
:10180000C3720F9B1A4082726205D20C0D9B1A4361
:101810001692FA68130E0372BB69FC697C4D2D6841
:101820002D0C05745204920F427211931394654C5F
:10183000A07B002809980E9E0B9F5FD0754800681A
:10184000007A0328099859D00C98007D084009288F
:10185000099853D1C320840108F0A6F905460C98D5
:10186000406A41070BD4594909680906890F06D116
:1018700008F09AF9401BA042F1D90C98406A410344
:101880000898884310A9888237E0D2070E9E0B9FE4
:1018900003D108230022154619E00C9B9A68029C8C
:1018A000224211D19A68520C02249443002213461A
:1018B00015460DE080A5010228A000503CA1005073
:1018C000FC1F00007EA501020425002213461446D9
:1018D0000843104318432843204310A98882384204
:1018E0000BD10C9B198A494A0A4010A9CA8219686F
:1018F0004905C90C0D9A11431691324C2921615C9E
:10190000002908D03037B84205D010A90846113058
:10191000123107F021FCE77A2A48047BE5192948AF
:1019200000790E9027484078401C2946FEF7D2FBEC
:1019300088000D9A104318900799614338011043AD
:1019400040182049497B4E4380191C2169434018A7
:101950000E9909191B4B1E4A12884A43801817908A
:10196000099A0C998A60987B002800D04A6298797D
:10197000401C9871187B99798142069F00D39A7117
:101980005978491C5970D97A0818597888420E4DEF
:1019900000D85A70187A401E18722820185C002847
:1019A00004D0996B002901D010A88847089A1742E3
:1019B00002D00F98000328601C480449486019B001
:1019C000F0BDC04680A5010228A000503CA10050F7
:1019D0007EA501024857204554206964782025647B
:1019E00020616E6420455420696478202564206954
:1019F0006E2052582064657363206D69736D617445
:101A000063680D0A0000000038200040FF0300005A
:101A100094300040BC930102604000404D4143209F
:101A20004556542025782025780D0A00FFFFFF0336
:101A3000F0B5A5B01E460C9208910024239422A96B
:101A40000C8016A90C8024A909250D80598C0D91B4
:101A5000FEF740FB2A99012900D0DFE031890129F6
:101A600000D0DBE0318C012900D0D7E00D990029AE
:101A700000D1D3E0224607962C990B912B99069121
:101A800080B205900F9415A8058090000E900C99D7
:101A90000C582E460025204629461746FEF7AEFD77
:101AA0000028119636D12C200A97784308990818F7
:101AB00017A90A4668C868C2E8C8E8C2E8C8E8C208
:101AC000079F119880B280000E5822AD019523A87F
:101AD000009020463946059A069B02F083FE0F9837
:101AE000401C0F90288800282DD03B8A239913ACE6
:101AF000039416A8029014A8019015AE009617A89A
:101B000024AA03F049F82588308811900120149EFA
:101B10000A9A05E013A8058014952E4628463A46F1
:101B20000E9F51000B9B119C5C52591808830D8429
:101B3000D81986600F981885521C0D9882426DD076
:101B400024A805889FE7099616A800250580149506
:101B500024A80688239812902F46109503E06D1C48
:101B6000A8B2B04213D8A8B2800017A90C582046DA
:101B70001299FEF751FD0028F1D1002FEFD115A8E1
:101B8000058016A80127078014941094E7E715A88C
:101B90000288B01A012805D115A80680099F14975C
:101BA000119628E010200799095E0129119221DB86
:101BB000551CA8B20C18109F0E9B099403E06D1CD5
:101BC000A8B2844218DDAAB2B242F8D8800017AA9F
:101BD00010581090394634461E46FEF70FFD334626
:101BE0002646099C0028EAD115A80580109F149765
:101BF0001195E4E7109F0E9B1C463E46384612990D
:101C0000FEF7DEFBFEF778FD0546052800D3052527
:101C100013A8058001200A9A274682E725B0F0BD67
:101C2000F0B58BB00243159A149C139E2BD0054639
:101C300001A856C0129CD869196A09900A911E46DB
:101C40009F6B0123009309A807AA0146059304F09E
:101C50009DFE716C3846FEF7B3FB0746E06A616B88
:101C6000FEF7AEFB002D069613D00446119801999D
:101C7000012924D10921081A0421069A515E8842BB
:101C800029D16425B1E000203080207010700BB0A5
:101C9000F0BDB08800226425002829D0059269494A
:101CA0003846FEF7D5FC0028049C039E6FD1664998
:101CB0003846FEF7CDFC00281DD05A2567E03C25AC
:101CC000082800D191E05F492046FEF7C1FC0028BA
:101CD00019D0502589E00A291DDB1D293BDC594913
:101CE0003846FEF7B5FC0022002854D05A253AE0C9
:101CF0003346049C39E055493846FEF7A9FC0028D4
:101D000021D0502543E050492046FEF7A1FC002891
:101D10002ED0462569E03C25012866D04949204659
:101D2000FEF796FC0028D4D147492046FEF790FCE8
:101D30000028EED145492046FEF78AFC002854D100
:101D4000434920466EE042493846FEF781FC0028B0
:101D50001CD128251BE03B493846FEF779FC0022C0
:101D6000002832D05025049C069B0299039E41E036
:101D700036492046FEF76CFC002836D1344920460F
:101D8000FEF766FC00282FD114252EE03725029996
:101D9000059A069B2EE005922B493846FEF758FC23
:101DA000002896D129493846FEF752FC0028B0D1C8
:101DB00027493846FEF74CFC0028049C069B0299F4
:101DC000039E059A3BD11E2514E005921E49384614
:101DD000FEF73EFC00289CD11C493846FEF738FC33
:101DE00000281DD03C2500E02325049C069B029979
:101DF000039E059A258032700020087030780028F4
:101E00000CD118681349FEF715FC002806D120886C
:101E1000102803D30F3820800BB0F0BD0BB0F0BDFD
:101E20000B493846FEF714FC0028049C069B0299D7
:101E3000039E059A01D11425DCE72325DAE72D2539
:101E4000D8E7C046CDCCCC3DCDCC4C3DCDCCCC3C68
:101E50000AD7233C0000204070B588B00C460646E7
:101E60004088002820D0FEF731FC059005A804A981
:101E700001252A4604F0F4FF3088B188081AFEF7DD
:101E80001AFC0390049903A807AA2B4604F0A8FFA4
:101E90005249079D2846FEF7DBFB002808D0BF20EB
:101EA0000006206008B070BD0020206008B070BD42
:101EB0004B492846FEF7B0FB002804D03F2000061F
:101EC000206008B070BD47492846FEF7C1FB0028D6
:101ED00001D0002010E000212846FEF7B9FB0028C1
:101EE00001D0022008E040492846FEF7B1FB002857
:101EF00001D0042000E0062001957F21C905029150
:101F000080003A49091801A806AA022304F01CFF20
:101F10000698206008B070BDF0B587B00C46054645
:101F20004768002638463146FEF7A0FB002802D05D
:101F3000266007B0F0BD049704A803A90126324625
:101F400004F08EFFA8682968FEF7F5F9029003995E
:101F500002A806AA334604F043FF2049069D2846FE
:101F6000FEF776FB002804D0BF200606266007B0E7
:101F7000F0BD1B492846FEF74FFB002804D03F2048
:101F80000606266007B0F0BD16492846FEF760FB3E
:101F9000002801D0002010E000212846FEF758FB61
:101FA000002801D0022008E00F492846FEF750FB28
:101FB000002801D0042000E0062000957F21C905FB
:101FC0000191800009490918684605AA022304F016
:101FD000BBFE059E266007B0F0BDC046CDCC0C3FD1
:101FE000295C0FBFCDCC4C3ECDCC4CBEC49301027E
:101FF000F0B587B00C4606467F270088002801D040
:10200000FD0503E0B08800282ED0334DFEF75EFBBF
:1020100003907088FEF75AFB049003A802A90126DA
:10202000324604F01DFF029904A806AA334604F0C4
:10203000D7FE2A49069E3046FEF70AFB002802D04A
:102040003F20010641E026493046FEF7E5FA002828
:1020500002D0BF20010638E022493046FEF7F8FAE8
:10206000002805D0002024E00020206007B0F0BD4B
:102070001D493046FEF7ECFA002801D0022018E096
:102080001A493046FEF7E4FA002801D0042010E097
:1020900017493046FEF7DCFA002801D0062008E098
:1020A00014493046FEF7D4FA002801D0082000E099
:1020B0000A200096F905019180000F490918684629
:1020C00005AA022304F040FE05992846FEF73BF9D5
:1020D000206007B0F0BDC046000080BF000038435C
:1020E0003333733F0000C8420000704200002042BA
:1020F0000000A0410000C040E4930102F0B59DB093
:1021000015460B917F210391C9051C9102911B91EA
:1021100019A900248C80199418941794598C06914D
:10212000198C0F91DE8B998B0791997805911F88F7
:102130002B21CA432799914201DB7F0015E0402201
:10214000D243914211DC4922D243914202DB790809
:10215000CF190AE05322D2439142EEDA5D22D243F4
:10216000914201DBBF0000E0FF000A971396269E14
:10217000597E00290BD0002132460F46D170917054
:1021800051701170121D7F1C5C7EA742F6D30C9318
:1021900011952599149122990D91159041088C4221
:1021A00011D2FD4A2346A00084583454270A451C06
:1021B0007755250C871CF555240EC01C34545B1C28
:1021C0009CB2A142EFD82398109001200990009072
:1021D00030463146149A159F3B4604F0E5FB0D98B6
:1021E00000060890400E139D00D186E06800049020
:1021F000002F3FD0002210461146144606E01C4630
:102200001146159F401C82B2BA420ED283B2AB4235
:10221000F8D09200149B9A5E0FB2BA42034600DCDB
:102220002346BA42EBDC0A46E9E7002F25D000221C
:1022300010461146129206E012931146159F401C5B
:1022400082B2BA4214D283B2AB42F8D0A5B2AB424A
:102250000CD09200149B9A5E0FB2BA42034600DC87
:10226000129BBA42139DE7DC0A46E5E7139DE6E7B9
:10227000129903E00024214600E0002112911098F9
:102280000183C4828582049FF057FEF714FA7921F6
:10229000C9050E91FEF757F81099C86109980743D0
:1022A000F057FEF708FA0E99FEF74DF8109F3862C6
:1022B0002004C40B3057FEF7FEF90E99FEF743F8E1
:1022C0007862601C3056FEF7F6F90E9C2146FEF748
:1022D0003AF8B86212980004C70BF057FEF7EBF912
:1022E0002146FEF730F8109CE062781C3056FEF76D
:1022F000E2F90E99FEF727F82063119805800C98F3
:10230000407E410000278D4228463A46149E1ED347
:102310000A9880B28AB29300F45E84420BDA491CB8
:102320008AB2AA42F6D9002728463A4681B2691AEB
:10233000012910D01BE0F018119B198007880804B0
:102340000FD0500040008019001F0288084681B25B
:10235000691A01290BD1A800301811990D8007883E
:1023600026E00020024681B2691A0129F3D00A99B9
:1023700089B2079B4B43BB421AD306998A4217D8AE
:102380000599002914D0401C82B2891803E0401C32
:1023900082B291420CD983B2AB42F8D89200B35EBC
:1023A000BCB2A342F3DDB218119B18801788EEE788
:1023B00012970B980580119800882B1A002B16DDB8
:1023C00002210F9A1143032942D10E93411C421E50
:1023D00010B281420EDA0E98032824DB0C98808C10
:1023E000012820D019A818A9FFF736FD1FE000200A
:1023F00018902BE00026F443374608E0B8B24000BE
:1024000019AD2B527F1C521C10B28142E3DB13B278
:10241000A3423346F2DD159B98423346EEDA800044
:10242000149B1B5AEAE719A818A9FFF7E1FD149EAF
:10243000139D0F9A012A13D0032A11D0022A04D126
:1024400011980088281A02280ADA0020179034E030
:10245000022A01D1022BB8DA00201890012AEBD110
:10246000681C691E0FB2B84208DA0C98808C0128EB
:102470001DD119A817A9FFF7BBFD1CE00022D3430B
:10248000144608E0A5B26D0019AF7E53641C491CC8
:102490000FB2B842E9DB0DB29D421646F2DD159D42
:1024A000AF421646EEDABD00149E765BEAE719A845
:1024B00017A9FFF7D1FC149E139D249F189C179910
:1024C0002046FDF738FF0F99012900D820463860D3
:1024D0000D98002800D1CBE011990888109FB8868C
:1024E0000888281AB880129880B2FEF7EFF8792190
:1024F000CC052146FDF727FF2146FDF724FFB863F1
:10250000119F3888002849D081008919091F09883E
:10251000129C0C191599884203D28000801980887A
:10252000041915984300534916AA304604F01AFCC2
:10253000169810994864FEF7F8F8A4B2A04201D1A9
:102540004D480FE0001BFEF7C1F81C901CA81BA90A
:10255000012204F085FC2046FEF7B8F801461B98DE
:10256000FDF7F1FE109908603988491B4A1C92B2A8
:10257000032A02D20021159F17E009B20229159FF4
:1025800012DB3F210906FEF763F8002802990CD1FF
:102590000998810709E0C046402100400020129CB4
:1025A00015998842B9D3BCE734491098016108985D
:1025B000800E5DD0002F1CD000221146144610461C
:1025C0004B1B1DB2ED135B196B40139D1BB29200A8
:1025D000B25E53431818A418491C8AB2BA42EFD30A
:1025E000FEF774F806462046FEF770F8002C03D17B
:1025F00000E000260398C0051C901CA81BA901251B
:102600002A4604F02DFC1B9C20463146FDF79BFE1C
:10261000014610988160002F119422D00024274693
:10262000264613951291B8B2FEF750F81299FDF7AD
:1026300082FE0546A0001499085EFEF73CF80146AC
:102640001398C00785432846FDF77DFE01463046B6
:10265000FDF720FE06467F1CBCB215988442E2D3EB
:1026600000E0002611983146FDF76DFE1099C86014
:102670001DB0F0BD809D01020000204100004040DF
:10268000F0B58FB00692F74A09AF70CA70C770CA2A
:1026900070C70328079320D88800F3A10858F6498B
:1026A000FDF7F8FD0446F549FDF7F4FD0D90F449FA
:1026B0002046FDF7EFFD0C90F2492046FDF7EAFDBC
:1026C0000B90F1492046FDF7E5FD0A90EF492046C1
:1026D000FDF7E0FD0990EE4969E0042822D00628C4
:1026E00020D88800EBA10858EE49FDF7D3FD044639
:1026F000ED49FDF7CFFD0D90EC492046FDF7CAFDF1
:102700000C90EB492046FDF7C5FD0B90E9492046AA
:10271000FDF7C0FD0A90E8492046FDF7BBFD099092
:10272000FD4944E00838022821D88800FBA1085858
:10273000D149FDF7AFFD0446FC49FDF7ABFD0D9017
:10274000FB492046FDF7A6FD0C90FF2081052046A1
:10275000FDF7A0FD0B90F7492046FDF79BFD0A9081
:10276000CA492046FDF796FD0990FE491FE0880002
:10277000F1A10858F449FDF78DFD0446F349FDF732
:1027800089FD0D90F2492046FDF784FD0C90F1493A
:102790002046FDF77FFD0B90EF492046FDF77AFDBF
:1027A0000A90EE492046FDF775FD0990EC4900942A
:1027B0002046FDF76FFDEC4909680E90EB48046870
:1027C000EB4801684808EB4F05463D400022002DCC
:1027D00008922DD0CA01120E07D0280CE90D12D193
:1027E0004000E649085AE6490AE0C903090E0CD040
:1027F000280AE90B10D14000E049085A8F218900CE
:102800004018E4300DE0DC490AE081B27F2905D8A8
:102810004800DA49085A04E0D94901E08F218900CB
:10282000401800B2FDF747FFD649FDF78CFD024680
:102830000292039507252606D34B1A68002A0898AA
:1028400040D0791C8A420BD21102090E13D0110C10
:102850001F46D00D1FD14800C849085AC84907E093
:102860001F46110E002A13D44800C449085AC24911
:102870004018E4301FE011041F46090E0ED0110A63
:10288000D00B12D14800BD49085A8F218900EFE7CB
:10289000BE4808180FE0B84808180CE091B27F292C
:1028A00006D84800B549085A05E0B548081802E0BE
:1028B0008F218900501800B2FDF7FDFEB149FDF7E8
:1028C00042FD3B460590159F2C40F50E5B69B049D3
:1028D0001940089810D0DA02D20E34D0C80B3E212D
:1028E0000140A648405AA6494018E43000B2FDF71E
:1028F000E2FEA449FDF727FD0490149E6800A5A1FF
:10290000085EFDF7D8FE0146A00009AA1058FDF7A1
:10291000C1FC0146B8B20128089F019102D1022CE6
:102920000AD9A74F052C24D1189808900C2D20D82F
:102930000B2D16D3A44918E00027022C089718D0B5
:102940008120C70515E01A04120E00D1CAE0080A5A
:10295000C90B00D0CDE040008849085A8F2189007A
:10296000C2E7092D00D2C7E096490898FDF792FC0E
:10297000089001200021B542034600D30B46052CE8
:1029800000D308461799169A1A9C199D1843069B5E
:10299000012B12D1079B402B22D1002840D0384672
:1029A000FDF778FC01460198FDF774FC014600989C
:1029B000FDF7C1FC059A04998AE0079B402B1FD1C3
:1029C000002838D03846FDF765FC01460198FDF730
:1029D00061FC01460098FDF7AEFC059A049977E08A
:1029E000002833D03846FDF755FC01460198FDF725
:1029F00051FC01460098FDF79EFC059A049967E09A
:102A000000285BD03846FDF745FC01460198FDF7EC
:102A100041FC01460098FDF78EFC059A049957E0A9
:102A200002981146FDF787FC0399002900D16748F9
:102A3000059A04994CE002981146FDF77CFC039935
:102A4000002900D16148059A049941E00298114695
:102A5000FDF771FC0399002900D15C48059A04999F
:102A600036E0C0460CC30000000068C1000088C109
:102A700066665EC1000084C1000084410000B4416C
:102A800000004841000020400000F0C0000084C168
:102A90000000F841333323C1000050C19A9929C185
:102AA0009A9949C19A9949413333CB416666764137
:102AB000CDCCAC40333393C09A9949C102981146AA
:102AC000FDF739FC0399002900D14048059A049983
:102AD00028601046FDF72FFC0899FDF72CFC2060BC
:102AE0000FB0F0BD99B27F2911D848002349085A88
:102AF000FCE623494018F9E6C12001060898FDF7D5
:102B0000C9FB0890062D00D933E7002030E78F215C
:102B100089005818EAE6C0463333F341000058C133
:102B20009A9961C19A9969C1000084C10000AC41C1
:102B300000003841000008C1CDCC80C1CDCC88C197
:102B400033338FC1333397C133339741CDCC8C416D
:102B50003333F3409A9919C0666646C1333397C13F
:102B6000CDCCB4410000D4410C00004050300040B6
:102B700068400040FFFFFF007C08000080C60000A6
:102B80005C050000919AF63C642000409C0B00001C
:102B9000FFFF1F00FAFFFCFFFEFF00000200040021
:102BA000060008000A000C000E00100012001400BD
:102BB000160018001A001C001E002000220024002D
:102BC000000080BF0000A0C0000040C00000DCC2C8
:102BD000F0B5FFB0ECB017460E460D900021E9911C
:102BE000E891DC9199919891979196911491139114
:102BF00012919AA8F49DF39CF29A002E00D1E6E17E
:102C00000B938030F09B1180099529602546DBAC41
:102C1000218095AC21800C952980DA917F24E405F0
:102C2000B994B894B794B694B594B494B394B29458
:102C3000B194B094AF94AE94AD94AC94AB94AA9488
:102C4000A994A894A794A694A594A494A394A294B8
:102C5000A194A0949F949E949D949C949B949A94E8
:102C6000046644668466C466046744678467C46710
:102C7000046444648464C464046544658465C46510
:102C8000046244628462C462046344638463C46310
:102C9000046044608460C460046144618461C46110
:102CA000B0090B250B2800D3AE011095012B0B9D0D
:102CB00000D070E12B89012B00D06CE1298C002918
:102CC0000E9200D18BE16B8C002B00D1FAE1AA8C23
:102CD0003021695C002900D188E10892109F5F4390
:102CE0001196304639460F93FDF7F4F90590FDF73C
:102CF000E2FC01462046FDF763FB8321C905FDF791
:102D000022FB064696A8021D119887420A9200D817
:102D100079E155A811909AA9069196AF15463A46C1
:102D2000059C234604F010F815A80F9006992A4632
:102D3000234604F009F802230D93384631463A46FB
:102D400004F04EF8012308930093E8AA1092384645
:102D5000394603F01BFEE898DD901198069D294640
:102D60003A46234603F0F0FF0F9829460A9A234675
:102D700003F0EAFF384631463A460D9B04F030F83E
:102D8000089B009338463946109A03F0FFFDE898F7
:102D9000DE9011982C4629463A46059D2B4603F0B5
:102DA000D3FF0F9821460A9A2C462B4603F0CCFFFE
:102DB000384631463A460D9B04F012F8089B0093C2
:102DC00038463946109A03F0E1FDE898DF901198F3
:102DD000069D29463A46234603F0B6FF0F9829463A
:102DE0000A9A2346254603F0AFFF384631463A4655
:102DF0000D9B03F0F5FF089B009338463946109A67
:102E000003F0C4FDE898E0901198069C21463A46EC
:102E10002B4603F099FF0F9821460A9A2C462B4621
:102E200003F092FF384631463A460D9B03F0D8FF37
:102E3000089B009338463946109A03F0A7FDE8989E
:102E4000E1901198069D29463A46234603F07CFFFF
:102E50000F9829460A9A2346254603F075FF3846FF
:102E600031463A460D9B03F0BBFF089B0093384662
:102E70003946109A03F08AFDE898E2901198069C72
:102E800021463A462B4603F05FFF0F9821460A9AE7
:102E90002B4603F059FF384631463A460D9B03F066
:102EA0009FFF089B009338463946109A03F06EFD49
:102EB000E898E390119821463A462B4603F044FFE8
:102EC0000F9821460A9A2B462C4603F03DFF3846C0
:102ED00031463A460D9B03F083FF089B009338462A
:102EE0003946109A03F052FDE898E4901198069D37
:102EF00029463A46234603F027FF0F9829460A9AA7
:102F00002546234603F020FF384631463A460D9BBE
:102F100003F066FF089B009338463946109A03F089
:102F200035FDE898E5901198069C21463A462B46D7
:102F300003F00AFF0F9821460A9A2B4603F004FF7C
:102F4000384631463A460D9B03F04AFF089B0093F2
:102F500038463946109A03F019FDE898E690119822
:102F600021463A462B4603F0EFFE0F9821460A9A77
:102F70002B4603F0E9FE384631463A460D9B03F0F6
:102F80002FFF089B009338463946109A03F0FEFC49
:102F9000E898E7907AE010880C9A108099919891BF
:102FA000DA9E08460F46099DF59CFDF7C4F9286096
:102FB000DC9827606060A6600C34DDA80EC80EC4E3
:102FC0002EC82EC42EC82EC47FB06CB0F0BDFF201A
:102FD00010800021296020807FB06CB0F0BD0022FD
:102FE00001233021695C002900D076E6DDAA1ACFE2
:102FF0001AC23ACF3AC23ACF3AC20B213046FDF755
:1030000069F8054642E000200690059D0796089F56
:103010001190069801460D9C0F9A4A43D219109BB5
:103020005A43119BD218D200A35889002E4655ADA1
:103030006B503546121DA25815AB5A50401C01B2B8
:103040008E42E9DC55A89AAE96AC314622462B4614
:1030500003F07AFE15A831460A9A2B4603F074FE57
:10306000022320460799224603F0BAFE012300936B
:10307000E8AA2046214603F089FC119B9800DDA9AF
:10308000E89A0A505B1C0B2B1846C1D1F19EDDA8B3
:103090009AA9DCAA0B2303F057FE09210E980F9181
:1030A00001800B98C168DC9C2046FDF74CF9014675
:1030B000A8B2E69F0F281BD808280DD30846FDF7B5
:1030C000E9F814E0FF2010800021099A11600C99A2
:1030D00008807FB06CB0F0BD042803D3812208467D
:1030E000D10502E0412208461106FDF72CF9014600
:1030F0002B20C04386420D9704DB0846FDF7CAF833
:10310000014603E04020C043864244DD0E9A0C9CF9
:103110000B98408A002811D00B98038A95A8039039
:10312000DBA80290DAA801900094DDA80D4601F01A
:1031300033FD29462488DA9E099D68E011910F9895
:10314000208000273D46109705E00E9804887F1CDC
:10315000B8B2A04211D8B8B28000DDA90C58204600
:103160001199FDF759FA0028EFD1002DEDD10C98F7
:10317000078001250F971094E7E7DBA805800F9AD9
:1031800090B2201A012811D10C9804800D9FDA9773
:103190003E46099D3AE04920C043864200DA8BE072
:1031A000FF2208469105FDF7CEF8A9E710200B99FC
:1031B0000E5E012E00DA90E0551CABB21846A1B2AB
:1031C000AAB28A4217D805E00E990C88A1B2AAB219
:1031D0008A4210D88000DDA90C58204610991F465D
:1031E000FDF70CFA3B46002805D10C9805800B989A
:1031F000068A0F95109430B2C1186D1CA8B2814296
:10320000E2DC109EDA960F9C099D0D9F11993046C5
:10321000FDF7D6F8FDF770FA052800D3052095A92B
:103220000880A0B20E990988814218D9401C611EFD
:103230000CB2A04218DA12A898A9FEF76DFE0E98FB
:103240000188481C491E0CB2A04221DA12A899A993
:10325000FEF762FE99999898099D0D9FA4E60021BA
:103260009891999108469FE60022134608E09CB287
:10327000A40012AF3D515B1C491C0CB2A042DADB2A
:103280008DB20A2D1546F2D8A400DDAD2D59EEE71A
:103290000022134608E09CB2A40012AF3D515B1C13
:1032A000491C0CB2A042D1DB8DB20A2D1546F2D8D2
:1032B000A400DDAD2D59EEE75320C043864200DB6C
:1032C0001BE70E460B9881692046FDF797F9002809
:1032D0000C9C08D10B98808B07E01446099D0D9F2C
:1032E0001199109E93E70B98C08BFDF7EFF90146FB
:1032F0003046FDF728F8119021E70000F0B58BB0BB
:103300001C4609930E46034600200A904048008858
:10331000224F05970AA9049103940292109C0194EC
:10332000012500950B21414389B230331C4A3046B8
:10333000FFF74EFC3868079078680890B8680690E8
:1033400033480088334F009501940297324E30364F
:103350003249334A3346FEF76BFB0698F86207980A
:10336000386308987863099800882E4905912E499A
:1033700004912E4903910297019000962C4B284608
:1033800029462A46FEF74CFC432001060A98FCF722
:10339000DAFFFDF7B1F90BB0F0BDC046489D010260
:1033A0002CB30102F0B589B00F9F0E9C002815D0F8
:1033B0001098079016480088164E01250095019137
:1033C00002960893144B30331449154AFEF730FB2C
:1033D000089BF76207983063746303E00D48476306
:1033E000C462002518880F4905910F4904910F49BF
:1033F0000391084902910190074830300090012163
:103400000B4B28460A46FEF70BFC09B0F0BDC04640
:10341000F8A30102F0A701029C960102B4950102F3
:10342000C0A50102709A0102E0A301028CA301026F
:1034300094A3010280B5124801681F220A4002606D
:1034400003200840022812D10E480268D30D02D092
:10345000FF231B06D2180C4B1A600C4A12680C4B47
:103460001A6080680B4A1080000C0B4A10801A48C2
:103470008268002A02D082680020904780BDC04642
:103480007420004064400040D4A501027830004020
:10349000D8A5010200970102E0A7010280B50D48FE
:1034A000016889070FD5052101600B48C178002903
:1034B00008D00021C170C168002903D0C2684168EA
:1034C0000020904780BD054805A10B4A0BA306F0DC
:1034D00071FCC0462C040040AC93010252D20000A3
:1034E0005048595F54494D45525F49525148616EA9
:1034F000646C6572000000008D0A0000556E6578EE
:1035000070656374656420696E7465727275707439
:103510000000000070B50446401E012814D80320A6
:10352000084011D13F2040030818050B28198028B6
:103530000AD8164E317801204840294602F04AFA4E
:10354000641E6D1C002CF5D170BDC04680B50020F6
:10355000014601F0D9FF002800D080BD0B480121B1
:10356000017080BD70B516460C460546FF22FCF77B
:10357000EDFD0548311805480278012050402A46E3
:10358000234602F0CFF870BD00E00704849F0102DB
:10359000012000037047012040037047F0B583B05D
:1035A0002E480068C16B0901890F01D003B0F0BD3E
:1035B000C16BC06B2A4D05404800400F082602969B
:1035C00086400227384601F043F801907043C10B52
:1035D0004A1B24485043FCF793FD044606F04AFA80
:1035E000032121A238461D4F0091234607F012FC0B
:1035F000F88A002814D0019840012946FCF76AFD9A
:1036000046431822324001200F2A014600D80021EB
:1036100073095B18194CA3420AD8174DED1A08E03C
:1036200038680021C160112001F002F803B0F0BD3C
:103630005D1C6D050F2A00D956422A0C029D2E40B2
:1036400009018919A34202D80098000400E040044F
:10365000081880183968086303B0F0BD3C94010273
:10366000FFFF1F0040420F0052434F33324B207088
:10367000706D2025640D0A00FF070000FE7F00002A
:10368000B0B582B0154908688269D2070CD0012212
:10369000C2610D69002D07D000686C46214605F017
:1036A00051FF00212046A84702B0B0BDB0B582B09E
:1036B0000A490868026C92070ED5026C0123134375
:1036C0000364CD68002D07D000686C46214605F0E4
:1036D00039FF00212046A84702B0B0BD3C9401024A
:1036E00007480168032291430160016801220A43EF
:1036F000026008F09DFA00F07FF806F0DFF9C0469E
:103700002800004080B50E480168002911D52349E2
:1037100009680422032901D0114300E01146016029
:103720001F480268002A03D01E4801680020904705
:1037300080BD04A00CA19E2211A306F03BFBC04655
:103740002C100140696E636C7564652F6472697634
:103750006572732F6D6B5F736C6565705F74696DF7
:1037600065722E6300000000534C4545505F54497C
:103770004D45525F49525148616E646C657200005C
:10378000556E657870656374656420736C656570EB
:1037900020696E7465727275707400005494010231
:1037A000E8A7010258940102B0B582B0044600783F
:1037B000002811D0094D01A908702868416A002924
:1037C000FCD101A901220020034608F095F8611CF4
:1037D000607800280C46EED102B0B0BD80940102A2
:1037E00080B504480168491C01600069002800D0C8
:1037F000804780BD58B3010201480249016070470B
:10380000089001020026B80380B582B00E4908680E
:103810000022C2600192CA68002A02D0016801A891
:10382000904702B080BDC04680B582B006490869A5
:103830000022C26001220192CA69002A02D00168F6
:1038400001A8904702B080BDA892010280B5002077
:1038500007F04EFD80BD80B5012007F049FD80BD19
:10386000F0B581B002F04AFF1A4C20601A4909787D
:10387000002901D001B0F0BD184A11780029F9D112
:1038800001211170002821D06426301A144F3968A4
:10389000814216D0144D38681249085C296888475F
:1038A0003868401C38603868642801DB00203860C4
:1038B00021683868022E04D36422511A761E884289
:1038C000E9D100200549087001B0F0BD002010705A
:1038D00001B0F0BD6C9A01027DA501027CA5010238
:1038E00078A5010214A5010288950102B0B582B045
:1038F000602833D0622843D0642854D101A82F49CE
:103900000180EFF3108072B600242046214601F0BA
:10391000FBFD2B4D002805D1012002030020294684
:1039200001F04EFD103501AA02232046294602F07F
:10393000BDF962B623A0FFF737FF64201B490C5284
:1039400005F046FF1A4800F03FFFBFF34F8F1948BC
:1039500019490160BFF34F8F00BFFDE76020134995
:1039600000220A5205F034FF114800F02DFFBFF38A
:103970004F8F104810490160BFF34F8F00BFFDE724
:1039800062200A4900220A520A8005F021FF0848F5
:1039900000F01AFFBFF34F8F064807490160BFF3DD
:1039A0004F8F00BFFDE702B0B0BDC046869F010249
:1039B000A08601000CED00E00400FA05AAAA0000B0
:1039C00000D00204BDF8C8EBC9FDBCB6C4A3CABD93
:1039D0000D0A0000F0B5D1B09F49097800291ED02A
:1039E0009E4F396808294CD88A0001A39A589746F7
:1039F000153A0000833A0000833A00008F3A000035
:103A0000B93A0000C13A0000C93A00009D3A0000EE
:103A1000D13A0000552800D0B1E00120ACE09B492C
:103A20000978002900D19DE0994D2A789949885458
:103A3000994E31783070994F3970521C2A700A288B
:103A400000D08FE00D2900D08CE003A8019037A8AA
:103A5000009090489249934C1DAB2246FCF788FB9E
:103A60009149086091A10522204603F0BDFF00287E
:103A70003DD090480021016041608F480160416065
:103A80005BE0AA2870D101296ED1022074E074494C
:103A900000220A707349087004206DE074490A78A6
:103AA000744B9854501C08706E490978491FC0B275
:103AB000814257D108205FE0052139606A49C7E09B
:103AC000062139606649C3E0072139606749BFE0D4
:103AD0006449097806295AD34A1F0024654D2346B4
:103AE0002E5D9B199BB2641C9442F9DB50E01DA82B
:103AF0000024214605F0ECFF6E4A03C237A8214698
:103B000005F0E6FF6C4F03C703A8083F00F0D6FAA4
:103B10006A49086003CF614F22462346FCF7B4FD93
:103B200000280AD1634903C900221346FCF7ACFD03
:103B3000002802D1624800F0CBFA56489621FCF7E3
:103B40000CFB1DA864242146FCF707FB37A821467F
:103B5000FCF703FB03A82146FCF7FFFA00203870AE
:103B60002870307051B0F0BD032808D1022906D169
:103B70004148012101700320386051B0F0BD384840
:103B80000021017039603748017051B0F0BD002349
:103B900018184118344800780918314B1D78491914
:103BA000324A14780919344A1278002A00D0C91C04
:103BB000C9B2FF2946D1012819D0022842D1304884
:103BC00040192C4E31462246FCF7AEFA30780128D7
:103BD00002D12846FFF78AFE05F0FAFDBFF34F8FAA
:103BE000284829490160BFF34F8F00BFFDE7234EEE
:103BF000B47103203071B070AA20707055203070FD
:103C000068087071651DF57040001D490918F01DA8
:103C10002246FCF789FA301DE11CEAB2D21C037877
:103C200092B2D218401C491EF9D1A019D143C171DA
:103C3000090A01720934012000233146224607F0A7
:103C40005BFE074B00201870386006490870084971
:103C5000087051B0F0BDC046ECA701029495010276
:103C60008F950102909501020C9001028E95010240
:103C70008C950102B0A401029195010224950102E4
:103C8000869F01020CED00E00400FA05A4930102F6
:103C90008D95010218A40102AFA40102AEA4010295
:103CA00074D00000E1A3010264960102474E474729
:103CB00041000000B8BB010200A4010220A60102DD
:103CC000F6A3010280B582B0002001900448C268CA
:103CD000002A02D001A80021904702B080BDC04652
:103CE00010950102F0B583B000242046FFF72EFCAA
:103CF000FFF751FC284F3860FFF74AFC274908605E
:103D0000274E0BE001A8C1888088084319D101A87B
:103D10004088241808343868844238D201AD08211C
:103D200028462246FFF71EFC28880028EAD0B04229
:103D30002DD001AD0421284600F030FDA98888422D
:103D4000E5D0184E3460386884420BD201AD0221B0
:103D500028462246FFF706FC28881149884201D0F0
:103D6000A41CF0E70D4F38682118491E4042084056
:103D700030600BD00024254601202946FFF7CAFBFE
:103D80003868451930688542F6D300E000240548BC
:103D9000046003B0F0BDC046C8BB0102C4BB010251
:103DA000FFFF0000C0BB0102F0B585B01F460492C2
:103DB0000646C8170C1844400A2C039109D3012564
:103DC0000A212046FCF786F96D1C632C0446F7D8BF
:103DD00000E0012504998D4200D329460A9C002F5A
:103DE00004D00398002803D4002202E0002205E05A
:103DF0000122042323409B081343FA1A0223234081
:103E000004980028029412D1002B10D0F468002CE2
:103E10005FD40398002822D40298400731D57068F7
:103E2000B5686F1C87422CD830682B2420E0E4074B
:103E3000ECD1002A0AD1E9E7376820203855B5606F
:103E4000F068441CF460521E002CDFD49142DDD295
:103E50007768B468651CBD42EED9F468F3E7404268
:103E600003907068B5686F1C87420AD830682D24AB
:103E70004455B760F068441CF4600025ED43A84247
:103E800027DB002B1CD00120029B1840049B184309
:103E900016D1002A03D113E0521E002C0ED49142F9
:103EA0000CD27068B3685D1C8542F5D83068302448
:103EB000C454B560F068441CF460EDE7002C08D4ED
:103EC0000092029801900A2230460399049B00F068
:103ED00003F805B0F0BD0000F0B587B01F461546E9
:103EE0000290012406919142009407D30124069880
:103EF0002946FCF7EFF8641CA842F9D20D980C9AF9
:103F0000BC42039700D3039400990140002A00911A
:103F100009D00029029C07D1202180075FD40846E0
:103F2000002F6BD05EE0029CE068002855D405901D
:103F3000012401E07F1E6C43022FFBD2069821462C
:103F40001646FCF7C7F83246A842F4D202988068B9
:103F50000490069F0195069738462146FCF7BAF86B
:103F6000049D691C029F7A68914202D9069F059AB6
:103F700009E0284A125C3B685A55B960FA68521C3D
:103F8000FA600491069F019D0592002A08D46043BF
:103F90003F1A20462946FCF79DF8AC420446DAD287
:103FA00000980028029C059B049D16D0002E14D07A
:103FB000701C01E0002B10D4401E039981420CD2EA
:103FC000691C62689142F5D8226820235355A1608C
:103FD000E268531CE3600D46ECE707B0F0BD30200B
:103FE000002F0BD0084609E023685854A260E1680E
:103FF000491CE1603246721E002995D40399914212
:1040000092D216466368A1684A1C9A42ECD9E168CC
:10401000F0E7C046B8C5000070B5002801D0012007
:1040200070BD0C461625284600F00AFB284605F010
:104030007BFA002C05D01948183014222146FCF7D1
:1040400073F828211548415C002923D041680029D4
:1040500013D403220B469343124A9C588D07ED0E4E
:10406000FF26AE40B4439C501F220A4001219140DC
:104070000D4A11600D4A11600CE08A07D20EFF2331
:1040800093400F220A40083A03218A4304495458B6
:104090009C43545001210161002070BD1090010229
:1040A0001CED00E000E400E080E200E000E100E060
:1040B0005A21014A505270479C96010280B503492B
:1040C000096884228958884780BDC0460090010253
:1040D000F0B581B004460078C043207023480078D2
:1040E000C001234909788901014322480078400131
:1040F0000843214909780901014320480078C0009C
:1041000008431F4F3978890001431E4D287840002D
:1041100008431D4E31780143C8B2FDF7C9F8642049
:1041200000F052FB2078C043207010480078C00196
:104130000F490978890101430E480078400108437E
:104140000D490978090101430C480078C000084373
:1041500039788900014328784000084331780143C9
:10416000C8B2FDF7A5F801B0F0BDC046B295010296
:10417000F5A30102A5930102B4BB0102F6A301025B
:10418000B39501026899010269990102B0B5094D20
:1041900028600B24002120460A4602F03FFB012143
:1041A0000522204602F0CCFB2A680321204602F0BB
:1041B000ADFAB0BD64970102B0B5094D2860022484
:1041C000002120460A4602F029FB01210522204653
:1041D00002F0B6FB2A680321204602F097FAB0BD30
:1041E000989501025C21AA480022425282847A21D9
:1041F00041840284C2830283C282028211494160E7
:104200008260C2603D21490441834182090C81835F
:10421000818270475C219E480022425282847A212A
:1042200041840284C2830283C282028205494160C2
:104230008260C2603D21490441834182090C81832F
:10424000818270474C37373770B592484C210160F6
:1042500001252C02601C00F075F9322000F0B4FA40
:1042600000F05EF9284600F065F9284600F074F881
:1042700000F050F90C4800F065F900263046314650
:1042800000F05AFA2846314600F056FA204600F06F
:1042900059F9022000F056F94834204605F032FC66
:1042A00005F088FC70BDC0460102000010B5044650
:1042B000072106F011FC07480460032406A22046EB
:1042C000214606F0A7FD0AA20F4B2046214606F024
:1042D000A1FD10BDB0BB010248656C6C6F20667219
:1042E0006F6D204D4B53454D49210D0A00000000D4
:1042F0004275696C6420696E666F726D6174696F76
:104300006E2025730D0A0000C8E3000010B50520DB
:104310000424214602F0ECFA0620214602F0E8FAD5
:104320000E20214602F0E4FA0D20214602F0E0FAC8
:1043300000240121204602F0DBFA02212046224619
:1043400002F0FEFA10BD000002480168012291430C
:10435000016070475800004002490A6802408242EA
:10436000FBD1704704600040B0B5494D2868810713
:10437000484C0ED528797F21084022688A431018BE
:10438000206023680B4002200321434A06F042FDCF
:10439000286880040ED55E20285C7F210840626872
:1043A0008A431018606063680B40022003213B4A77
:1043B00006F030FD172000F043F939480168022269
:1043C0000A4301218A430260364837490160374871
:1043D0000021C17181791F2529408171817A427C38
:1043E000837C1B029A18C37C1B04D218037D1B0616
:1043F000D2182F4B9A4218D1427B837B1B029A180A
:10440000C37B1B04D218037C1B06D218294B9A428B
:104410000BD1C27A037B491E122906D819028918CA
:10442000254A914201D1202101720178CA0602D1A8
:104430001022114301701C3C206820218843206019
:104440001E481F49016041680029FCD503F0D4FAD9
:104450000446022003211BA2234606F0DBFC0A20AF
:10446000C441032C05D8022003211DA206F0D2FC72
:10447000FEE71848C1680F229143C1600168164ADF
:104480000A40026019200001144948600D60B0BD67
:104490000497010248000040ACCD000096CD00001A
:1044A000040200400C060040AF6B100A6B00014094
:1044B0004D383650312E323607340000006000404F
:1044C000FE1C0080436869702049443A202530383A
:1044D000780D0A00C8600040FEFFC3FF0C040040D6
:1044E0004F6C642063686970206D6F64656C20692F
:1044F00073206E6F7420737570706F7274656420B2
:10450000627920746869732053444B2121210D0A7C
:104510000000000080B5172000F08AF8002080BD60
:1045200010B51724204600F08BF8204604F0FCFF5D
:10453000002010BD0121C9070143014801607047F7
:104540000060004010B5C1B2000AC2B202290CD00E
:10455000012913D0002930D1911E744802291BD2A1
:104560000121032A2AD0490429E070484168002A21
:104570001FD00246203A1143416010BD6B480168CC
:10458000D31E022B10D3012A27D0002A3FD10122AB
:1045900092079143016010BD002A16D101214907FD
:1045A00002688A43026010BD0123042A1DD05A0408
:1045B0001CE0012292079143416010BD0904184A92
:1045C0007F32C36A13405918C16216498A6992073B
:1045D000FCD501214907026804E005221207914336
:1045E0000246203A0A43026010BD1A04836A0C4C4A
:1045F0001C40A21882620B4A131F00241C600A4B45
:104600000A4C1C600D235B0214681C431460054AAD
:1046100093695B06FCD5052212071143016010BDAA
:1046200080FFFCFF1402004004010040FF0F000067
:10463000012181403D4802688A4302607047C046BC
:1046400001218140394802680A4302607047C04630
:1046500010B505280ED8C04678440079400087443C
:10466000020B1219292C31490A680868C0002BD5A1
:1046700030482AE0002010BD2C490A680868C000B4
:1046800029D52C4828E029490A680868C0002CD59B
:1046900028482BE025494C680120C0030A680B46D6
:1046A000203B1C4234D00C68E40032D5214C1A4225
:1046B00033D031E01D4800680AE01C490A680868E8
:1046C000C0001AD51B4819E0194820390A421FD1E9
:1046D0000120C00310BD16480B46203B1A4201D1F1
:1046E0000120C003496889001DE011480B46203BAA
:1046F0001A4212D10120C0030FE00D480B46203BA7
:104700001A4201D10120C00349680903890FC8403A
:1047100010BD074C1A4200D020464A689200920F02
:10472000D04049680901890FC84010BD20000040F1
:10473000006CDC020026B80304282CD8164AC046B8
:104740007844007940008744020A121A21000320AD
:104750000007136883438807800818181AE00320AD
:1047600080061368834388070009181812E00320A5
:104770008004136883438807000B18180AE0FF20A1
:104780000002136883430802181803E01068FF232F
:10479000984340181060704724000040B0B50022D4
:1047A00000290CD0074B047895B22D0A65406C00A7
:1047B0001C5B12026240491E401C0029F3D190B2DA
:1047C000B0BDC046B8C3000000280AD030B40725E9
:1047D0002C02CD256419604340091238001FFDD812
:1047E00030BC7047F0B583B01F4616460D460146F3
:1047F000E8680291FBF7A7FD04460F2E11D8082E9A
:1048000004D320462146FBF745FD09E0042E02D3E0
:104810008120C10501E0412001062046FBF793FD00
:1048200004460999089E2B20C043874205DB204699
:104830000F462146FBF72EFD0DE03F20C043874287
:104840000BDA4920C04387420CDBFF200F4681056D
:104850002046FBF778FD39460446688A08803460B4
:1048600003B0F0BD01915320C043874206DB2046D0
:104870002146FBF70FFD0446688A10E0A8690299FB
:10488000FBF7D8FE002801D1A88B00E0E88BFBF7EE
:104890001DFF01462046FBF756FD04460020019906
:1048A0000880346003B0F0BDF0B581B0054601204A
:1048B000072D66D80C46002963D04A4F3868016935
:1048C000C90736D105263046FFF7BAFE304604F058
:1048D0002BFE03CF0369012213430361002918D47F
:1048E00003200B4683438E481E588807C00EFF27BF
:1048F0008740BE4340278740374389481F501F20C9
:104900000840824087480260874802603548006856
:104910000FE08A07D20EFF2696400F230B40083B7C
:1049200003218B437D495F58B743402696403E4361
:104930005E5069014018012109024218E369DB0653
:104940009B0CA569ED00EDB2EB185360626852074D
:10495000520B23685B075B099A18A3685B079B0CE3
:10496000D218E3685B075B0DD21823695B01DBB2E9
:10497000D21863699B07DB0ED21880231343435080
:10498000002001B0F0BDC046F0B581B0002A23D0B0
:1049900005460835134C2668F668EE40F50702D048
:1049A000022001B0F0BD069D8600A619B560400149
:1049B00024682018009301231D02461977680724F4
:1049C000A7437760F16032610099B16041591943A2
:1049D0004151002001B0F0BD03A00AA174220DA333
:1049E00005F0E8F960920102696E636C7564652FE9
:1049F000647269766572732F6D6B5F646D612E638F
:104A000000000000646D615F7472616E73666572B0
:104A100000000000496E76616C6964207472616EFA
:104A200073666572206473742061646472000000B0
:104A300000015849085840687047C046F0B581B039
:104A400005460120012D4CD80C46002949D0002DE7
:104A500003D0012D04D10F2000E00E20FFF7F0FD60
:104A6000A668012E04D0002E4FD1E08900284CD139
:104A70002901294843580020D860F507AD0F276861
:104A80006668B607360F76192569EA07920EB618DA
:104A9000022F04D0012F03D10122164300E040363B
:104AA0001D4F9E60E2681A6079188D606269CA6065
:104AB0004968002917D403220B469343184A9C588F
:104AC0008D07ED0EFF26AE40B4438026AE40264350
:104AD0009E501F220A4001219140124A1160124A41
:104AE000116001B0F0BD8A07D20EFF2494400F235D
:104AF0000B40083B03218B4308495D58A5438024A4
:104B000094402C435C5001B0F0BD08A00FA1492295
:104B100012A305F04FF9C046A89201021CED00E077
:104B200000E400E080E200E000E100E0696E636C18
:104B30007564652F647269766572732F6D6B5F643F
:104B400075616C5F74696D65722E63006475616C6C
:104B50005F74696D65725F6F70656E00636F6E661E
:104B6000696720697320696E76616C696400000072
:104B70000001084A10580160816880220A4382605F
:104B80007047C0460001034908588168802291435C
:104B900081607047A8920102F0B58DB0019315466F
:104BA0000E460A901298002408900480149F3C80BE
:104BB000139809900460159804900480FF208105E3
:104BC0003046FBF7C0FB0290304603963146FBF7B8
:104BD00061FB2B463D460690274607950B9311E057
:104BE0001180188880002858099908600120079DC5
:104BF00028800520049908807F1CBCB21888844254
:104C000000D9A0E028880028F6D1A0000A9D2E58DF
:104C100030460699FBF700FD002817D0304603996F
:104C2000FBF7FAFC00280B9B079DE5D1089A17803B
:104C3000099D2E601888011B012934D11080198824
:104C400089000A9A51582960059035E0089A178022
:104C5000099806600B9B1988081B0128C0D00C9688
:104C6000019825187E1CB0B28542BFD389B2B2B27A
:104C70008A420ED880000A990C5820460C99FBF7FE
:104C8000BDFC0B9B002804D109980460089806809D
:104C90000C94761CB0B28542A8D3198889B2B2B2FE
:104CA0008A42E7D9F5E70C96019962187D1CA9B2F2
:104CB00016468A4205972CD2059884B2A5000A9E12
:104CC0007259002C104609D0A819001F016810461F
:104CD0000C92FBF7DFFA0C9A062C07D80446A819A9
:104CE00041681046FBF7D6FA0C902046079D0299C2
:104CF000FBF7A0FC00280B9B07D10C980299FBF74F
:104D00008BFC0B9B002800D076E701202880032035
:104D100070E780B2AAB282420FD888000A990C5874
:104D200020460C99FBF76AFC0B9B002805D10998DB
:104D300004600898058005950C946D1CA9B28E42FC
:104D4000BAD31888E5E70DB0F0BD00000A490A683B
:104D50000A4802400A60FD214900094A1268515C74
:104D6000002908D007490A6C02400A6401200006A5
:104D70000A6882430A60704700040040FFFFFF7F1B
:104D8000BC9301022000004000207047F0B585B0C0
:104D90000E4607467C25454361484419E069216A6F
:104DA000FBF798F90396B04200D8B2E004970121CE
:104DB000EFF310860E4002D1EFF3108272B6274651
:104DC000103723690020062B0DD80A469A40D306D7
:104DD0005B0F07D161231A4200D194E00846002EF0
:104DE00003D003E00220002E00D162B6002801D0DB
:104DF00005B0F0BD02972746203749484059102199
:104E0000C1612646143604F0CFFE05462068C0690D
:104E1000C00605D504F0C8FE401B31888842F5D98C
:104E20000621049800F0C2FE386803994143A06946
:104E30000918206881601721615625461735002919
:104E400009D5C16920220A43C2610121E1668905B1
:104E500002680A4302600521049F384600F0A6FE5E
:104E6000287841B200200029C2D401903B48006854
:104E70007D25E900FBF72EF96D01454304F094FE12
:104E800003900221384600F091FE04F08DFE0746A3
:104E90002068C169890606D404F086FEC01B3188EB
:104EA0008842F5D92068007DC007049F08D064209F
:104EB000FFF78AFC04F078FE0399401AA842E0D973
:104EC00004F072FE05462068C069C00705D004F0F2
:104ED0006BFE401B31888842F5D904F065FE05461B
:104EE000029F2068C169890706D504F05DFE401B5A
:104EF00031888842F5D92068012139604F498161A4
:104F0000019805B0F0BD03213960002E00D16CE797
:104F10006CE7044804A1094A09A304F04BFFC0460A
:104F2000D0920102DCCD0000666C6173685F626C38
:104F30006F636B5F65726173650000005D02000066
:104F4000626C6F636B20696478206973206F76658B
:104F5000722072616E67650D0A0000006CB3010279
:104F6000F0B583B002907C2141438E4A5418E56E1F
:104F7000EAB2511E02291DD229040126090E5AD077
:104F800001960092022100F011FE2746143704F02A
:104F90000BFE06462068C169890606D404F004FEAB
:104FA000801B39888842F5D92068007DC007019EA2
:104FB00041D105E0032A32D100922804000E30D0FE
:104FC00020466C302D0C00210191016027461437DA
:104FD00004F0EAFD06462068C069C00705D004F069
:104FE000E3FD801B39888842F5D904F0DDFD0646D3
:104FF0002068C169890706D504F0D6FD801B398871
:105000008842F5D920680D498161E9B20120002963
:1050100009D003290099019E07D0062005E000264B
:1050200009E0012607E00099019E2061226F002A15
:1050300001D002A89047304603B0F0BD000093EBCA
:1050400070B5002801D0012070BD7825CD4E705D6F
:1050500000280ED000240921204600F0A7FD0F20D3
:10506000FFF7B2FB1520FFF7E3FA745534612046D1
:1050700070BD042070BDC046F0B581B00C4600780C
:10508000484EF16881422CD1032C54D1706EB16E20
:10509000884261D900240621204600F087FD30684F
:1050A000F16D81602046214600F080FD3546603577
:1050B0002CCDF0683168B48C414F00975B1BA34244
:1050C00000D81C46A3081431FFF75EFCB06E00192F
:1050D000B066306E00193066F06D0019F06501B0F1
:1050E000F0BDB168814255D1032C45D1F08CF16DF2
:1050F0000918F165316E09183166B16E0818B0668D
:10510000716E814238D900240621204600F04EFD00
:105110003068F16D81600121204600F047FD316E5D
:10512000B068F38C3268264C009414329B08FFF769
:105130002BFC01B0F0BD30681021C16104F034FDDA
:1051400005463068C069C00616D504F02DFD401B29
:10515000B18A8842F5D90FE030681021C16104F0AE
:1051600023FD05463068C069C00605D504F01CFD66
:10517000401BB18A8842F5D90120C1073268136803
:105180008B431360F16E22040A4300021043F06661
:1051900001B0F0BD4D200201034804A1844B04F08E
:1051A00009FEC046D0920102DCCD0000666C61733E
:1051B000685F646D615F63616C6C6261636B00006A
:1051C00079500000F0B581B000786E4DAA68824237
:1051D00000D0D0E001263002032942D16A6DAA66D0
:1051E000AB6DAC6AA418EB652C66AB6C5B1CAB6456
:1051F0006B6E934235D95E30FFF7E6FA686CA96CA6
:1052000002293AD3814238D1E88C696D0818686563
:105210000020062100F0CAFC2868E96D81602F6D2E
:1052200004F0C2FC04462868C069C00705D004F039
:10523000BBFC001BA98A8842F5D904F0B5FC0446E2
:105240002A68D069800706D504F0AEFC001BA98A45
:105250008842F5D92A687420285C012841D0F104DD
:1052600040E0F2072B681C6894431C60EA6E090456
:1052700011430143E96601B0F0BD0229FBD381422D
:10528000F9D2E88C696D09186965A96D0818A865D7
:105290000020062100F08AFC2868E96D8160EF8C0F
:1052A00004F082FC04462868C069C00705D004F0F9
:1052B0007BFC001BA98A8842F5D904F075FC0446E2
:1052C0002A68D069800706D504F06EFC001BA98A05
:1052D0008842F5D92A687420285C012822D0F1047C
:1052E00021E03105334B3B405918012802D01920E9
:1052F000400601E00720C00608182F4940185060FA
:10530000002F0DD004F050FC04462A68D0698007B5
:1053100006D404F049FC001BA98A8842F5D92A6802
:105320002B6D1FE03105234B3B40C918012802D0EB
:105330001920400601E00720C00608181E49401841
:105340005060002F0DD004F02FFC04462A68D0696D
:10535000800706D404F028FC001BA98A8842F5D9EE
:105360002A68EB8C296EA868144C00941432FFF75D
:105370000BFB01B0F0BD044804A10C4A0C4B04F037
:1053800019FDC046D0920102DCCD0000666C61734D
:10539000685F646D615F77726974655F6E6279746E
:1053A00065735F63616C6C6261636B007204000023
:1053B000C3CD0000FF3F000000808000C551000009
:1053C000F0B587B004460126880E1AD01546002A8B
:1053D00017D00F468120C004401B884211D37C2087
:1053E0006043C74908180590818C38460691FAF742
:1053F00071FE002905D128460699FAF76BFE0029AF
:1054000002D0304607B0F0BD059880693E1A30469C
:105410000699FAF75FFE0746039670190190069EFB
:105420003146FAF757FE0546C01B04900598006AFE
:1054300002903146FAF74EFE049981420FD20026BF
:10544000BD42DED92046394600F0C4FA2046FFF7B7
:1054500087FD0028FAD17F1CAF42F3D3D1E700903B
:105460000398029D2946FAF735FE06462846704302
:105470000399081A019800D0761C2946009D7543AF
:10548000FAF728FE0590029941430198401A0390CB
:105490000699FAF71FFE0490AF420BD22046394618
:1054A00000F098FA2046FFF75BFD0028FAD17F1C38
:1054B000AF42F3D305988642069D009F0CD220464A
:1054C0003146FFF763FC2046FFF74AFD0028FAD17A
:1054D000761C05988642F2D30398A84201D2002692
:1054E0008FE7059847430025E919204600F072FA36
:1054F0002046FFF735FD0028FAD16D1C00260498E0
:105500008542F1D37DE7C046F0B581B0002801D0D7
:105510000124F2E078227A4FB85C002801D0002400
:10552000EBE00092002905D0384614300CC90CC0BD
:105530001CC91CC00020F86615242046FFF780F81F
:10554000204603F0F1FF38681021C16104F02CFB04
:1055500004463868C169C90607D504F025FB001B5D
:10556000B98A8842F5D9386800E0B98ABA7D12074D
:10557000120B5218F97DCB07DB08D2188B07DB0F13
:105580005B05D218CB06DB0FDB05D2184B07DB0F10
:10559000DB06D2188B06DB0F5B07D2180907C90F91
:1055A00089071143016000240A21204600F0FEFA19
:1055B0003220FFF709F90821204600F0F7FA04F03D
:1055C000F3FA05463868C169890606D404F0ECFA96
:1055D000401BB98A8842F5D93868017D0A46C23A2B
:1055E000534253417426BB550904027D12025118DF
:1055F000007D0B180220032542A2294605F00AFC73
:10560000B85D012803D1F97D012008401BE000208E
:10561000032100F0CBFA04F0C7FA06463868C169E6
:10562000890606D404F0C0FA801BB98A8842F5D9ED
:105630003868007D420801201040F97D0A43D207F6
:1056400001D0014004D001214140002000F0F6FFCC
:105650007720385C012803D102200021FFF76CF885
:1056600004F0A2FA06463868C069C00705D004F005
:105670009BFA801BB98A8842F5D904F095FA064650
:105680003868C169890706D504F08EFA801BB98A8B
:105690008842F5D93868CE498161172038560028EC
:1056A00027D57868002815D40146A9431A4A8B5893
:1056B0008507ED0EFF26AE40B3438026AE401E4365
:1056C0008E501F2101400120884014490860144970
:1056D00008600EE08107C90EFF228A400F230340B5
:1056E000083BAB430B481D58954380228A402A4310
:1056F0001A500120009978543861204601B0F0BD5D
:10570000D09201026A656465635F69642025780D43
:105710000A0000001CED00E000E400E080E200E090
:1057200000E100E0F0B593B07C270A90474393482E
:10573000C619980704D0F07D4024044000D016E13B
:105740000125880E00D1EBE0002B00D1E8E081209C
:10575000C004C01A884200D2E2E009920122EFF3AD
:105760001084144002D1EFF3108072B6304610302E
:1057700005903069002506280891069310D80794F3
:1057800014468440E106490F04D161210C4203D044
:10579000154604E0022502E00221059B1960079CE2
:1057A000002C00D162B6002D00D0B9E03446173489
:1057B0007248C05910210491C1613746143704F072
:1057C000F3F905463068C069C00605D504F0ECF968
:1057D000401B39888842F5D92078400663D4029767
:1057E000B78C069C20463946FAF774FC0790394678
:1057F0004143601A039035462435A74200D892E011
:10580000039800281CD006210A9C204600F0CEF9FF
:10581000288807994843089940183168886000270C
:105820002046039C394600F0C1F9079B099A288855
:105830005843C0193168097D11547F1CA742F6D323
:1058400030680499C16104F0AFF90446029D3068E4
:10585000C069C00605D504F0A7F9001B2988884255
:10586000F5D904F0A1F904463068C069C00705D035
:1058700004F09AF9001B29888842F5D904F094F9BC
:1058800004463068C169890706D504F08DF9001B0C
:1058900029888842F5D930680121059A1160C249EA
:1058A000816100253CE003200025089FF7650999E8
:1058B000316606997166B566F0660120C0073168E9
:1058C0000A6802430A6006210A9C204600F06EF92D
:1058D000306887602046294600F068F93A4F0BAAE5
:1058E0000A921BCF1BC21BCF1BC2B48CF0680A9953
:1058F000FEF7DAFFF0683168344A0092069A944263
:1059000000D31446A3081431099AFFF73DF8B06E8E
:105910000019B066306E00193066F06D0019F06540
:10592000284613B0F0BD002404E0641C07988442AC
:1059300000D365E706210A9800F038F9288860430B
:10594000089940183168886000270A98394600F0A5
:105950002DF928880028099AE7D06043101831688B
:10596000097DC1557F1C28888742F6D3DDE70448AE
:1059700004A1074A07A304F01DFAC046D092010211
:10598000DCCD0000666C6173685F72656164000065
:10599000C603000054686520444D4120726561646F
:1059A000206C656E6774682073686F756C64206224
:1059B0006520746865206D756C7469706C65206F06
:1059C0006620340D0A00000038C60000795000003F
:1059D000000093EBF0B585B00E4607467C254543A5
:1059E00061484419E069A18CFAF774FB0396B04250
:1059F00000D8B3E004970121EFF310860E4002D1E6
:105A0000EFF3108272B62746103723690020062B69
:105A10000DD80A469A40D3065B0F07D161231A427C
:105A200000D195E00846002E03D003E00220002EAE
:105A300000D162B6002801D005B0F0BD029727461C
:105A40002437494840591021C1612646143604F0D4
:105A5000ABF805462068C069C00605D504F0A4F877
:105A6000401B31888842F5D90621049800F09EF841
:105A7000388803994143A06909182068816017217B
:105A8000615625461735002909D5C16920220A43E8
:105A9000C2610121E166890502680A4302600421AE
:105AA000049F384600F082F8287841B2002000298F
:105AB000C2D401903B4800687D21C900FAF70AFB77
:105AC000304D2D35454304F06FF8039002213846E0
:105AD00000F06CF804F068F807462068C169890690
:105AE00006D404F061F8C01B31888842F5D92068DB
:105AF000007DC007049F08D06420FEF765FE04F017
:105B000053F80399401AA842E0D904F04DF805462D
:105B10002068C069C00705D004F046F8401B3188F2
:105B20008842F5D904F040F80546029F2068C16913
:105B3000890706D504F038F8401B31888842F5D92A
:105B400020680121396018498161019805B0F0BDD4
:105B500003213960002E00D16BE76BE7034804A1F5
:105B6000084A09A304F026F9D0920102DCCD000016
:105B7000666C6173685F736563746F725F65726191
:105B8000736500002B020000736563746F722069F7
:105B90006478206973206F7665722072616E676524
:105BA0000D0A00006CB30102000093EBF0B585B064
:105BB000049104467C20604339490F183D46143552
:105BC00003F0F2FF06463868C069C00705D003F04D
:105BD000EBFF801B29888842F5D903F0E5FF0646D4
:105BE0003868C069800705D503F0DEFF801B29886F
:105BF0008842F5D91421049B5943DC206043294A8B
:105C00001018039002914018018A8268C47C74269F
:105C1000BE5D012E0FD10191012B029900D102220C
:105C2000012B00D138247526BE5D012E06D0019EC1
:105C3000072B06D106E00E46029903E00326072B48
:105C400000D0019E184B334024069207D20A121945
:105C5000D218039B5958C907490C52184168CB0701
:105C60001B0CD218837C5B075B0BD218C068400703
:105C7000000A10183A685060002E0ED001290CD18D
:105C800003F092FF04463868C069800705D403F02A
:105C90008BFF001B29888842F5D905B0F0BDC046AE
:105CA000D092010280C70000FF3F0000F0B59BB01A
:105CB0000D460127890E01D100F0B0FC002B01D167
:105CC00000F0ACFC0D928121C9041193C91AA942BC
:105CD00001D200F0A3FC0121EFF310840C4002D1AB
:105CE000EFF3108272B67C224243E04B10929E1872
:105CF00032461032039233690027062B0ED80A462B
:105D00009A40D3065B0F08D161231A4201D100F0FB
:105D100050FC0F46002C03D003E00227002C00D1DA
:105D200062B6002F01D000F079FC1290B565002119
:105D30000F9171651198401E0E904019B164B169C0
:105D40000B916C1A0D99B162F56230637463F18C3A
:105D50000C912046FAF7BEF90746B0630E9820185A
:105D60000C9C2146FAF7B6F93B46C11B4A1C374644
:105D70003C3707C7119A0F9F0029114608D060438E
:105D800051190B9A891A0F1A6343501B0019C11835
:105D9000304648300B90304644300A903046403010
:105DA0000990304626300290304658300F903046E9
:105DB00054300E90F16437651098AC4908581021A2
:105DC000C1613446143430465030019030464C3076
:105DD0000C9003F0E9FE05463068C069C00605D5A1
:105DE00003F0E2FE401B21888842F5D9F07D400691
:105DF00000D55BE301200B9908600A990968002926
:105E000000D1B4E3324674320892C204059202050E
:105E100007921922520604920722D206069212E035
:105E20000C9800680F9A1168091811600E9A116891
:105E3000081810600B990868401C08600A990968E6
:105E4000884200D993E3099A1268012A00D186E0BA
:105E5000002A00D012E10C9807680E980068109094
:105E60000F980568062112981191FFF79FFE306880
:105E700085600D981099451803F096FE10903068D3
:105E8000C069C00706D003F08FFE1099401A218820
:105E90008842F4D903F088FE10903068C169890700
:105EA00007D503F081FE1099401A21888842F4D961
:105EB000306808990A78012A069900D0049910914F
:105EC000012A079A00D0059A3B4669490B401343C3
:105ED00010990B4367490B434360002F13D003F025
:105EE00063FE10903068C069800706D403F05CFE42
:105EF0001099401A21888842F4D9306829780175B0
:105F00006D1C7F1EFAD15C4800687D21C900FAF73C
:105F1000E1F811994143119103F046FE0546022133
:105F20001298FFF743FE03F03FFE07463068C16951
:105F3000890606D403F038FEC01B21888842F5D9B3
:105F40003068007DC00700D174E76420FEF73CFC98
:105F500003F02AFE401B11998842E0D96AE7012824
:105F600000D012E10C9807680E98006810900F9806
:105F70000568062112981191FFF718FE30688560B8
:105F80000D981099451803F00FFE10903068C06905
:105F9000C00706D003F008FE1099401A21888842F5
:105FA000F4D903F001FE10903068C169890707D564
:105FB00003F0FAFD1099401A21888842F4D930681C
:105FC00008990A78012A069900D004991091012AAB
:105FD000079A00D0059A3B4625490B401343109978
:105FE0000B4324490B434360002F13D003F0DCFD27
:105FF00010903068C069800706D403F0D5FD109971
:10600000401A21888842F4D93068297801756D1CBE
:106010007F1EFAD1184800687D21C900FAF75AF8A6
:1060200011994143119103F0BFFD054602211298D9
:10603000FFF7BCFD03F0B8FD07463068C16989066B
:1060400006D403F0B1FDC01B21888842F5D9306821
:10605000007DC00700D1E3E66420FEF7B5FB03F046
:10606000A3FD401B11998842E0D9D9E6D0920102E4
:10607000FF3F0000008080006CB3010201280C9AF1
:1060800000D009E117680E98006810900F98056815
:10609000062112981191FFF789FD306885600D98EF
:1060A0001099451803F080FD10903068C069C00752
:1060B00006D003F079FD1099401A21888842F4D95E
:1060C00003F072FD10903068C169890707D503F0AD
:1060D0006BFD1099401A21888842F4D930680899DC
:1060E0000A78012A069900D004991091012A079A8A
:1060F00000D0059A3B46EA490B40134310990B43E5
:10610000E8490B434360002F13D003F04DFD10907E
:106110003068C069800706D403F046FD1099401A24
:1061200021888842F4D93068297801756D1C7F1E5A
:10613000FAD1DD4800687D21C900F9F7CBFF11993C
:106140004143119103F030FD054602211298FFF7FB
:106150002DFD03F029FD07463068C169890606D484
:1061600003F022FDC01B21888842F5D93068007DEC
:10617000C00700D154E66420FEF726FB03F014FDAF
:10618000401B11998842E0D94AE6884200D051E686
:10619000019807680E98006810900F98056806210E
:1061A00012981191FFF702FD306885600D981099E3
:1061B000451803F0F9FC10903068C069C00706D09C
:1061C00003F0F2FC1099401A21888842F4D903F0B8
:1061D000EBFC10903068C169890707D503F0E4FC37
:1061E0001099401A21888842F4D9306808990A78B1
:1061F000012A069900D004991091012A079A00D02B
:10620000059A3B46A6490B40134310990B43A549F9
:106210000B434360002F13D003F0C6FC109030688E
:10622000C069800706D403F0BFFC1099401A21888A
:106230008842F4D93068297801756D1C7F1EFAD127
:10624000FC4800687D21C900F9F744FF11994143DA
:10625000119103F0A9FC054602211298FFF7A6FC54
:1062600003F0A2FC07463068C169890606D403F032
:106270009BFCC01B21888842F5D93068007DC0078F
:1062800000D1D7E56420FEF79FFA03F08DFC401B98
:1062900011998842E0D9CDE50E9A12680D9B9F189E
:1062A0000F9A1268884210927CD1019805680621E5
:1062B00012981191FFF77AFC30681099816003F011
:1062C00073FC10903068C069C00706D003F06CFC06
:1062D0001099401A21888842F4D903F065FC109087
:1062E0003068C169890707D503F05EFC1099401A30
:1062F00021888842F4D9306808990A78012A0699D9
:1063000000D004991091012A079A00D0059A2B46D3
:10631000C5490B40134310990B43C4490B434360D9
:10632000002D13D003F040FC10903068C069800746
:1063300006D403F039FC1099401A21888842F4D918
:106340003068397801757F1C6D1EFAD1EA48006803
:106350007D21C900F9F7BEFE11994143119103F067
:1063600023FC054602211298FFF720FC03F01CFCD9
:1063700007463068C169890606D403F015FCC01BC6
:1063800021888842F5D93068007DC00700D151E5E9
:106390006420FEF719FA03F007FC401B11998842AC
:1063A000E0D947E502980588062112981191FFF778
:1063B000FDFB30681099816003F0F6FB10903068A7
:1063C000C069C00706D003F0EFFB1099401A21887E
:1063D0008842F4D903F0E8FB10903068C16989075E
:1063E00007D503F0E1FB1099401A21888842F4D9BF
:1063F000306808990A78012A069900D0049910910A
:10640000012A079A00D0059A2B4687490B4013436F
:1064100010990B4385490B434360002D13D003F0C3
:10642000C3FB10903068C069800706D403F0BCFB42
:106430001099401A21888842F4D93068397801755A
:106440007F1C6D1EFAD1AC4800687D21C900F9F7A8
:1064500041FE11994143119103F0A6FB054602212B
:106460001298FFF7A3FB03F09FFB07463068C16952
:10647000890606D403F098FBC01B21888842F5D911
:106480003068007DC00708D06420FEF79DF903F056
:106490008BFB401B11998842E1D902980088C1E426
:1064A000FF3F0000008080006CB301025D4913AA29
:1064B0001092A9C9A9C2A9C9A9C201200D90C007FB
:1064C00031680A6802430A60B0681099FEF7ECF977
:1064D000022000270F9B1968B26AF1653266119994
:1064E0007166B766F0660C9800680E9A1168091814
:1064F00011600B9D29684A1C2A601A6810181860E0
:10650000002900D08AE030466030119035465C3575
:1065100030460830109006211298FFF747FB30688C
:10652000296881600C980068129003F03DFB0546D5
:106530003068C069C00705D003F036FB401B2188D6
:106540008842F5D903F030FB05463268D0698007F0
:1065500006D503F029FB401B21888842F5D9326813
:106560007420305C01282DD00D99C9042CE003F073
:106570001BFB05463068C069C00705D003F014FB5B
:10658000401B21888842F5D903F00EFB0546306890
:10659000C169890706D503F007FB401B21888842A3
:1065A000F5D930680121039A1160234981610027E0
:1065B00034E00421039A1160002C01D1FFF7B0FBF5
:1065C000FFF7AFFB0D990905129D174B2B4059188A
:1065D000012802D01920400601E00720C006081853
:1065E000124940185060002D0DD003F0DDFA054629
:1065F0003268D069800706D403F0D6FA401B2188A0
:106600008842F5D932680C9803681198016810988F
:106610000068074C00941432FEF7B6F938461BB0F8
:10662000F0BDC046F8C50000FF3F000000808000BC
:10663000C55100006CB30102000093EBF0B583B0CC
:106640000C4605460621FFF7B1FA07212846FFF759
:10665000ADFA7C200295684326490D187420285C09
:10666000012811D1601E8441A10128680175002113
:1066700001757521695C01290ED114307621695CA0
:106680004A424A41510006E0286800210175611E16
:106690008C41610014300170174800687D21C900E9
:1066A000F9F718FD282444432F46143703F07CFAE9
:1066B000019002210298FFF779FA03F075FA064675
:1066C0002868C169890606D403F06EFA801B3988F0
:1066D0008842F5D92868007DC00708D06420FEF7FD
:1066E00073F803F061FA0199401AA042E1D903B0AE
:1066F000F0BDC046D09201026CB301023920C00047
:10670000014909680858704760920102F0B50329F1
:1067100020D8C0467944097949008F4401080F15F3
:10672000012181404E4B1B685963D96212E001215F
:1067300081404B4B1B681963D9620BE001218140FA
:10674000474B1B68596304E001218140444B1B689F
:106750001963996283004249CB18DA608A68002A7B
:1067600029D14A68002A16D4032314469C43174BA8
:10677000E5589607F60EFF27B740BD438027B74080
:106780002F43E7501F23134001229A40104B1A60F9
:10679000104B1A600FE09307DB0EFF259D400F247E
:1067A0001440083C03229443074AA658AE43802570
:1067B0009D403543A55001228240086802628868E6
:1067C00010438860F0BDC0461CED00E000E400E02E
:1067D00080E200E000E100E010B501242046FDF772
:1067E0002FFF204602F0A0FE002010BD01218140B5
:1067F0001B48006842688A4342607047184909682C
:106800000968C140012008407047C046012181400D
:106810001348006842680A4342607047012907D064
:1068200000290ED1012181400E4802680A430DE083
:10683000012181400A4800684368002A0BD00B43BD
:106840000AE001218140074802688A430260044847
:106850000068416170478B43436001617047C046E7
:10686000509301020801004080B5114A1170114A8D
:1068700010708001C90101430F48007840010843AE
:106880000E490978090101430D480078C00008430A
:106890000C490978890001430B48007840000843FF
:1068A0000A4909780143C8B2FAF702FD80BDC04623
:1068B000B2950102F5A30102A5930102B4BB010246
:1068C000F6A30102B39501026899010269990102D8
:1068D000012282400548002903D00168114301606C
:1068E00070470168914301607047C0460001004055
:1068F000124A072809D880000F238340814019409D
:10690000106898430843106070470F280AD8800029
:1069100020380F2383408140194050689843084332
:1069200050607047800040380F23834081401940F9
:1069300090689843084390607047C0463400004018
:10694000F0B54307DC0E0726A640C3089D000E4B9A
:10695000EF187D68B5433E1D002908D0356001223F
:10696000824001290CD1186810431860F0BD012144
:106970008140186888431860A24015433560F0BD17
:10698000186890431860F0BD0C01004010B582B04B
:1069900014460A46014604980093019008202346B5
:1069A00000F092F802B010BDB0B584B014460A46AB
:1069B000014608980225009501930290072023467E
:1069C00000F052F904B0B0BD70B500285BD0314979
:1069D0000A783149002A03D14A68012313434B60E6
:1069E000428803881B049A180B46183B1A60828859
:1069F00083891B049B180C460C3C23600B46083B08
:106A000084681C60446903232340057CAD00EB18B7
:106A10008569AD072D0D5B19457C2D035B19C56993
:106A2000AE07B60A9B19867CB6059B190E1F33600C
:106A3000036A122B04D107240C60541EA2410AE001
:106A4000032C05D1012D03D807220A60012202E0A0
:106A500006220A600122114C002525700F246401D2
:106A60002034C57C6D0225401B069B0BD218C379D0
:106A70001B07DB0ED21880790007C00D10184019D3
:106A80001439086070BD064806A1862209A303F0E8
:106A900091F9C04610A401021810005012A401027E
:106AA0000FD100006C73705F656E67696E655F7211
:106AB000756E0000506172616D6574657220697356
:106AC000206E756C6C000000F0B58BB0109E340425
:106AD0003ED00D46D64C2140012701977F06B94292
:106AE0003CD111462140B9423FD11C40BC4243D168
:106AF000119902AC0027E781E78066802780278212
:106B0000A774E1749908A181A908A1800A90099746
:106B100008970797900880B204902046FFF754FF2B
:106B2000AA480078002801D00BB0F0BDAB4801683E
:106B3000C90708D10168C90705D10168C90702D191
:106B40000168C907F3D07F48019901700BB0F0BD0F
:106B5000B8480D49AF22C14B03F02CF90095B54858
:106B60000949B022754B03F025F90092B148064956
:106B7000B122724B03F01EF90093AE480249B222D3
:106B80006E4B03F017F9C046E5D00000F0B58DB0AC
:106B90000392139E340446D00A46A54C2140012599
:106BA00002956F06B94244D103992140B94247D1B9
:106BB0001C40BC424CD11499129D04ACE17429498B
:106BC00021820027E781E780668027809908A181DC
:106BD0009108A1800B95012D01D16121CF43A774AC
:106BE0000C9002200A9009900398800880B20690C9
:106BF0002046FFF7E9FE75480078002801D00DB067
:106C0000F0BD76480168C90708D10168C90705D1F8
:106C10000168C90702D10168C907F3D04948029940
:106C200001700DB0F0BD83480D49FB228B4B03F082
:106C3000C1F800927F480A49FC22404B03F0BAF8A1
:106C4000039800907B480649FD223C4B03F0B2F8C4
:106C5000009378480249FE22384B03F0ABF8C04657
:106C6000F2D000008E8E0000F0B58BB0119E34047F
:106C700047D00D466E4C2140012701977F06B9424F
:106C800045D111462140B94248D11C40BC424CD1AB
:106C90001299109F02ACE174294921820021E181FF
:106CA000E180668021809908A181A908A1800997C7
:106CB000012F01D0712100E06121C943A1740A9024
:106CC000032008900790900880B204902046FFF7B8
:106CD0007BFE3E480078002801D00BB0F0BD3F4855
:106CE0000168C90708D10168C90705D10168C9074A
:106CF00002D10168C907F3D01248019901700BB0A5
:106D0000F0BD4C480C49D522544B03F053F8009584
:106D100048480949D622094B03F04CF800924548EF
:106D20000549D722054B03F045F800934148024935
:106D3000D822024B03F03EF801D100002FD1000011
:106D40008686000012A4010210B582B014460A46DD
:106D5000014600200093019004202346FFF7B4FE73
:106D600002B010BD10B584B014460A46014600209A
:106D700000900193029004202346FFF707FF04B020
:106D800010BD000070B50D46064604242046FDF7F0
:106D900057FC204602F0C8FB0B4805600B48067004
:106DA000002E0ED00A48016880220A437F218A43C0
:106DB000026001200003074908600749086007488E
:106DC0000460002070BDC04614A4010210A401029A
:106DD0000CE400E080E200E000E100E01C10005064
:106DE000B0B582B0144602461148204001256D0618
:106DF000A8420DD1180413D0174801600020009359
:106E00000190062011462346FFF75EFE02B0B0BD9A
:106E10000094FF228C320748074908A302F0CAFFFA
:106E2000FF208C30421C034803490C4B02F0C2FF88
:106E30000300FCFF0FD10000D7D000004473742082
:106E40006164647265737320257820697320696EAC
:106E500076616C6964000000081000504DD100009C
:106E600080B582B00B4601460020009201900320BD
:106E70000A46FFF729FE02B080BD0000002801D0BD
:106E8000042100E00221C24A5172411E8841800162
:106E900003490A6840239A43101808607047C046A7
:106EA00050A00050F0B583B002912E49CD7A0E7BF0
:106EB000771987424FD908990191182545434126F2
:106EC000F604BF00BE19745B34490C4057033C19EB
:106ED0009B07D90C6418324B1B681B7A74537519C5
:106EE0006C880326B60326409B079B0C9B193F2406
:106EF00004401819029CA3061B0DC0186880012AC3
:106F0000184E13D8707B14224243307B50234343E6
:106F100024011B199A18F37AC0181C234343D01874
:106F200080081E4A104007430F432F800198686075
:106F300001F07EFEA860E8681A4908403030E86039
:106F4000286908402721715C4018286100F010FE74
:106F5000686103B0F0BDFF228832034803A108A393
:106F600002F028FF80A501029ED100006D61635FE1
:106F700063735F636F6E73747275637400000000F7
:106F8000435320696E646578206973206F7665725B
:106F90002072616E67650D0A00000000FF070000A7
:106FA000BC9301020000F0FFF0B581B000931446DD
:106FB0000D46074606263046FDF742FB304602F0F6
:106FC000B3FA26211D484754002101704170817198
:106FD000017181704171C170C17102224272C1623E
:106FE00001634163816304734273C572009A561C46
:106FF000134A168001724120C00401214903F9F7A8
:10700000ACF8502060432901081861198A008018E3
:1070100018224A438018B2B24A43801809494018DE
:107020000949884204D200F0B5F8002001B0F0BD53
:10703000064807A19A2209A302F0BCFE80A501021E
:107040007EA5010228000802012008029ED100004E
:107050006D61635F696E697400000000454D206FCB
:10706000766572666C6F770D0A000000A448C179DE
:10707000002901D001207047007A411E88417047E5
:10708000F0B583B002912A494B7B834248D9CB7A31
:107090000C7BE31818245C439B00E3184124E404B0
:1070A0001A19142401900546654300265651009292
:1070B0005519EE882E4F0B467A1C3240F54E368815
:1070C000497A711A2B4E0E40B618EE803740997BE4
:1070D000EF80AA88284F17404A424A419100791808
:1070E000264A8918A980264F0F402D1D0298012895
:1070F0000AD124490E400921C90271186980012171
:10710000C9037918298000E02F8001984443009832
:107110000019074A918C4182118C018203B0F0BDA5
:107120003520C200034804A109A302F043FEC04673
:1071300080A501029ED100006D61635F6C696E6B7A
:107140005F646573635F636F6E73747275637400FD
:107150004C696E6B206465736320696E646578208A
:107160006973206F7665722072616E67650D0A0023
:10717000FFFBFFFFFF03000003D0FFFFE80F00004D
:10718000EF1F0000FF830000BE4A50639163704709
:1071900080A50102F0B581B04348CC2101600321F4
:1071A0004160B8490A7BD304404C1B19CC7AA21821
:1071B000541E1C431823534392009A184B7B1425EA
:1071C0005D43521992012243012463061343436134
:1071D00000228262C262026342638263C2634265CA
:1071E0000267334B1A605A609A60324B1A601A6118
:1071F0009A61DC61304C1C62304C251D1D632546B4
:107200000C3D5D632546283D9D632D4EDE631C6469
:107210005C642C4D2F461C379F642746143FDF6467
:10722000103C1C65284C5C65284C9C650C369E67A0
:10723000274CA5634035E563DA651A665A669A6697
:10724000DA661A67234DDD6702258561224DC56127
:10725000C325AD03CD620A63D2435A601F4A136847
:10726000FF25AB4326254D5DAD072D0EEB181360B2
:107270001B4A102313601B4A1360272260238B5480
:1072800019498160C160016121607D2109010166A8
:1072900041661649C164164941641649016400F00B
:1072A00057FC01B0F0BDC04604A000500000F8FF3C
:1072B00094A0005034A10050FF185A003004004040
:1072C000041000401C20004054300040604000404A
:1072D000B8A1005014001400FF3F3FFF04E400E099
:1072E00080E200E000E100E0DC05DC053F02700226
:1072F0000133D007D007D0072921C64A5054704720
:1073000080A50102F0B58BB0079208910146C14FEC
:10731000B8780991FFF7B4FE78793A7B79790691CC
:10732000824200D89FE0FB7A9A18182353439200B8
:107330004124E10404915218D2187B7B14214B4361
:10734000D21850246043155801230A93DB022E46BD
:107350009E4316504E4B2B4005937D7B03914D432E
:107360003E7B7443F97A0B011B195B1971181C24BD
:10737000029461435918A84B1B88069C5C43091969
:10738000C904490D059BC91811501018079941608F
:1073900038787979089A00920322099BFFF782FDD9
:1073A000F87A397B09183878814263D983000993C8
:1073B000049AD45C0894F7212140D154D1184D7817
:1073C0008E7836027619CB781B04F31807900A984A
:1073D00086051E43330CCB70FB7A387BBC784D702E
:1073E0009F4D3540039E6643C018029B4343981946
:1073F00040029C4B03405C19200A8870200CC87026
:10740000F023089D2B401B1D3D7B0895FE7A099DAE
:107410005355C8700620079A50438019089A80185F
:1074200048701F22D20222400243100A88707879E5
:10743000401C7871387B7979814201D300217971C0
:107440003978491C3970F97A08183978884201D896
:107450000020387028200A993954387A401C387234
:10746000387A0BB0F0BDA7204200D2480649074B3E
:1074700002F0A0FCA72042007A32CE487349744B38
:1074800002F098FC80A50102BED1000067D1000087
:1074900000F0FFFF7EA501020320000605490A68EF
:1074A00082430A600A6802430A60034801210160BE
:1074B0007047C0461C0000401CA0005080B5012051
:1074C000FDF760FB80BD0000F0B587B0069306466F
:1074D000504C607A504B1B88181A0C9DA84200DC57
:1074E00089E00F460592012E06D156480021C1625F
:1074F0000169554A89180160A0783146FFF7C0FD3F
:10750000E078E178069A2B4600F0AEF82078E17832
:107510000097002206923346FFF7C4FCE07A217BF5
:107520000818217888426ED94120C204049188004D
:10753000815C0391F7250D40029285544549455CD5
:107540004549465C360276194449475C3F04F619C2
:107550000127BF0537433E0C4654E67A217BA378CA
:107560003C4A85543E4D3D4014275F4389191C23F6
:107570004B43D91949023B4B0B405D19290A364B45
:10758000C1542E0C35494654F02703990F400599F4
:10759000002900D13F1D217BE37A029A87542F4AAC
:1075A00086540622049E7243D2185118294A8154E7
:1075B0001F22D20215400D43290A274A8154E07840
:1075C000401CE070E07AE178814201D30699E170D5
:1075D0002178491C2170217B08182178884201D824
:1075E00006982070E079401CE071A07A401CA072DF
:1075F000E07907B0F0BD3920C2001632074808A173
:1076000009A302F0D7FB3920C20004480F49104BF0
:1076100002F0D0FB80A501027EA501029ED10000F0
:107620006D61635F747800004D4143205458206CB5
:10763000656E206973206F7665722072616E676572
:107640000D0A00000804004090D00300D4D10000CF
:1076500085D10000010008020200080203000802B0
:10766000FF07C0FF00F83F00F0B589B00893019212
:1076700004914F4DEF7A874200D891E0297B502644
:1076800032464A434124E3040693D218CC19A100A0
:1076900051181822059254430A19697B1423079341
:1076A0005943531802900001195804460390504A58
:1076B0000A40A97AC902511808988205D2088A1886
:1076C0001A514C4911402A7B00965643384CE57AB2
:1076D0002C0106982418A719354E5419A5007D19B8
:1076E000059844432819747B079D6C430519049F32
:1076F000D2194148048854432A19089CD204520DD7
:1077000051181D460398195000F03CFA0146707A52
:10771000001902043E460CD080B2C000002900D1FE
:10772000801E029FA5214900F8F7D4FC1F210140CB
:1077300001E00021029F38012818427983791B0259
:107740009A18C3791B04D2182C4B134043710904B7
:107750005918090CC171002C20D015483546064631
:10776000007B009B4343F17A0A01069F3A43D218FB
:1077700041188B00D218059B4B43D118727B079B95
:107780005343C91840191C4A12884243881801996A
:10779000884203D001992246F8F7C6FC09B0F0BD33
:1077A000FF225C32034804A109A302F003FBC04698
:1077B00080A501029ED100006D61635F74785F64F3
:1077C0006573635F636F6E7374727563740000003A
:1077D0005458204445534320696E6465782069738A
:1077E000206F7665722072616E67650D0A00000079
:1077F000FF0700E000F8FFFF7EA50102EFFFE000B9
:1078000082B0FCF721FDFCF781FD0020FCF74EFD66
:1078100001F00AFE01F002FE564801685648006871
:10782000890309D403210907084001210907884277
:1078300002D0FCF7D7FC06E0FCF754FAFCF7EAFCB0
:107840000020FDF7FDFBFCF78FFD0020019004F008
:10785000E3FC032049A2014603F0DCFAFEF7BCFF7B
:10786000F9F7B1FD01254B49284603F061FE284692
:107870002946FEF7F9FF48484849016000F0D6F86C
:10788000934CA08846490860A17A464A1170A189A4
:10789000454A1180A18A454A1180E28A444B1A80E8
:1078A000444B5A831983618B198198807D20C000D5
:1078B000E188F8F70FFC4049088040496422404BBA
:1078C000284603F009FF01F08DFB3E48608302F07B
:1078D00099F93D490860012802D13C48056007E05C
:1078E0003A48022101603A480188002900D1058008
:1078F000384A2846294602F08DF80095E80302F040
:10790000BDF83548FCF742FC3448FCF755FC2F4FD6
:107910002F4D334E334C01E0F9F78EFD38680028C7
:107920000CD002280FD00128F8D120780028F3D0FD
:107930000198207004F0ACFB01F06AFF04F086FBB4
:10794000F9F77AFDEAE73078002802D02888002885
:10795000E2D00198288004F09BFB02F053F91A4909
:10796000086004F073FB184800680028D4D0009821
:107970003860D1E7180000403000014055574220E0
:1079800073696D706C65206578616D706C650D0A4A
:10799000000000006094010288950102D5390000C2
:1079A000409D0102F7A30102449D0102B6BB010202
:1079B00038A60102A8A7010270B3010214A50102B2
:1079C000E1B80000221100000CA401022095010280
:1079D000809F0102B199000015C20000217A0000C9
:1079E00008A401024F93010280B5024B1B689B69FA
:1079F000984780BD00900102014800687047C0466A
:107A00000C00004081B080B581B0039303AB0093BC
:107A100002F08AFE01B080BC02BC01B00847000041
:107A20000148002101607047BCA50102F0B581B09A
:107A3000002630463146FDF767FD0125AC0223499B
:107A4000234F30463A462346FDF76CFE39882148DD
:107A5000814238D064217E5262217E5260217E5262
:107A600044217E5250217E52FD87BD87782179873F
:107A7000022139874321F986BE83FE811649B981E7
:107A80007E810A2139811549B9803880FE8314200E
:107A9000B8827D208000F880EFF3108072B6304607
:107AA0003146FDF731FD00280CD12A03002630466F
:107AB000064D2946FDF784FC054A304629462346F3
:107AC000FEF7F4F862B601B0F0BDC04600E0020473
:107AD000869F0102AA550000E1FF00003412000059
:107AE0000020704710B50024002809D0002905D0D7
:107AF00003464A0003481946F8F716FB204610BD16
:107B0000E04310BDC8920102014600200A2901DAB3
:107B1000C0437047014A11807047C0464C93010230
:107B20000020704780B50188064A11808178064A96
:107B30001170C178054A11700079FCF7B9FA00207C
:107B400080BDC046A6930102A8930102D0A5010200
:107B50000448054901601521090441600349816019
:107B60007047C0469C3000404100080034000700C8
:107B70000748006840697047FD20400004490968D3
:107B8000085C7047024800686221405C7047C0464C
:107B9000BC9301020A491A220A600A4948704878CF
:107BA000FF210902084A13688B43800380B2C01882
:107BB00010600648202101600548016000207047E0
:107BC00070200040AC93010204E400E080E200E099
:107BD00000E100E0F0B5A9B016460F460546C648DC
:107BE000002B024600D01A463921CC003D21C900A5
:107BF000511811918242189206D001204202BE49CA
:107C00001898F8F791FA189A6120111913910E211A
:107C1000119C0A91A170002F0D9501D00A2100E05E
:107C20000921592317938300E17078427841139911
:107C30000870307810901070F17AE174717851709A
:107C4000B7789770F178D17035791571747954716E
:107C5000B1799171F179D171317A1172717A517270
:107C6000B17A91727E1EF0B200210328169106D8D7
:107C700070B28000A1A210586A00805A169017981E
:107C800082001898C0181490F81E022804D3012E00
:107C9000084604D89D4800E09D48031918781290C2
:107CA000189DA81817902846303015902C46563449
:107CB0006D2080002950974A974B149E3362726260
:107CC000B362F2623176F182139B597009229A7085
:107CD000281841608160C1600161109880008F495F
:107CE0000858F8F75BFD012F10900F9104D0022F78
:107CF00005D17F217E2004E07C217B2001E05B21F7
:107D00005A20159DA984207003200C90A080012684
:107D100066701F200B90A8821820A8740A46083AA3
:107D2000179BDA76169B129AD2184A439100189A3A
:107D30009163B702791E8B420E9109D97848608011
:107D4000342068847748288277481399088339E07B
:107D50007F2B10DD802B18D031028B421BD071029B
:107D60008B4227D16E49618068846F4813990883DC
:107D7000CF20C00025E0202B17D0402B1AD1684817
:107D800060800420688469481BE0654860800620A4
:107D90006884674815E06248608010206884624803
:107DA00013990883C520C0000BE062486080022060
:107DB000688404E004206884812040006080FF2003
:107DC00002302882104600F0D7FE1298102806D004
:107DD000402808D108201499C876072000E0042024
:107DE0001799887002E017980C9981701898169A64
:107DF0008078C11E02290CD3022811D001280CD191
:107E00002672BA4200D900266672BA4213D8F448E4
:107E100012E00D200002119908800120800201E08B
:107E20000C9800022081BA4201D8EE4800E0FA2006
:107E3000179988600EE0FA201799886013980078E7
:107E40000028119901D0E8484880E848139A108327
:107E5000E7480880A88CF8F741FC0026E54B32463D
:107E6000F8F7ECFA02460B46E3493046F8F74EFBCA
:107E7000E24B3246F8F7E2FAF8F76CFC0746E0808E
:107E8000DF493046109A0F9BF8F740FBDD4B324636
:107E9000F8F7D4FAF8F75EFC78434042800B608133
:107EA00016990E98814208D90C20149FB872D648B2
:107EB000179988831220189A0EE0480A189A149F7E
:107EC00001D00D2003E0080A00D1DBE20A98B87265
:107ED000CE48179988831220F872D078052844D8A4
:107EE00078440079400087440227402C3339C84841
:107EF000B881C8482FE0C04660900102C8C50000A4
:107F0000C8C50000D8C50000D8C5000024C30000C3
:107F10002BC30000307500001027000078C300005C
:107F200005020000FF060000040800000A0400002B
:107F30003604000003020000B748F881B7483880D3
:107F400013E0B748F881B7483882B74838600CE08A
:107F5000B448B881B5481799C88306E0B448788218
:107F6000B448B8800B9800069064AE483881A748A2
:107F7000F880B14802882A84B0480078E874B04894
:107F80000078119F7875387D139000285ED0AD4938
:107F90000A681023DA413A600A794B79CF88678002
:107FA0001B029A186A840A7A4B7A8F7AC87A0D7BF8
:107FB00065701B029A183B04D21800061018179F10
:107FC000F860487B8A7BCB7B3B771202101860817C
:107FD000087C7877487C149A9072887CD072C87C30
:107FE000159B1874087D5874487D11909874C87D4D
:107FF0000A7E120212181A84887DD87418464B7EA5
:10800000C375887ECD7E2D022818B880087F4D7FED
:108010002D022818F880887FB877C87FF87720204D
:10802000085C149D28732120085C68732A20085C72
:108030002A314D782D0228188D782D044019C978E1
:108040000906401818998864119801E0EB7DA87C16
:108050007D498B700A8080001F38C882C8831398BE
:1080600000281FD022227748825C034622335B78A7
:108070001B029A180A842422825C034624335B780C
:108080001B029A18CA842622825C034626335B7838
:108090001B029A188A832822825C283040780002CA
:1080A000801888846948032569A2294602F0B2FE37
:1080B000189F387814907B78B8780F90FA78B87950
:1080C0001390F8791190387A1090787AB97A0890EC
:1080D000099100930F9801900292169803901298BC
:1080E0000490139805901198069010980790FAA2A2
:1080F000F8482946149B02F08DFE3D4664358021E8
:108100002846F8F72AF8B878C11E02290ED30128AC
:1081100000D18FE1022800D0ABE11691149078785D
:108120007F225043F7494018F74907E01691149011
:1081300078785B225043F1494018F14941182846AC
:10814000F7F7F2FF0D9D1898C6870E34324602E00D
:10815000641C0F2A0ADA21780029F9D0491C890702
:10816000C90F91400E43C687521CF1E716990229A8
:1081700007D31499491E012900D97DE14279D249DA
:1081800001E04279CF4989180C78002D00D177E1C0
:10819000C1790E91032900D94AE14279062A00D912
:1081A00079E14921890041181191E43010900E982D
:1081B000401E129019A800190F90002313921494D6
:1081C00003E01898290600D15AE1052A5AD8C0467A
:1081D0007A44127952009744455C728598ABC04648
:1081E00088130000E20400000C080000060A0000EA
:1081F000040F00000000104130C1BD41000070407C
:108200000000F0400000D041120C0000140B0000F0
:1082100012120000140E00000E160000130D0000D4
:10822000121600000E120000140B0E0A12080000B5
:10823000101600000E0B0000A6930102A893010285
:10824000D0A50102DCA5010214940102010800007E
:108250004361736520706172616D65746572733A14
:10826000200D0A001693DFB2002F04D019A80122B6
:108270003946F7F76BFF002C00D191E019A8C0191F
:10828000BB498AE0E8B2022867D00027022867D0FD
:108290006BE00E98022872D1E8B2022800D10346A2
:1082A0001693DFB2002F04D019A801223946F7F740
:1082B0004DFF002C74D019A8C019ACA16DE0E8B234
:1082C000022800D104231693DFB2002F04D019A88E
:1082D00001223946F7F73AFF002C61D019A8C019DE
:1082E0009FA15AE0E8B2022800D106231693DFB21C
:1082F000002F04D019A801223946F7F727FF002CD8
:108300004ED019A8C01992A147E0E8B2022800D1C6
:108310000C231693DFB2002F04D019A8012239468E
:10832000F7F714FF002C3BD019A8C019874934E097
:10833000E8B2811E4A424A419700022804D119A896
:1083400001223946F7F702FF002C16D019A8C019F0
:108350007CA12246F7F7E8FE0FE00627022804D1A9
:1083600019A801223946F7F7F1FE002C05D019A80B
:10837000C01980492246F7F7D7FE169710E01693EA
:10838000DFB2002F04D019A801223946F7F7DEFE2C
:10839000002C05D019A8C01973492246F7F7C4FE6E
:1083A0003C193F2C05D80F98C0194021091BF7F73D
:1083B000D4FE12980228189801D2002002E0C0785A
:1083C000411E884115990870611E2E46E8B20228A8
:1083D0000CD1179A517019A9119AB8C9B8C2B8C965
:1083E000B8C2B8C9B8C2B8C9B8C20DE0179A1170FE
:1083F00019A9109AB8C9B8C2B8C9B8C2B8C9B8C220
:10840000B8C9B8C2C10709D180073546149C139A70
:10841000169B00D4D5E602208543D2E6FE203546E1
:1084200005401898149C139A169B290628D0CCE670
:1084300037A231E01691149078780B994143334874
:1084400008181F386F21C9430D9D7A180378D42767
:10845000D3554378D827D3558378DC27D3550029C3
:1084600000D170E6C378E027D3551031001D189F66
:10847000EBE70120404A10E00024002D00D087E601
:1084800029B0F0BD80290ED30F20B872104817997B
:108490008883102020E525A20120014602F0BAFCC5
:1084A000189829B0F0BD1020402904D3B8720849AB
:1084B000179B998310E5B872044817998883142094
:1084C0000AE5C0462BC3000024C30000150F0000BE
:1084D000140B000001080000256420256420256499
:1084E000202564202564202564202564202564201F
:1084F00025642025642025640D0A00005ADB000055
:108500001DF7FFFF72D2000089FBFFFF62DA000057
:108510007472785F6D6F646520706172616D6574EF
:108520006572206572726F720D0A00004E73666488
:1085300020706172616D65746572206572726F7210
:108540000D0A0000FFFFFFFF01FF000058C60000FA
:10855000FFFFFFFFFF0101FFFF01FF01FFFF01FF21
:10856000FFFFFF01FFFF01FF5CC80000FFFF01FFED
:1085700078C60000E8C5000010D20000002800D135
:10858000014806490860704760900102F0B586B066
:10859000002805D10148006802E0C046BC930102F2
:1085A0003121C900049141188A791F231A40CD79DD
:1085B000ED06AD0DAA180D7AED066D0C52194D7A27
:1085C000ED062D0B52198D7AED06ED095219CD7A73
:1085D000ED06AD0852194D7CED075219BD4C2260D5
:1085E0000A7B1A404E7BF606B60DB2188E7BF60655
:1085F000760C9219CE7BF606360B92190E79F6069A
:10860000F60992194E79F606B608921962604A6A1E
:10861000B14D2A40A2608A6A2A40E2602D22D2002F
:1086200087183A7E1A4003937E7EF606B60DB2187E
:10863000BE7EF606760C9219FE7EF606360B921971
:108640003E7FF606F60992197E7FF606B608921965
:108650000E7CF60792192261BA7F1A400597FE7FB9
:10866000F606B60DB218049BC35CDB065B0CD21891
:108670004B78DB061B0BD2188B78DB06DB09D21894
:10868000CB78DB069B08D2186261CA692A40A261D6
:108690000A6A2A40E2618A7C01252A40CB7CDB07FA
:1086A0009B0F9A180B7DDB075B0FD2184B7D9B0746
:1086B000DB0ED2188B7DDB079B0ED218CB7D1B0700
:1086C0009B0D9A180B7E1B079B0CD2184B7E5B06EA
:1086D000DB0A13438A7E520612091A43CB7E5B07DC
:1086E0005B0813432362CA6A62620A6BA2624A6B26
:1086F000E2628A6B22633922D200835C1E462E40DE
:1087000066635E425E41B304AE04744F3C68B4439A
:10871000E3183B6083185A782A409C782407E40EBB
:10872000A2188C8F6401A2186D4C1440C98FC90522
:10873000490A0919DA78D207120A89181A79120730
:10874000120989185A79D207D2088918FB4EB163E9
:108750009968F163997904952940DA79D207920FE3
:1087600051181A7B5207D20E89185A7BD206920DE5
:1087700051189A7B5207D20C8918DA7BD206920BD9
:1087800089181A7CD206520A89185A7C5207920913
:108790000A43997CC906490851183164D97C039A67
:1087A00011401A7DD206920D51185A7DD206520CF4
:1087B00089189A7DD206120B8918DA7DD206D20961
:1087C00089187164197E0F2421405A7E12015118B4
:1087D0009A7E12038918DA7E1207120A51181A7F3C
:1087E0001207120989185A7F12078918B164997FF4
:1087F00001942140DA7F1207120E51183D22D20057
:10880000835C5B075B0D5918841862781207520C61
:108810008918A278D206120B8918E278D206D209FA
:108820008918F164217907220A406179C900891801
:10883000A2795206920B5118E2799207120B89180D
:10884000227AD2078A18BF490A60627AA37A1B0289
:108850009A18E37A1B04D2184A60E289BA4B134093
:108860000394228AD2049209D2188A6003463033D4
:10887000598CB64A114002939A8CD205D20A5118EB
:108880005622825C12068918B14D29600146563184
:108890004A788C782402A2188C8864056409A2188E
:1088A000CC78240712196A60CA880C7AA407A40B32
:1088B000A2184C7A6407E40A1219AA604989E9608F
:1088C000492189004118FF22663282180092103532
:1088D000002207E000300040FFFFFF0004040040DA
:1088E000FF3F000084186427E65D03273E406523B0
:1088F000E35C9B071B0F9B196626A65DB607B60EA9
:10890000F3186726A65DB601F318DBB26826A65DEC
:10891000B607B60DF3186926A65DB607360DF3182F
:108920006A26A65DB607B60CF3186B26A65DB607D9
:10893000360CF3186C26A65DB607B60BF3186D2639
:10894000A65DB607360BF3186E26A65DB607B60A07
:10895000F3186F26A65DB607360AF3187026A65DD3
:10896000B607B609F3187126A65DB6073609F318DF
:108970007226A65DB607B608F3187326A45DA40791
:10898000E31808C51032802AACD1019AD243704E48
:10899000B4180B783B404D78AD072D0FEB188D7850
:1089A000AD07AD0EEB18CD78AD01EB18DBB20D794C
:1089B000AD07AD0DEB184D79AD072D0DEB188D7989
:1089C000AD07AD0CEB18CD79AD072D0CEB180D7A7A
:1089D000AD07AD0BEB184D7AAD072D0BEB188D7A6B
:1089E000AD07AD0AEB18CD7AAD072D0AEB180D7B5C
:1089F000AD07AD09EB184D7BAD072D09EB188D7B4D
:108A0000AD07AD08EB18CD7BAD07EB18A3641031B3
:108A1000121DBDD1009B19785A785207520D51187A
:108A20009A78D207120D8918B164059B1968F16410
:108A3000D97D5A681202511831659968454A0A4031
:108A4000998A490589187165D9683D4C2140B165FD
:108A500019692140F165029E3178049D2940827890
:108A60005207120F5118C2799207920E8918427A52
:108A70009207920D5118827A9207120D8918C27AC4
:108A8000D207920C89189A7DD207520C89187278F5
:108A90009207D20B8918B2781207D20A8918F27895
:108AA0001207D2098A182C490A60327C737C1B0792
:108AB0001B0D9A18B37C9B069B0BD218F37C1B07EB
:108AC0009B0AD218337DDB065B09D218737DDB0766
:108AD0001B09D2184A60B27D2A40C38F5B009A18E6
:108AE0008A60826CCA60C26C22400A61F27D7F2378
:108AF0001340328C5204520AD2184A6102698A61C8
:108B00004269CA6182690A62C2694A62026A8A6209
:108B1000426ACA62826A0A63C26A4A63039A927CA0
:108B2000D201121D0A64027A3A40CA65808F074A50
:108B300010400866002006B0F0BDC046003000407E
:108B4000FFFFFF009C300040FF1F0000FF030000FC
:108B500000400040FFFF1F00002000400448006864
:108B6000806B800803490968490040180930704744
:108B7000BC9301021004004010B52D21C90041181A
:108B8000027A032A04D10079002807D0082006E0E1
:108B90008378DA1E022A05D2032412E014208860AA
:108BA0001C203DE0012B02D1C8228A6012E004792A
:108BB000042C01D3462404E0032C01D1322400E02C
:108BC00014248C605B1E022B04D3022A10D242793B
:108BD000154B01E04279154B9B181B78402B04D0B4
:108BE000102B06D11423442405E02A233E2402E05E
:108BF0004279342348244B800C80022A06D0062A6E
:108C000008D0052A08D118224C2301E01422502351
:108C10000B8000E01C224A80C078042803D1142075
:108C200048806420088010BD2BC3000024C30000CE
:108C3000134800687047C04610B5104A1070917014
:108C40000F49002813D050680861042048619078CB
:108C5000FF2212020B4B1C689443800380B2001960
:108C6000186001204007084A1060084A1060002080
:108C70000860074901220A6010BDC046AC9301029A
:108C8000180400401CE400E080E200E000E100E0A5
:108C900070000040F0B591B0002801D1C0480068D4
:108CA0008778F91E022913D3012F21D0022F3CD13E
:108CB0001021CA4344782146193991423DD8009782
:108CC0000125B94A28462946234602F0A3F853E174
:108CD0000821CA43447821462139914218D8009787
:108CE0000125B14A28462946234602F093F843E17C
:108CF0000821CA43447821460939914234D8009763
:108D00000125A94A28462946234602F083F833E183
:108D1000032F3CD0042F43D1C3780125042B00D06E
:108D20002DE106462A02042343E00125A6A2284697
:108D300029463B4602F06EF81EE1C3780125052B5B
:108D40000AD806462A02284698401B21084230D1FC
:108D50000021052B08462ED002200090914A28467B
:108D6000294602F057F807E10646C3780021022B96
:108D70001ED3032B1CD0042B08460A461BD001250A
:108D80000095884A2846294602F044F8F4E0C37862
:108D90000125032B00D0FAE006462A02032308E04F
:108DA000012583A2284629463B4602F033F8E3E03A
:108DB0000A46012148020F91592189007518FD21A9
:108DC000490071180291314662313F05D219641E83
:108DD0001F2727405C013C19144304433279520792
:108DE000D20C22432B789B065B0BD218B379DB079E
:108DF0001B0B13436D4D2B60F279032310931A4024
:108E0000737A9B079B0E9A18B37A5B07DB0D9A184F
:108E1000F37ADB079B0DD218337BDB075B0DD2188F
:108E2000737B1B075B0CD218AA603269EA60726917
:108E30002A61B2696A61F269AA61326AEA61726A98
:108E40002A62B26A6A620F980870F06AA8623F20CC
:108E5000C4432C353046E4300F903046E5300E9058
:108E60003046E6300D903046E7300C903046E83022
:108E70000B903046E9300A903046EA30099030468F
:108E8000EB3008903046EC3007903046ED300690DD
:108E90003046EE3005903046EF3004903046F030EA
:108EA00003903746F1373046F230F3360F990A19FE
:108EB0004021525C109B1A400E9B1B195B5C9B0768
:108EC0001B0F9A180D9B1B195B5C9B079B0E9A1836
:108ED0000C9B1B195B5C9B019A18D2B20B9B1B1954
:108EE0005B5C9B079B0D9A180A9B1B195B5C9B079D
:108EF0001B0D9A18099B1B195B5C9B079B0C9A180E
:108F0000089B1B195B5C9B071B0C9A18079B1B1982
:108F10005B5C9B079B0B9A18069B1B195B5C9B0772
:108F20001B0B9A18059B1B195B5C9B079B0A9A18E5
:108F3000049B1B195B5C9B071B0A9A18039B1B195C
:108F40005B5C9B079B099A183B195B5C9B071B09A1
:108F50009A1803195B5C9B079B089A183319595C94
:108F60008907891802C51034A0D10298007804211D
:108F700001430E48C1630025284611B0F0BD04200E
:108F80000090084A2846294601F044FFF4E70320F0
:108F90000090044A2846294601F03CFFECE7C04611
:108FA000BC930102E5D100002BD20000001000406C
:108FB000556E646566696E6564206D65616E2050EE
:108FC00052462025640D0A00496E76616C69642062
:108FD0006D65616E205052462025640D0A00000028
:108FE0007047704780B50E490E480246083A12682D
:108FF000920000D4603142680A4342600A490A681C
:1090000008239A430A60091F012252040A600321BF
:10901000890402688A430260FBF796F980BDC04666
:10902000200000802800004004020040B0B503206A
:1090300000072D490A688243012568071018086057
:1090400000242046FFF7CDFF2046FFF7C9FFEFF3CE
:109050001080284002D1EFF3108172B68021C943FD
:10906000224A13680B40136053680B4053609368A7
:109070000B409360D3680B40D36013690B401361BE
:10908000002800D162B6B0BD70B50C4603210907B7
:10909000154A13680B4313600122EFF3108111404E
:1090A00002D1EFF3108272B68025EA430F4B1E689F
:1090B00016401E605E682E435E609D6815409D6090
:1090C000DD681540DD601D6915401D61002900D176
:1090D00062B6002802D00120FFF783FF002C02D0E7
:1090E0000120FFF77DFF70BD0004004024A60102AF
:1090F0000D4A002907D001290BD1012181401068B8
:109100008843106007E00121814010680843106027
:1091100001E001218140101F02680A430121C907B3
:10912000114301607047C04644000040032804D842
:1091300040000649085A00B27047002000B270474C
:10914000032802D84000014A115270473CA6010290
:109150009E4908707047C04670B58AB00C460546F7
:10916000FF20FC30A8490E68315C59208000335C38
:10917000B278307808AE069609AE05960C4E049685
:109180002126760603960B4E0296012601960E26A0
:1091900000965B1CDBB2F9F773FA0998F7F7ACFAA3
:1091A00028700898F7F7A8FA20700AB070BDC0467A
:1091B0000000204100000443F0B58BB00446457C1C
:1091C000824800788249002822D000200880814A05
:1091D0001080814B01269E761E830A907F4800787E
:1091E0007F4E36786DB205957E4D04957E4D039584
:1091F0000AAD02957D4D01950096F8F77FFF0A9D17
:10920000112020567A497B4A00F06CFC064626E085
:1092100000260E806F4A16806F4B012098761883C7
:1092200009966E4800786E4F3F786DB205956D4D8A
:1092300004956D4D039509AD02956C4D0195009710
:10924000F8F75CFF099D112021567F20C005009092
:1092500001900296664A674B3046FAF7A3F843201E
:1092600001062846F7F76FF8F7F746FA08906248C4
:109270000078002824D05120800060494A7D424374
:109280008D185F480068A8642F4640375048007822
:10929000B87450480078F8745548007838755548C7
:1092A0000078787557480078F87550480069F7F7E6
:1092B00023FAB87552484069E8644C48006868640D
:1092C000FF20FE3050490968085C3922D200891815
:1092D000022812D303D04E48007801280DD14B4804
:1092E0000660434800883A4A108042480088394A5C
:1092F000108009200790089605E04448089A02600B
:109300003548C08B07900B780022002B01D0114606
:1093100000E0D1430125002B01D0042300E0EB4302
:10932000A67AAD1BEE175B1971416568AE0F277AFF
:10933000AD00ED195641677A3F1FF817ED197041DE
:109340004000EE0F80196D00EB1848418001990E26
:109350004118980127239B02C31A91411D48058893
:109360001B480088854201D00798421B10202056D8
:10937000C001194D2D8C032D07D1E468E5176D0A46
:109380006419E4150519EC170FE0E468E5176D0A98
:109390006519EC17ED15C6174519744197B2002FE2
:1093A00000D03446002F00D00546581BA1411304BD
:1093B00009D012B2D2015242D31780185941089BEA
:1093C000DA17C01A91410BB0F0BDC0464E930102AE
:1093D00090A301028EA30102149401025190010294
:1093E000509001026C9901026897010294A3010256
:1093F000DEA30102DCA301023C9D0102749A01027A
:10940000642000408CA30102BC93010288A30102E6
:10941000E0A30102C10D4002803070470120C00767
:109420001B4908607047C04610B519480068C1075D
:1094300010D1810711D4410712D4010713D4C106FA
:1094400014D4810615D4410616D48021084016D0C4
:1094500031A215E001240FA213E0022411A210E0B2
:10946000032414A20DE0042416A20AE0052419A284
:1094700007E006241CA204E0072421A201E0254AFB
:1094800004090220032101F0C5FC204610BDC0469E
:109490005C000040526573657420627920504F5221
:1094A0000D0A0000526573657420627920424F52A4
:1094B0000D0A000052657365742062792050494E90
:1094C0000D0A000052657365742062792057445478
:1094D0000D0A00005265736574206279204C4F4379
:1094E0004B55500D0A000000526573657420627977
:1094F000205357205265626F6F740D0A0000000000
:109500005265736574206279205359535245510D49
:109510000A0000003ACE000052657365742062793B
:1095200020445644440D0A0001218140044A1F286A
:1095300002D01068884310601068084310607047BC
:109540001C000040F0B585B0049104465F49F6F771
:10955000C1FD05465E4902942046F6F7BBFD5D4914
:1095600047185D49794301956D185C494418642199
:109570002046F6F7AFFD2818A108451A584920469D
:10958000F6F7BEFD2818574940180390564D07D4EA
:1095900003263E4064213846F6F79CFD019B18E007
:1095A00003262640A7B264213846F6F793FDB7207C
:1095B0004000002E01D1002907D14C4A7A430423F0
:1095C000DA414B4B9A4200D3401E019B039A82180A
:1095D00003925D4304980780481E814172427241A4
:1095E000424B7B430420C341414E0124B3422346F6
:1095F00000D30023029EAD19039F1F2F01DA2046DE
:109600004AE00A4013431F3F002B07D11C21791A5F
:1096100007D41F2907DA03200F463DE01D21791AE0
:10962000F7D5022038E03D2902DA1F390F4633E032
:109630005C2903DA3D3905200F462DE07A2903DA4B
:109640005C3906200F4627E0992903DA7A3907208A
:109650000F4621E0B82903DA993908200F461BE0AC
:10966000D62903DAB83909200F4615E0F52903DABF
:10967000D6390A200F460FE0B72042005B3A9142EC
:1096800001DB0C2000E00B20914203DB124A57184B
:109690005A3701E0F5390F46049EB070781CF0701F
:1096A000E12001012846F6F715FD3071C0B21149DD
:1096B00041434C193C212046F6F70CFD70713B21CB
:1096C000C94341430819B07105B0F0BD8051010094
:1096D0008033E101B207000093FEFFFFB1070000F5
:1096E00070FEFFFFA7FA0A0080AEFEFF295C8FC262
:1096F0000BD7A300F0F1FFFFB0B50446FFF796FCCF
:10970000A08A00281BD02A480ECC0EC00ECC0EC05A
:109710000ECC0EC027490020088027490A78521C29
:109720000A70D2B2142A06D1244A01231380087089
:10973000B54802210160954802210170B0BDE08A60
:109740001C4A1080A16912889148F6F7EDFC184D6B
:1097500028460ECC0EC00ECC0EC00ECC0EC0FFF7AD
:1097600067FA174908606C68FFF7F8F9201A15497D
:1097700008602846FFF720FD05460C467B48007B25
:10978000FFF7D4FC814901220A700B4900220A70BC
:109790000D490A68521C0A6081B2C90B401800B218
:1097A000C1174010094A281A10608C415460B0BD9E
:1097B0001CA701021AA7010278A60102809F0102DC
:1097C00074B301020CA6010210A6010218A6010240
:1097D000F0B581B0EFF3108072B600200146FBF7C0
:1097E00093FE044600280DD101273A030025074EB9
:1097F00028463146FBF7E4FDBB02814A2846314644
:10980000FCF754FA62B6204601B0F0BD00E0020455
:10981000F0B583B002F070FC544C607802F01AFA94
:1098200053498A8801A882800A88498809048918CE
:109830000191FEF777F96078052801D0022200E057
:1098400001224C49092800D0891849792078621CE6
:1098500002F0C4FA607AFFF77BFC47484749FDF7FE
:1098600093FCFFF7E5F9464908600027454A38466A
:10987000394602F073FCFDF7F9FB0028FBD1FFF736
:10988000D7F9414D28604148007801286CD1404CFF
:10989000207840490978814266D1607A202863D1D6
:1098A000FFF7C6F92860A67A3B4806706079A1796F
:1098B00009020D18394805800B34720038482146DA
:1098C000F6F732FC002E4CD03648036800223449AB
:1098D000009306E04000354B1D52009B521CB242E3
:1098E00024D05000085A8342F8D12F480378002B27
:1098F0000CD0314600202D4F3E88AE420BD0BF1C0D
:10990000401C8342F8D11F46184605E00027384620
:10991000172B05D9DEE7C7B20E462149172BD9D838
:109920009F42D7D15B1C204F3B70D3E7002E0ED057
:109930001C4801680020227863781B029A18914223
:1099400007D0A41C401C8642F5D1374609E0002709
:1099500007E0C4B22046F7F757FB0F480778A74245
:1099600002D13846F7F750FB03B0F0BD5290010228
:1099700048C300000497010225B00000F9960000DA
:1099800080B30102102700007CB3010277A6010218
:1099900084A60102F7A3010276A6010272B30102B6
:1099A00044A60102409D01029A96010268960102B6
:1099B00010B5124C20687F21C905F6F76BFC2060BA
:1099C0000F4880790F490A78101808700E4800680F
:1099D000022808D0012810D10D48012101700B4840
:1099E0000021017010BD09480178491CCAB23C2A07
:1099F00000D10021017002F0E7F810BDBCA5010202
:109A0000869F0102A4A701022095010208A4010279
:109A10004F93010270B514460D4606461120FAF721
:109A20000FFE2448042101600D48046022480560AF
:109A30000C480660002E0DD0FF2000060A490A6877
:109A400082430120C00710180860084808210160FF
:109A5000074801601A200221FFF74AFB70BDC0468B
:109A6000E8A701025C94010200E400E080E200E06B
:109A700000E100E00C4908607047C04610B504469C
:109A80000948006860430949F6F73AFB001908499C
:109A9000086008480022026002460C3A096811601A
:109AA00005490968016010BDE4A7010240420F00AA
:109AB000589401022C1001405494010200480047C0
:109AC000C100000080B506490968C96D884780BD9E
:109AD00080B5034A12689023D258904780BDC04693
:109AE0000090010280B582B013460A4600900348F8
:109AF000011D0348F9F702FC02B080BD28A801024D
:109B00009C96010210B50C498A1C90420DD2401E51
:109B10000D4A50600D4803680B4003218C071B1948
:109B2000036000209060116010BD04480449E622E3
:109B3000044B00F03FF9C046FFFFFF0011CE0000CC
:109B40002BCE0000F7CD000010E000E020ED00E09B
:109B5000B0B50120EFF31081014002D1EFF3108284
:109B600072B60E4A13680E4C2268646885060D486A
:109B700000682840850E5D192923DB006B43002C0B
:109B80001D4602D0121BD218551C002800D01D46BD
:109B90001E206843002900D162B6B0BD58B301024F
:109BA00014E000E004ED00E080B50020FAF740FF8B
:109BB000404280BDB0B586B0104869460A4638C8F4
:109BC00038C238C838C200242046FAF737FF039954
:109BD0002046FAF7CDFF0198012803D00824002879
:109BE00004D102E00424002800D104460220FAF740
:109BF0002FFDE0400249086006B0B0BD30C3000050
:109C00006CB30102F0B585B002F076FA584C60787A
:109C100002F020F857498A8803A882800A88498878
:109C2000090489180391FDF77DFF6078052801D0AC
:109C3000022200E001225049092800D08918497900
:109C40002078621C02F0CAF8607AFFF781FA4B486C
:109C50004B49FDF799FAFEF7EBFF4A4908600025EA
:109C6000494A2846294602F079FAFDF7FFF900280B
:109C7000FBD1FEF7DDFF454C206045480078012808
:109C800069D1444D287844490978012201928142E2
:109C90005ED1687A20285DD1FEF7CAFF2060AE7AD7
:109CA0003E4806706879A97909020C183C4804807E
:109CB0000B3572003B482946F6F736FA002E41D0A4
:109CC0003948036800223749029306E05800384BB0
:109CD0001C52029B521CB24224D05000085A8342AC
:109CE000F8D13248007800280CD031460023304F9C
:109CF0003E88A6420BD0BF1C5B1C9842F8D1074699
:109D0000034605E000273B46172805D9DEE7DFB20A
:109D10000E4624491728D9D88742D7D1401C234F53
:109D20003870D3E7002E0DD01F48016800202A7834
:109D30006B781B029A18914210D0AD1C401C8642D1
:109D4000F5D100E00026019D3046F7F75DF902E00D
:109D5000019D00E0019D284605B0F0BDC5B2284632
:109D6000F7F752F90D480678AE42019DF3D1EBE7C3
:109D70005290010248C300000497010225B0000080
:109D8000F996000080B3010280841E007CB30102BA
:109D900077A6010284A60102F7A3010276A60102BA
:109DA00072B3010244A60102409D01029A9601028B
:109DB0006896010290B01C4605AB07C3EFF3108014
:109DC000C00702D1EFF3108072B6EFF310800B9052
:109DD00068460E907046089010AB0F93CF4F3E1D13
:109DE00001200490C50230462946224600F09CFC22
:109DF00000213154EFF303800990EFF308800C90B9
:109E0000EFF309800D90EFF314800A9000F026FC28
:109E10003868012833D80028C14F00D0C14F2A200C
:109E2000C1497A69920703D50A783A60401E491CF5
:109E30000028F6D1B948041D2046FFF743FE00284C
:109E400007D079698907FAD521783960401E641CEA
:109E5000F5E70220B5497A69920703D50A783A6096
:109E6000401E491C0028F6D12A20AF497A69920782
:109E700003D50A783A60401E491C0028F6D1FFF746
:109E800067FE0346AA4A30462946FDF7BBFD044655
:109E90003018291B089F3B1F049A9343A5A2FDF786
:109EA000B1FD9E490968012966D8001900299C4C1A
:109EB00000D09C4C00280AD09849091D626992077D
:109EC00003D50A782260401E491C0028F6D10A20DA
:109ED0009F496269920703D50A782260401E491C97
:109EE0000028F6D10598FFF7EDFD002809D061693B
:109EF0008907FAD5059A11782160401E521C0592F7
:109F0000F3E7022089496269920703D50A78226043
:109F1000401E491C0028F6D10A208EA162699207D2
:109F200003D50A782260401E491C0028F6D1069805
:109F3000FFF7C8FD002809D061698907FAD5069A9C
:109F400011782160401E521C0692F3E702207749E7
:109F50006269920703D50A782260401E491C0028D6
:109F6000F6D10A207EA16269920703D50A782260A1
:109F7000401E491C0028F6D17CA230462946079B8A
:109F8000FDF740FD6549096801290E9B1BD8002992
:109F9000634900D0634900280AD0604A121D4C6909
:109FA000A40703D514780C60401E521C0028F6D17B
:109FB00002205E4A4C69A40703D514780C60401E49
:109FC000521C0028F6D16AA230462946FDF71AFD38
:109FD00004463018291B694A3B46FDF713FD4F49DB
:109FE0000968012911D8001900294D4900D04D49AF
:109FF00000280AD0494A121D4B699B0703D51378E4
:10A000000B60401E521C0028F6D15D4A304629469E
:10A01000099F3B46FDF7F6FC0446F800C00FB90067
:10A02000C90F7A00D20F0092019102903019291BBA
:10A03000FB0F544AFDF7E6FC04193019291B3F2396
:10A040003B40514AFDF7DEFC34490968012911D82B
:10A0500020180029324900D0324900280AD02F4A5E
:10A06000121D4B699B0703D513780B60401E521CD1
:10A070000028F6D1454A304629460B9BFDF7C2FC25
:10A0800004463018291B424A0A9BFDF7BBFC2349B2
:10A090000968012911D800190029214900D0214956
:10A0A00000280AD01D4A121D4B699B0703D513785F
:10A0B0000B60401E521C0028F6D1364A3046294615
:10A0C0000C9BFDF79FFC04463018291B324A0D9B60
:10A0D000FDF798FC114909680129114A0DD80019AA
:10A0E000002908D00F4A06E05169890703D5317865
:10A0F0001160401E761C0028F6D128490E98091AD6
:10A10000A94200D32946890800F00EFE24480068C1
:10A11000002800D0804700F045F8C0469CB30102FB
:10A120000090014000A001406BCE00004FD2000023
:10A1300054CE00000D0A232323204153534552548B
:10A14000204020307825303858202323230D0A0062
:10A150002ECF000046554E4354494F4E3A20000042
:10A160004C494E45202020203A2000002564000064
:10A170000D0A53503D253038580D0A00F3CE00002B
:10A1800009CF000015CF0000FDCE0000B2CE0000C8
:10A19000C1CE0000D0CE0000DBCE000000F80202ED
:10A1A00098B30102F4480068012811D8002801D0B2
:10A1B000FB4800E0F9480C21094A01E0002907D0DA
:10A1C00043699B07FAD513780360491E521CF5E7D3
:10A1D0001E20FFF7A9F900BF00BF00BF00BFFAE7CC
:10A1E0005ECE00008AB00646E248B06600F036FA5D
:10A1F000FFF7AEFC0346E048041D01200590C502B0
:10A20000DE4A20462946FDF7FDFB07460894201844
:10A21000D94C0995E91BF36C3F2206921340D8A252
:10A22000FDF7F0FB2168012910D8C0190029DB498E
:10A2300000D0DB49002809D0221D4B699B0703D5BC
:10A2400013780B60401E521C0028F6D1F36BD5A288
:10A25000089C2046099D2946FDF7D4FB0746291A8C
:10A260002018336C069A134003D1D6A2FDF7CAFB1F
:10A2700002E0CEA2FDF7C6FBBF4C2168012910D831
:10A28000C0190029C54900D0C549002809D0221DA0
:10A290004B699B0703D513780B60401E521C0028A6
:10A2A000F6D10027CBA5B80030580090089809993E
:10A2B0002A463B46FDF7A6FB216801290FD8002955
:10A2C000B64900D0B649002809D0221D4B699B072A
:10A2D00003D513780B60401E521C0028F6D17F1C5A
:10A2E0000D2FE0D1736BBFA2089C2046099D294623
:10A2F000FDF788FB074620189F4CE91BB36BBC4A4F
:10A30000FDF780FB2168012910D8C0190029A34955
:10A3100000D0A349002809D0221D4B699B0703D513
:10A3200013780B60401E521C0028F6D1336CB14AE2
:10A33000089C2046099D2946FDF764FB0746326CC0
:10A34000D000C00F9100C90F5300DB0F00930191A3
:10A350000290E019E91BD30FA74AFDF753FB3246E1
:10A36000C619A019A91B1546136C069A1340A34AD7
:10A37000FDF748FB80490968012911D88019002997
:10A38000864900D0864900280AD07B4A121D4B69B5
:10A390009B0703D513780B60401E521C0028F6D192
:10A3A0002E466B6C964A089C2046099D2946FDF76F
:10A3B00029FB07462018E91B0796B36C914AFDF765
:10A3C00021FB6D4A1168012910D8C0190029734971
:10A3D00000D07349002809D0121D4B699B0703D593
:10A3E00013780B60401E521C0028F6D10798426E6D
:10A3F000042360215C2004931A400B4600D00346DE
:10A400000693002A00D00846079E33587E4A089CCF
:10A410002046099D2946FDF7F5FA07460698335868
:10A42000E019E91B794AFDF7EDFAC619A019A91B35
:10A43000079A536E76A2FDF7E5FA4F49096802299B
:10A4400011D280190029554900D0554900280AD059
:10A45000494A121D4B699B0703D513780B60401EB8
:10A46000521C0028F6D10798C36C06466DA2089CC2
:10A470002046099D2946FDF7C5FA07462018E91B25
:10A48000336D6B4AFDF7BEFAC619A019A91B079FC9
:10A490007B6D68A2FDF7B6FA8619A019A91BBB6DE2
:10A4A00067A2FDF7AFFA344909680129059C11D864
:10A4B00080190029394900D0394900280AD02E4A8C
:10A4C000121D4B699B0703D513780B60401E521C6D
:10A4D0000028F6D10798476B5D4A974237D2032090
:10A4E00087430026059CB00039580246049B1A4356
:10A4F000BA5808230343FB580C2505437D590091A6
:10A500000192029303953B1808980999514AFDF767
:10A5100079FA1949096801290FD800291F4900D083
:10A520001F49002809D0089A4B699B0703D5137867
:10A530000B60401E521C0028F6D11B2E444A06D840
:10A540000798406B361DB10040189042CBD3079856
:10A55000406B111A099A914201D8890800E0610202
:10A5600000F0E2FB3C480068002800D08047FFF77D
:10A5700019FEC04622224B4D9CB3010254CE00006E
:10A580000D0A0D0A23232320455843455054494FB3
:10A590004E202564202323230D0A00000090014053
:10A5A00000A0014050433D25303858002C2045780C
:10A5B00063657074696F6E4E756D6265723D25647A
:10A5C0000D0A00002C205468726561644D6F64654B
:10A5D0000D0A000052252D32643D253038580D0AF1
:10A5E0000000000053503D253038580D0A0000008F
:10A5F000F3CE000009CF000015CF0000FDCE000013
:10A60000B2CE0000C1CE0000D0CE0000DBCE0000F4
:10A610004558435F52455455524E3D253038580DEC
:10A620000A000000494353523D253038580D0A00B6
:10A63000E6CE00005343523D253038580D0A000045
:10A640004343523D253038580D0A0D0A00000000E2
:10A6500000F8020296CE000098B30102F0B581B076
:10A66000284D2C68012C06D8601E8441204601F03C
:10A670009BFA0028FAD10120EFF3108101400091EC
:10A6800002D1EFF3108072B61F482A5A1F48295A88
:10A69000914208D12348002129540098002800D174
:10A6A00062B601B0F0BD2B68002B01D0194C07E059
:10A6B000174C05E0024614482A5290B28142E9D074
:10A6C00097B2B942084601D81348401C861A134A6B
:10A6D000AE52012B0FD832040DD0EA19121DB7B2B9
:10A6E00001E0002F07D06669B607FAD51678266014
:10A6F0007F1E521CF5E7084A9042DBD9084A8218AF
:10A70000D9E7C0469CB301020A080000080800000F
:10A710000090014000A00140FF0700000C0800006D
:10A7200000F8FFFF0F080000F0B58DB00793174643
:10A7300000240C9409AA13C215E006986849F5F79D
:10A7400002FEF5F7D9FFC117401848406549F5F7F3
:10A75000C1FC009509A806223346F9F725FBB9E0AC
:10A76000002C00D5B2E138787F1C25280DD00028B8
:10A7700000D1ABE10B9A511C0A9B9942F0D8099B7E
:10A780009854641C0C940B91EAE7089400253978DE
:10A7900023390D2914D801207944097949008F44BF
:10A7A000090F0F0F0F0F0F0F0B0F060F0F0D0543A4
:10A7B0007F1CECE70820FAE70420F8E70220F6E720
:10A7C0003878014630390024092902D9264639460D
:10A7D0000BE000260A2171430E18303E791C787870
:10A7E0000246303A0A2A0F46F4D32E2813D14A1CC7
:10A7F000487801463039092901D911460BE0002477
:10A800000A2161430C18303C511C50780246303A02
:10A810000A2A0A46F4D34F1C2538532800D959E098
:10A820004000C04678448088400087449D00530023
:10A830005300530053005300530053005300530080
:10A840005300530053005300530053005300530070
:10A850005300530053005300530053005300530060
:10A8600053005300530053005300530053005D0046
:10A870005300530053005300530053005300530040
:10A880005300530053005300530053005300530030
:10A8900053009500530053005300530053005300DE
:10A8A0005300530053005300AA00B30053005D004F
:10A8B00053005500530053005300550053005300FC
:10A8C0005300DB0053005300BA005300D000530084
:10A8D000530095000C9C43E7791C38780F469BE7A2
:10A8E0000024744940420F000799C91D0720814385
:10A8F000086807914968F5F765FF00210690F5F7AC
:10A9000099FE00280BD10B99481C0A9A904206D850
:10A91000099A2D2353540899491C0C910B900798C0
:10A92000083007900698F5F7E7FE0095C2178118E2
:10A93000514009A822463346F9F736FA0B98411CD4
:10A940000A9A914200D9F8E6099A2E2313540B91E2
:10A950000C98401C0C90F0E6079802C807900096EF
:10A96000019509A8102239E00B98411C0A9A9142DE
:10A97000B0D8099A252313540B910C98401C0C90C5
:10A98000A8E70B9A511C079C201D0A9B994239D9B4
:10A9900007909FE7079802C80790009509A82246EC
:10A9A000DAE6079901C9079109990A9A089E02E017
:10A9B000401C002E8ED40378002B8BD00B9D6C1C7A
:10A9C0009442F5D84B55761C0C960B94F0E70798FB
:10A9D00002C807900096019509A80A222346F9F7B4
:10A9E0007BFA77E7079B10CB102C079308D3002046
:10A9F0002146401C0A09FF291146FAD806280AD820
:10AA0000082009E02368099CA354089A521C0C9260
:10AA10000B9107905EE7401C069009230C980B9D54
:10AA2000099905910A9E04940DE0202104463046C0
:10AA3000059E715506462046049C401C154601465D
:10AA40000891002908D45B1E0699994204D26A1C19
:10AA5000B242EAD90899F3E70C900B9508980028C0
:10AA600000D537E70126082501E06D1E3601022DCD
:10AA7000FBD220463146F5F72DFB0F28F6D80C986F
:10AA80000590099803900A9806900B9D2046314640
:10AA9000F5F720FB691C069A914201D9089908E054
:10AAA0000C4A125C039B5A55089A521C0D4605929B
:10AAB00011460891002905D47043241A3009102E3C
:10AAC0000646E3D205980C900B9503E720460DB09F
:10AAD000F0BDC046B8C5000070B588B0002203289C
:10AAE00001D9D2431EE07E4CC24D2A510F4B104E6D
:10AAF000EE5081231E010123AB5528602C196260A2
:10AB000001280FD80793002206920592049203238E
:10AB10000393029201920091411E8841694600F020
:10AB200007FD0246104608B070BDC046040800008C
:10AB3000FFC0FFC0F0B583B00C460023D943012C01
:10AB40001BDB074602910126EFF31085354002D149
:10AB5000EFF3108072B65649564A505C002800D078
:10AB60009FE056545D48115A5D48105A0196F20212
:10AB7000161A814203D8324602E00C468EE0424269
:10AB80005218A24211DA594A4A4EB25C002A45D004
:10AB9000574AB25A51188AB2524CA242444C029FB0
:10ABA00001D9514A89184E4A3BE000930295A642CA
:10ABB000354600DB25463F490818001D39462A4620
:10ABC000F5F7B2FAA6423B4E04DA7919621B301D42
:10ABD000F5F7AAFA4248305A001981B2414A914227
:10ABE00001D941494018029D009B3D4970523046B1
:10ABF0003E4E805D00284BD1EFF310850198054053
:10AC000002D1EFF3108072B62A4A3448115A344800
:10AC1000105A884218D13648135235E0244C304A35
:10AC2000029F3355B152421A89B2884202D22D484E
:10AC30008018421C93B23048012130A200F0EAF89B
:10AC40003C46002D2AD128E0019F9755884201D823
:10AC50002448401C421A90B2800A01D00198820216
:10AC60002348144F3A52386801280DD8431E9841A2
:10AC7000104B5918091D92B21E4B00F03DFE009B6F
:10AC8000002801D00B488355002D029D00D162B6EB
:10AC9000074808490B54002D00D162B6204603B086
:10ACA000F0BD054805A1094A09A3FFF783F8C0468E
:10ACB0000E0800009CB30102AACF00007472616309
:10ACC000655F6F7574707574000000000E020000FF
:10ACD0005452414345204255535900000A08000090
:10ACE00008080000FF07000000F8FFFF0F08000041
:10ACF0000C08000041AF000002FF00000D0A547272
:10AD00006163652062756666657220697320667589
:10AD10006C6C2C20646973636172647320257520E8
:10AD200062797465730D0A00F0B587B00546002698
:10AD300006960596049603960296800701D007B002
:10AD4000F0BD019102A8142126A2FCF75BFE29495F
:10AD50000968012911D80029274900D0274900286E
:10AD60000BD002AA01E0002807D04B699B07FAD557
:10AD700013780B60401E521CF5E701990029DED0C4
:10AD8000204C3746B8002B58D80724D0581EA04274
:10AD900004D31B4818181C4A90421CD802A814213E
:10ADA0001AA2FCF72FFE13490968012911D80029BE
:10ADB000114900D0114900280BD002AA01E0002857
:10ADC00007D04B699B07FAD513780B60401E521CC5
:10ADD000F5E7761C01997F1C8F42B0D2322ED1D379
:10ADE000ADE7C0460D0A4261636B74726163653AF8
:10ADF000200D0A009CB301020090014000A0014018
:10AE0000FFFFFFFCFFFF0200FEFF01002530385866
:10AE10000D0A000081B0F0B5C4B00E460746499354
:10AE2000812000012F49085C002845D002920120B2
:10AE3000050204A82946F5F790F9FCB20021C843A1
:10AE40000C2C3AD8721E032A37D82748005DB0422E
:10AE5000084632D3F80535D50021B8050DD404A82D
:10AE600001904018691AA20022A39B582E4AFCF7B1
:10AE7000C9FD0198FEF726FE014678050ED404AF01
:10AE80007818691AB20029A3D218121F1368264A2B
:10AE9000FCF7B8FD3846FEF715FE0146029A04AEEF
:10AEA00070180C46691A49AB0393FFF73DFC011972
:10AEB0003046FFF73FFE00E0002044B0F0BC02BC8B
:10AEC00001B00847FEF744FE034604A8019007A21C
:10AED0002946FCF797FD0198FEF7F4FD0146B805F9
:10AEE000BDD5CAE79CB3010232DE000025313075C2
:10AEF000207C20004ECF0000A4CF00009ECF000099
:10AF00007DCF000048CF000069CF000097CF000040
:10AF100090CF00008BCF000041CF000054CF000045
:10AF200064CF000039CF0000C5CF000083CF000000
:10AF30006FCF000076CF00005ACF00000000000065
:10AF4000F0B581B00B460120EFF31084044002D12C
:10AF5000EFF3108172B6990F07D0022001212DA2C4
:10AF6000FFF758FF002C3DD141E02249224D002738
:10AF70006F54224AAB5A224AAE5AF3189EB2F60ACE
:10AF800001D0204E9B19AB52EFF31086064002D140
:10AF9000EFF3108372B6AA5A1C4BEB5A934202D1BC
:10AFA00016482F521AE06854934201D8164B5B1C86
:10AFB0009B1A99B2890A00D0830210482B52286844
:10AFC00001280BD8411E8841A918091D9AB2104BBF
:10AFD00000F092FC002801D006482F54002E03D028
:10AFE000002C04D001B0F0BD62B6002CFAD162B6DC
:10AFF00001B0F0BD0F0800009CB301020C08000076
:10B000000A08000000F8FFFFFF0700000808000022
:10B0100041AF000055415254204572726F72202595
:10B02000780D0A0010B582B00446FDF7FFFFA08A34
:10B03000002801D002B010BDFDF7FAFD08490860F4
:10B040000849086008480168491C0160074803680E
:10B050000091032006A20146FFF7DCFE02B010BDFE
:10B0600074B3010288B3010280A6010210A6010296
:10B07000706F6C6C5F72785F6E756D2069732025E0
:10B08000642C726573705F74785F6E756D20697380
:10B090002025640D0A000000B0B50A2000242146D6
:10B0A000FBF726FC09202146FBF722FC0124204661
:10B0B00000F02CF80E2004252946FBF719FC0D2082
:10B0C0002946FBF715FC1049204600F031FAB0BDC7
:10B0D000B0B50E2000242146FBF70AFC0D202146C6
:10B0E000FBF706FC0124204600F010F80A20042596
:10B0F0002946FBF7FDFB09202946FBF7F9FB02492E
:10B10000204600F015FAB0BD6094010270B5012828
:10B1100001D9012070BD48224243F64B9C58A569D5
:10B120001F218D43A5610625A5600F2525629C186A
:10B13000A27C002A05D1627C002A02D1227C002A4E
:10B1400014D06368002B11D4251D0B400122164634
:10B150009E400C4B1E60BFF34F8FBFF36F8F2B6869
:10B16000002B03D40B409A4007490A60002803D003
:10B17000012804D1092000E00820F9F759FA00203D
:10B18000A06170BD80E100E080E200E0F0B585B034
:10B190000D460278D748C36893421AD0446D944252
:10B1A00017D08368934203D0016D914200D07BE0B9
:10B1B0009B1A591E8B41049348215943032D3FD1BB
:10B1C0004418E169002947D01C340020206005B0F4
:10B1D000F0BD9B1A5A1E93410493032D1AD1039577
:10B1E00048225A438418A26B0121EFF310850D40C9
:10B1F00002D1EFF3108772B6A7691026B743A76193
:10B20000A669002E01D118342160002D00D162B64C
:10B21000039D0CE0482159434218916918323029A6
:10B2200002D01168102947D18021116000224821E5
:10B2300059434018002181630162816224302AE071
:10B24000421891691832302902D0116820293CD166
:10B2500080211160002216E00395E26B0126EFF3D6
:10B260001085354002D1EFF3108172B6A169202715
:10B27000B943A161A169002901D118342660002DCC
:10B2800000D162B6039D4821594340180021C16393
:10B29000C1624163303000210160002A97D004A8C8
:10B2A0002946904705B0F0BD00920D4A2E329248D3
:10B2B0000C490D4BFEF77EFD1068009301908E48FF
:10B2C0000849074A094BFEF775FD10680093019085
:10B2D000034A2432F9480349044BFEF76BFDC0468C
:10B2E000B102000029D00000FECF0000E2CF000034
:10B2F000F0B585B0049048210A4642437D4B9C58E6
:10B30000E6690F2535409A18167C002E33D04F2061
:10B3100040026169014260D0A06904218843A061B4
:10B3200002202062012081076918D161D36BEFF3FD
:10B330001084044002D1EFF3108572B6956920267F
:10B34000B54395619569002D02D1154618352860E1
:10B3500010463C30002C00D162B600240460D46258
:10B360005463303200201060002B00D1B6E004A8F6
:10B37000984705B0F0BD0C2D00D9AFE07D442D7984
:10B380006D00AF445AAB5CAB06AB8E58ABABABAB0E
:10B3900006009569202D05D0154618352D68302DED
:10B3A00000D09BE0156B566B3432AE421BD26669FF
:10B3B000360718D5646815686E1C1660484318185F
:10B3C000C06A445504980C4644431A19156B566BD1
:10B3D0003432AE4207D21C59E9E70C2D9CD0012D26
:10B3E00000D199E77AE01268AA4200D076E04143A2
:10B3F000585882690524A24382615A18D36B0121EF
:10B40000EFF31080084002D1EFF3108472B6946914
:10B410002025AC4394619469002C02D11446183461
:10B42000216014463C34002800D162B6002121601E
:10B43000D162516395E7042034E0012032E0082511
:10B440002562164618369569102D02D03568302DC4
:10B4500046D10396566A15462835976AB74224D1D5
:10B46000A06902218843A061936B0121EFF3108052
:10B47000084002D1EFF3108472B6039E346810279F
:10B48000BC4334603468002C00D131601446383439
:10B49000002800D162B600212160296011622432A7
:10B4A00060E70220206205B0F0BD2A68B24215D2E2
:10B4B0006269920712D52A68561C2E6048431818F4
:10B4C000006A805C206004980A4642439D18AC6A7A
:10B4D0006E6AB44202D228359C58E9E705B0F0BD47
:10B4E000316800900191044804A1094A09A3FEF7BC
:10B4F00061FCC04680940102C8CF0000756172747F
:10B500005F6972715F68616E646C65720000000053
:10B510003D030000556172742025642073746174CA
:10B520006520676F65732077726F6E6720256400F2
:10B53000F0B585B00E460546022804D3002E02D190
:10B54000012005B0F0BD002D03D0012D08D1092444
:10B5500000E008242046F9F773F82046FDF7E4FFE1
:10B5600048216943DC4A505883691F240294A3434D
:10B570008361062383600F2301930362571800231E
:10B58000BB62BB63FB633B627B62FB623B63317FFD
:10B590003974727F7A74B27FBA7404937B63736870
:10B5A000B268F468920022435B1E032B0ED8C0469B
:10B5B0007B441B795B009F4401050307082304E0DB
:10B5C000282302E0182300E038231A43C260C90789
:10B5D000090F72699201D2B28918B2699207920E6C
:10B5E0008918491C816079613169012901D12221C1
:10B5F0000161012D5CD831680E2959D238461230CC
:10B6000003900324002D01D0204600E004204C4389
:10B610002D490E19B178F9F78FF83968CA68802575
:10B6200010462843C8602848005D73781B0218182C
:10B63000C862AA43CA60F9F7C7F8039800780028DF
:10B6400009D1384611300078002804D1384610302E
:10B650000078002827D07868002815D403210246F6
:10B660008A431B4953588407E40EFF26A640B34380
:10B67000A5401D435550029901400120884097493B
:10B680000860144908600EE08107C90EFF228A4055
:10B69000019C0440083C032084430C4823589343F6
:10B6A0008D401D4325500120B861049805B0F0BDC0
:10B6B00002480349DA22034BFEF77CFBC8CF0000A7
:10B6C0003BD0000018D000004EC300001CED00E08D
:10B6D00000E400E000E100E0F0B58FB00E9001253D
:10B6E000002900D19CE0039304910592002A00D127
:10B6F00096E00121EFF3108201910A4002D1EFF3AD
:10B70000108172B64827029747437349CE19B5692D
:10B710000023302D23D831461831C0467D442D7981
:10B720006D00AF44202426262626262626262626F9
:10B730002626262659262626262626262626262676
:10B7400026262626182626262626262626262626A7
:10B750002626262618000223002A0CD00CE0402DB5
:10B7600001D0802D05D10123002A04D004E020243B
:10B770000C60002A00D162B61D46002B50D1002576
:10B7800075630399F1630499F16205993163524C31
:10B79000E35959691322D202114205D0062199605A
:10B7A0000F21196271699960317C00290CD0F56113
:10B7B00009950895079506950D950B9502210A9117
:10B7C00001280ED017200DE0717C9A6900292AD03B
:10B7D000952002439A6123E030240C60002ACAD0ED
:10B7E000CAE71920049F0C907068002805D41F2117
:10B7F0000840019981403948016014209861B0687F
:10B8000006A9F9F751F80E9802994143601880682B
:10B810006158E44A0092091D3A46059BF9F7B4F8CD
:10B8200028460FB0F0BD3436110602D580218A4378
:10B830009A6131680025059A914229D205955D6982
:10B840004F214A0215421BD1E90502D4029CDD4F6B
:10B850000AE0596833685C1C3460029C6043D94F2D
:10B860003818C06AC1540E98214641437E18736B44
:10B87000346BA3422BD234367B585D691542E3D03A
:10B8800002211962019EB10729433546CD4C01E0E2
:10B890002946019EEFF31082324002D1EFF310836C
:10B8A00072B6029B4343E01883692024A34383615B
:10B8B0008369002B02D1034618331E60002A00D191
:10B8C00062B6C26B002AABD00EA89047A8E7294603
:10B8D000059D019E3C46DDE78094010280E200E088
:10B8E00080B5012002496422024BFFF7F5FE80BDBE
:10B8F00014A50102E1B80000F0B591B01090012646
:10B90000002900D1ECE003930591002A00D1E7E083
:10B9100007900121EFF310800291084002D1EFF36C
:10B92000108172B604924823069307994B43A549A8
:10B93000C9188D690026302D6ED80C461834AD001C
:10B94000374602A675593E46AF46C04621BA0000AA
:10B9500029BA00002DBA00002DBA00002DBA00004F
:10B960002DBA00002DBA00002DBA00002DBA00003B
:10B970002DBA00002DBA00002DBA00002DBA00002B
:10B980002DBA00002DBA00002DBA000011BA000037
:10B990002DBA00002DBA00002DBA00002DBA00000B
:10B9A0002DBA00002DBA00002DBA00002DBA0000FB
:10B9B0002DBA00002DBA00002DBA00002DBA0000EB
:10B9C0002DBA00002DBA00002DBA0000B5BA000053
:10B9D0002DBA00002DBA00002DBA00002DBA0000CB
:10B9E0002DBA00002DBA00002DBA00002DBA0000BB
:10B9F0002DBA00002DBA00002DBA00002DBA0000AB
:10BA00002DBA00002DBA00002DBA000011BA0000B6
:10BA1000022600280CD00CE0402D01D0802D05D14D
:10BA20000126002804D004E010252560002800D15C
:10BA300062B6002E069D634F049C079850D10026E5
:10BA40008E62039A8A63059A0A624C620A7C002A13
:10BA50000BD00C960B960A96099608960E96022223
:10BA60000D9201282BD018202AE08A7C2831002A48
:10BA700039D00A68A24216D22B464343FA58546979
:10BA8000A40710D50868441C0C60F918096A085C02
:10BA900010601098294641437A1811462831936A5C
:10BAA000526A9342E8D345437859816982220A4316
:10BAB000826115E0302525600028B9D0B9E71A2049
:10BAC0000F90C86808A9F8F7EFFE109845437A5917
:10BAD0007819C0683349009105992346F8F754FF57
:10BAE000304611B0F0BDFB589A69140602D5802487
:10BAF000A2439A610A680026049882422ED25D69A8
:10BB00004F225202154207980AD002211962029E62
:10BB1000B10729431FE028315D6915423E46F4D143
:10BB200037465C69A40702D40699264E0AE00C68E1
:10BB3000661C0E6006994843224E3018006A005D6C
:10BB4000186010984143735871188C6A4E6AB44259
:10BB5000E1D329463E46069D1A4F01E0314607983B
:10BB60005A6A002AFCD1EFF31082029B1A4002D1DC
:10BB7000EFF3108372B64543781983691024A34309
:10BB800083618369002B03D103461833029C1C6038
:10BB9000002A00D162B6826B002AA1D010A890477B
:10BBA0009EE7C0468DB10000482141430548421838
:10BBB0009269D20601D400207047405841690120A3
:10BBC000084070478094010280B511480078C00198
:10BBD00010490978890101430F4800784001084362
:10BBE0000E490978090101430D480078C000084357
:10BBF0000C490978890001430B480078400008434C
:10BC00000A4909780143C8B2F5F752FB80BDC04626
:10BC1000B2950102F5A30102A5930102B4BB010292
:10BC2000F6A30102B3950102689901026999010224
:10BC300004480068202801D0044800E00248044974
:10BC4000086070470C00004024D6010330CF010388
:10BC500000900102F0B587B00146012702250528B2
:10BC60003A4600D02A4600200929014600D0114654
:10BC7000C900374A54180E210591615EFDF760FA3C
:10BC80001026A15F3846FDF75BFA1227E15F2846D0
:10BC9000FDF756FA06951425615F03200490FDF721
:10BCA0004FFA0598235EA05FE15F625F00AD07C5B4
:10BCB00028A2069F3846049D2946FFF7ABF8204688
:10BCC000263004263146FBF70DFF2620235E282070
:10BCD000205E2A21615E2C22A25E009001910292D8
:10BCE00024A238462946FFF795F827463E373846BE
:10BCF0003146FBF715FF3E20235E06983C5EB95F98
:10BD00000622BA5E00940191029221A207462E46B5
:10BD10002946FFF77FF856240D4D285FFBF7F4FE08
:10BD20002B5F2C4621A2384631463546FFF772F884
:10BD3000264658363046FBF7D3FE5820235EF05F88
:10BD400000901FA238462946FFF764F807B0F0BDFF
:10BD500004970102546F4620616E742064656C6123
:10BD600079732025642025642025642025640D0A2C
:10BD70000000000050446F412064656C61797320BD
:10BD800025642025642025642025640D0A00000018
:10BD900050446F41206761696E73202564202564DB
:10BDA0002025642025640D0A0000000050446F41E6
:10BDB00020616E742073706163652025640D0A0034
:10BDC00050446F4120616E676C65206F66667365D5
:10BDD00074732025642025640D0A0000F0B587B037
:10BDE0001546764B1A680F24A2432F783A431A60FF
:10BDF000734C23462C3B734A1A6004900346224638
:10BE0000283A12681207FAD56F4E092F029306D905
:10BE1000714A326072600C2F09D171480FE0042F13
:10BE200007D96C4A32606C4A7260092F06D36D489C
:10BE300005E0664830607060654800E067486A4A1F
:10BE40001060EB7AFF2B039102D10020B0620AE070
:10BE500003210B406548C05C40220243B2620220CD
:10BE6000634AFEF7D7FF029F0021384605952A4610
:10BE70000B46FBF7AFFE0646022503215DA22846CE
:10BE800001913346FEF7C6FF06963046FCF776FB77
:10BE9000012104980091084006D02E4605460698D8
:10BEA000FCF7F8FE284635463D4006D02E460546AE
:10BEB0000698FCF76BFB284635465549002855D0B7
:10BEC0005448086154484861544888611520C86145
:10BED0005348016840220A430260072108033A4B95
:10BEE0005A6982430098400310185861052203984C
:10BEF00042433D4803689818454E766B47780F409B
:10BF0000995C0907490EC919CA03464B33409A1870
:10BF1000C9015118444A89183D4A51633C49896B0B
:10BF20003822914382785207920E891804220A43DC
:10BF300037498A63244B19690279019E3240C078DF
:10BF40004007C00E80181F22914308181861552021
:10BF50004003411C216020606420F8F735FC334A1F
:10BF60002A483146039BFEF755FF2949002D1ED074
:10BF70002F48A062E062206360632E4860622E4812
:10BF80000860152085046E1C8E608D606424204638
:10BF90000F46F8F719FC3E603D602046F8F714FCA8
:10BFA000281D3860032125A21848FEF733FF0598A5
:10BFB000007BFAF763FF069807B0F0BD0404004069
:10BFC0002C60004000040080000600400F040F04B5
:10BFD000CDC900000304030400040004FECA0000ED
:10BFE0009CC800002FCC0000C093010260CD00006F
:10BFF00067D0000050485920706172616D732073E2
:10C0000065747320253038780D0A0000020800009E
:10C010009060004012A83E009DD79B5AD579BD493B
:10C02000340200403F0080FF4040000049D0000043
:10C030002008820002D50F00020255007577625F6A
:10C0400072785F696E69740D0A00000080B522483D
:10C050000021017022480078C00120490978890137
:10C06000014320480078400108431F490978C9006E
:10C0700001431E480078800008431D4909784900A3
:10C0800001431C4800780843C0B2F5F711F980BDA0
:10C0900080B51148012101701048007880011049D5
:10C0A0000978C90101430F480078400108430E494F
:10C0B0000978C90001430D480078800008430C4905
:10C0C0000978490001430B480078084310210143D7
:10C0D000C8B2F5F7EDF880BDB4BB0102F5A30102CB
:10C0E000B2950102A5930102F6A30102B3950102E4
:10C0F0006899010269990102F0B581B01820FDF735
:10C1000013FA1920FDF710FA002420462146F7F70C
:10C1100083FF20462146FAF735FE012603257F23BB
:10C12000304629462A46FAF73FFF3046FBF7E4F847
:10C1300002273846FBF72EFD30463146FCF77CFDE2
:10C1400003A238462946FEF765FE204601B0F0BD41
:10C150007577625F6F70656E0D0A0000F0B581B093
:10C16000164600910446002001273946FCF78CFF53
:10C17000EFF310853D4002D1EFF3108072B6272017
:10C18000400170430A21F3F7A5FF0246002C02D0BC
:10C190000020009901E002200021FBF7B3F80446DB
:10C1A000FBF77AF9002D00D162B6204601B0F0BD50
:10C1B000F0B581B01D460E460446022A0DD1012776
:10C1C00038463946FCF760FF00960022384629467B
:10C1D0002346FBF779F9044617E0174601200021B2
:10C1E000FCF752FF012F08D1009600202946024695
:10C1F0002346FBF769F9044607E000960220002178
:10C200000A462346FBF760F90446FBF745F920464A
:10C2100001B0F0BD7047000070B5002801D00120CA
:10C2200070BD0325A9020F4802680F4B535000242C
:10C230009460012253030D4E3360BFF34F8FBFF361
:10C240006F8F0B4E336003685A5084720481102044
:10C25000F8F7EEF9022007A22946FEF7DBFD20469B
:10C2600070BDC0461095010251E5CC1A80E100E096
:10C2700080E200E057445420636C6F73650D0A0040
:10C280002021020C01D010211046020A01D01046D4
:10C290000839020901D01046091F820801D0104652
:10C2A000891E420801D0881E7047081A704702E0B4
:10C2B00008C8121F08C1002AFAD170477047002031
:10C2C00001E001C1121F002AFBD17047DDDDDDDD79
:10C2D000DCBBBBDDDDDDDDDDDDDDDDDD9888888817
:10C2E00088888888777777777788888885555556BE
:10C2F0006666666666666666666888888333333215
:10C3000022222222222222222228888D000084C179
:10C31000000008C10000C03F000038410000AC41EF
:10C320000000D4410840080000081008040810204C
:10C33000000000000000000001000000FFFFFFFF00
:10C340000000000000000000280004000000590662
:10C350002014032145012882003241003219004196
:10C360001300390300B506002D03002D0200220141
:10C37000002201003E0100208009EE4D5048504F40
:10C3800080096E4F58E5854F80096E4FB867C14FE1
:10C390005048D04FB867C14FE828DF4F8009EE4FB3
:10C3A00018EAFC4F8009EE4F58E50550A4550D5092
:10C3B000F0C51450A4550D500000211042206330E8
:10C3C0008440A550C660E770088129914AA16BB1ED
:10C3D0008CC1ADD1CEE1EFF1311210027332522295
:10C3E000B5529442F772D662399318837BB35AA33D
:10C3F000BDD39CC3FFF3DEE3622443342004011465
:10C40000E664C774A44485546AA54BB5288509958C
:10C41000EEE5CFF5ACC58DD5533672261116300634
:10C42000D776F6669556B4465BB77AA719973887DC
:10C43000DFF7FEE79DD7BCC7C448E5588668A778F4
:10C440004008611802282338CCC9EDD98EE9AFF92C
:10C45000488969990AA92BB9F55AD44AB77A966AD4
:10C46000711A500A333A122AFDDBDCCBBFFB9EEB7C
:10C47000799B588B3BBB1AABA66C877CE44CC55CA4
:10C48000222C033C600C411CAEED8FFDECCDCDDDCC
:10C490002AAD0BBD688D499D977EB66ED55EF44E74
:10C4A000133E322E511E700E9FFFBEEFDDDFFCCF1C
:10C4B0001BBF3AAF599F788F8891A981CAB1EBA170
:10C4C0000CD12DC14EF16FE18010A100C230E320EC
:10C4D0000450254046706760B9839893FBA3DAB394
:10C4E0003DC31CD37FE35EF3B1029012F322D2323C
:10C4F0003542145277625672EAB5CBA5A895898564
:10C500006EF54FE52CD50DC5E234C324A01481048B
:10C510006674476424540544DBA7FAB79987B89733
:10C520005FE77EF71DC73CD7D326F2369106B016DB
:10C5300057667676154634564CD96DC90EF92FE9F3
:10C54000C899E9898AB9ABA944586548067827682B
:10C55000C018E1088238A3287DCB5CDB3FEB1EFBD3
:10C56000F98BD89BBBAB9ABB754A545A376A167A7B
:10C57000F10AD01AB32A923A2EFD0FED6CDD4DCDA3
:10C58000AABD8BADE89DC98D267C076C645C454CCB
:10C59000A23C832CE01CC10C1FEF3EFF5DCF7CDF73
:10C5A0009BAFBABFD98FF89F176E367E554E745E1B
:10C5B000932EB23ED10EF01E303132333435363741
:10C5C0003839414243444546100040008000000194
:10C5D00000020004000800101000180020003000C5
:10C5E0004000600080000001FFFFFFFF01FF01FF2E
:10C5F000FF0101FFFF01000000000000000000003B
:10C600000000000000000000000000000200000028
:10C6100000000000140000000200000007000000FD
:10C620000200000002000000000000000200000004
:10C6300000000000140000000200000001000000E3
:10C6400002000000020000000200000000000000E4
:10C650001400000000000000FFFFFFFFFFFFFF01CC
:10C66000FFFF01FFFF01FF01FF01FFFFFF0101FFCE
:10C67000FFFF01FF0101FFFF000100FF010000FFBC
:10C68000000064009E00C800E800020119012C01AE
:10C690003D014C015A01660172017D018701900143
:10C6A0009901A101A901B001B701BE01C401CA01EC
:10C6B000D001D601DB01E101E601EB01EF01F4015C
:10C6C000F801FD010102050209020D021102140226
:10C6D00018021B021F022202250228022B022E0230
:10C6E0003102340237023A023D023F024202450261
:10C6F00047024A024C024F025102530256025802AC
:10C700005A025C025F02610263026502670269020B
:10C710006B026D026F02710273027502760278027B
:10C720007A027C027E027F028102830284028602F8
:10C73000880289028B028C028E028F029102920281
:10C7400094029502970298029A029B029D029E0211
:10C750009F02A102A202A302A502A602A702A902A9
:10C76000AA02AB02AD02AE02AF02B002B102B30246
:10C77000B402B502B602B702B902BA02BB02BC02E9
:10C7800000000000000000000200000004000000A3
:10C79000001003EB00000000010000000100000099
:10C7A0000400000000010032000000000000000052
:10C7B0000000000001000000010000050000000072
:10C7C0000000000000000000010000000100003532
:10C7D0000000000001000000000000000400000054
:10C7E0000000002000000000010000000000000028
:10C7F00004000000000000D800000000010000005C
:10C800000000000001000000000000060000000021
:10C810000100000000000000010000000200000113
:10C820000000000000000000000000000100000007
:10C830000300009F00000000010000000000000055
:10C8400001000000000000B900000000010000002D
:10C850000000000001000000000000AB000100FF2C
:10C86000010000FF000100FF010000FFFF000001C8
:10C8700000FF00010001000000FF00FF00FF0000BA
:10C880000100FFFF00FF010000000001010000FFA8
:10C89000FFFF01FF01010000000001010003020190
:10C8A0000000050201000001030100000303010074
:10C8B0000100030100010203010002000301000264
:10C8C0000203010003020301000304030100040248
:10C8D000030100000003020000030302000006033E
:10C8E000020001000302000103030200010603022B
:10C8F0000002010302000204030200020703020017
:10C900000303030200000107030000060703000100
:10C9100000040300010007030001040703000107EE
:10C9200007030002000703000204070300020707D1
:10C9300003000302070300030607030004020703C2
:10C9400000040607030005010403000502070300B5
:10C950000506070300060007030006040703000698
:10C960000707030007030703000707070300080280
:10C97000070300080607030009020703000906076A
:10C9800003000A020703000A070703000B05070359
:10C99000000C030703000C070703000D0707030043
:10C9A0000E070703000E060704000E070704030E18
:10C9B000070704030E070704030E070704030E0707
:10C9C0000704030E070704030E070704030007000C
:10C9D000020201000002020004010202000701023B
:10C9E000020202000202010101020201060102022A
:10C9F0000305000202040200020202060102020311
:10CA000000010202030501020205030002020405FF
:10CA100001020202040202020207020202050301ED
:10CA200002020506010202060001020206030102DB
:10CA300002020503020202060302020106040202C8
:10CA400001060702020203040202020307020202B5
:10CA50000607020203020702020305070202030798
:10CA6000070202040704020205010402020501078D
:10CA70000202050307020205060702020602070278
:10CA80000206050702020701070202070407020265
:10CA9000080104020208020702020805070202094F
:10CAA0000304020209040702020A000702020A0242
:10CAB0000702020A050702020A070702020B030720
:10CAC00002020B060702020C010702020C04070215
:10CAD000020D010702020E000702020E0407020205
:10CAE0000F010702020F050702020E040703030FDE
:10CAF000030703030F070703030F070703030000E0
:10CB00000002020000000202000000020200000019
:10CB10000202000000020200000002020001000206
:10CB200002000400020200070002020101000202EA
:10CB300001040002020107000202020300020201D6
:10CB400004010202010601020203050002020204BE
:10CB500001020203010102020303010202040101B6
:10CB6000020204040102020206020202030202029D
:10CB7000020106030202020203020201020702028C
:10CB80000104070202030303020202040402020278
:10CB90000507020203010702020305040202040161
:10CBA000070202040307020205060302020500074A
:10CBB000020205020702020504070202060007023C
:10CBC0000206020702020605070202060707020222
:10CBD000070407020207070402020802070202080C
:10CBE00005070202090107020209040702020A00FE
:10CBF0000702020A030702020A060702020B0207E3
:10CC000002020B050702020C010702020C050702D3
:10CC1000020D020702020C010703030C06070303BF
:10CC20000D020703030E020703030E0707030300A9
:10CC300000000202000000020200000002020000E8
:10CC400000020200030002020100000202010200D1
:10CC500002020005010202020200020203010002B8
:10CC600002020101020202040102020102020202A6
:10CC70000104020202030401020202020202020291
:10CC80000502020200020702020004070202000677
:10CC9000070202010207020201040702020106075D
:10CCA0000202020307020202050702020302070250
:10CCB000020304070202040207020204040702023C
:10CCC0000406070202050107020205030702020526
:10CCD0000507020206020702020604070202060610
:10CCE00007020207040702020801070202090007FF
:10CCF0000202090107020209030702020A000702F1
:10CD0000020A020702020B000702020B02070202DC
:10CD10000C000702020B060702020C040702020CB9
:10CD2000060702020D030702030C000703030C02AF
:10CD30000703030C050703030C070703030D05078F
:10CD400003030D070703030D070703030D0707037D
:10CD5000030D070703030D070703030D070703036D
:10CD60000E0D0B07696E636C7564652F64726976CE
:10CD70006572732F6D6B5F6164632E6300696E6310
:10CD80006C7564652F647269766572732F6D6B5F65
:10CD90006165732E630033324B206C6F61642063D6
:10CDA00061702076616C2025640D0A005854414C56
:10CDB000206C6F6164206361702076616C20256453
:10CDC0000D0A00556E657870656374656420646D46
:10CDD00061206368616E6E656C0D0A00696E636C3C
:10CDE0007564652F647269766572732F6D6B5F660B
:10CDF0006C6173682E630052656C6F6164207661AC
:10CE00006C756520696D706F737369626C650D0A6E
:10CE100000696E636C7564652F6472697665727300
:10CE20002F6D6B5F6D6973632E63007379735F742D
:10CE300069636B5F7374617274005265736574200B
:10CE4000627920756E6B6E6F776E20736F7572638B
:10CE5000650D0A0025313064207C200D0A004372E4
:10CE600061736865642121210D0A002D2D2D2D2D62
:10CE70002D2D2D2D2D2D2D2D2D2D2D2D2D2D2D2DE2
:10CE80002D2D2D2D2D2D2D2D2D2D2D2D2D2D2D2DD2
:10CE90002D2D2D0D0A00253038583A2025303858D0
:10CEA0002025303858202530385820253038580D66
:10CEB0000A005052494D41534B3D253038580D0A18
:10CEC00000434F4E54524F4C3D253038580D0A0008
:10CED0004D53503D253038580D0A005053503D25D4
:10CEE0003038580D0A0041495243523D25303858D8
:10CEF0000D0A004C523D253038580D0A0049505358
:10CF0000523D253038580D0A00785053523D253097
:10CF100038580D0A004E3D25642C205A3D25642CBE
:10CF200020433D25642C20563D25640D0A004649CA
:10CF30004C45202020203A20005B53435030335D85
:10CF4000005B464952415D005B5557425D005B4DB9
:10CF500041435D005B4343435D005B564552424F96
:10CF600053455D005B53455D005B5543495D005B88
:10CF70005741524E5D005B494E464F5D005B41504C
:10CF8000505D005B4552524F525D005B4F535D0058
:10CF90005B424F4F545D005B544553545D005B440E
:10CFA00052565D005B5048595D00696E636C756454
:10CFB000652F647269766572732F6D6B5F74726131
:10CFC00063652E6300257300696E636C7564652F5D
:10CFD000647269766572732F6D6B5F756172742E02
:10CFE0006300556E65787065637465642075617261
:10CFF0007420256420737461746520256400556E67
:10D00000657870656374656420646D612063686130
:10D010006E6E656C20256400506172616D7465727E
:10D0200020696E76616C696400756172745F646D0D
:10D03000615F63616C6C6261636B00756172745FE8
:10D04000626175645F736574007577625F74785FA1
:10D05000696E69742C20706F776572206C657665D7
:10D060006C2025640D0A004F70656E20414E5425DA
:10D07000640D0A0024255B5E2C5D2C252A5B5E2C4A
:10D080005D2C255B5E2C5D2C252A5B5E2C5D2C25A2
:10D090005B5E2C5D2C252A5B5E2C5D2C255B5E2C5B
:10D0A0005D2C252A5B5E2C5D2C252A5B5E2C5D2C7D
:10D0B000252A5B5E2C5D2C252A5B5E2C5D2C252AA7
:10D0C0005B5E2C5D2C252A5B5E2C5D2C252A5B5E2D
:10D0D0002C5D2C252A73006C73705F7363616C6523
:10D0E0005F663332006C73705F675F6F705F6633CB
:10D0F00032006C73705F675F6F705F696E7431369A
:10D10000006C73705F675F6F705F696E7438002EBC
:10D110002E2F2E2E2F2E2E2F2E2E2F2E2E2F6472B0
:10D1200069766572732F6D6B5F6C73702E63004F41
:10D13000706572616E64206164647265737320252A
:10D140007820697320696E76616C6964004E65654C
:10D1500064206174206C65617374206F6E65206F4C
:10D16000706572616E6400525820444553432069D3
:10D170006E646578206973206F7665722072616EC7
:10D1800067650D0A00455420696E646578206973EF
:10D19000206F7665722072616E67650D0A002E2E13
:10D1A0002F2E2E2F2E2E2F2E2E2F2E2E2F647269E5
:10D1B000766572732F6D6B5F6D61632E63006D61B9
:10D1C000635F72785F646573635F636F6E737472BD
:10D1D000756374006D61635F65745F636F6E737414
:10D1E0007275637400556E646566696E656420626D
:10D1F0006974207261746520256420666F72206DE9
:10D2000065616E20505246206F662025640D0A002D
:10D210004D45414E2050524620706172616D6574DB
:10D220006572206572726F720D0A00436F6465202B
:10D2300069647820256420616E64206D65616E20CC
:10D2400050524620256420636F6E666C6963740DCE
:10D250000A002E2E2F2E2E2F2E2E2F2E2E2F2E2E3C
:10D260002F647269766572732F6D6B5F7068792EAB
:10D27000630001000001000000FF00FFFF0000FF4D
:10D28000FF01000100010000FF01FF01010001009A
:10D290000000000101FF000000010000FF0000FF8E
:10D2A000FF00FF01000100FFFF00FF01010100017D
:10D2B0000100000001FF00010000FF000101FF006C
:10D2C0000101010000FF01000001000100FF000159
:10D2D00001FF01FFFF01000000000000010000004D
:10D2E0000000FF0100000000FF00FF000000FFFF42
:10D2F00001010100000100FF010000010000010028
:10D300000000000000FF000000FF0000FFFF000021
:10D3100000FF0001FF0100FF0001FF00FF0100000E
:10D3200000000001FF0000010100FF00010000FFFC
:10D33000FF0100000101FF010001FF0001000000EA
:10D3400000FF00FF00FF00FF0101FF0100010000DE
:10D35000010001000000FF0100010101000000FFC9
:10D36000FFFFFF0101010000000001010100FFFFBC
:10D37000FF01FF00000000010000FFFF00000000AF
:10D3800000FF000100010001FF000100000100009A
:10D390000100FF0000FF010101000001000000FF8B
:10D3A00001000100FF000000000101010101FF0177
:10D3B0000001FFFF0001FF000101FFFF00FF00006F
:10D3C000000100FF010000010001FFFFFFFF00005E
:10D3D00000FF000000000000FF01000001FF00014D
:10D3E000010000000101FF00000101FF00FF00FF3C
:10D3F00001000101000000000000FF000100FF012A
:10D4000000FFFFFF01FF01010000FF01000101001B
:10D410000100010001000000FF0000FF0000FF010B
:10D42000000001FF0101000000FF01FF00FF0101FA
:10D4300000FF000101010100FF0000FF00010100E9
:10D440000001000100000101FF00000100000001D7
:10D45000FF000000FF00FFFF0100000000FF0000D0
:10D460000000FFFF0001000000000001FFFF0100BD
:10D470000000FFFF00000000FFFF010100FF0101AD
:10D48000010100FF000101000100FF0000FF010099
:10D49000010100000101FF0001010001FF0100FF87
:10D4A0000000010000FF00FFFF000000FF01FF007F
:10D4B000000100000000FF000101FF00000000006B
:10D4C00001FF00FF000000000000FF0000FF01FF5F
:10D4D0000101FF01000000FF000100010001010146
:10D4E000FF0000FFFF00000100010000000100003C
:10D4F00000010100FF000100FF000001FF00FF012B
:10D5000000FF000001000100000000010001FF0019
:10D510000000000101000001000101010101FF0103
:10D5200000FF0001FF00FFFF01000101FFFF0000FD
:10D5300000FFFFFF000100000001000100FF01FFEC
:10D5400000000000000001FF01FF00FFFF000001DC
:10D5500001000000FF00000100000101FF0000FFCA
:10D56000FF0101FF0000FF00000000000001FF00BC
:10D57000000100FF000000FF010100000000FFFFAC
:10D58000FF0101000000010001FF00FF010000FF9A
:10D5900001000000FFFF00FF0000FFFF00FFFF0190
:10D5A0000101FF0100FF0101000001FF0101000175
:10D5B00000000000000100FF00010101FF00000168
:10D5C000000001000000FF00000000010000FFFF5C
:10D5D000010001010001000100FF0000FF00FF0148
:10D5E000FF00010001010000000000010100000037
:10D5F000000100000001000001FFFF0001FF010128
:10D6000000FF000000FFFF000001FF00010000011B
:10D6100001000000010101000001000100FF00FF06
:10D6200001FF00FF0001000001000001000101FFF7
:10D63000FFFFFF0100000101FFFF010001FF00FFEC
:10D64000FF01000000000000FF00FF00000000FFDD
:10D650000100FFFF000001000000000001FF0101C8
:10D66000000000FF00FF0100010001FFFF000000BB
:10D67000FF00FF0000000001FF00000000000100AB
:10D68000000000000001FFFF01FF010100FF000199
:10D690000001000001FF000001010100FF01010085
:10D6A000FF00000100FF0100000001010001010175
:10D6B000FF00FFFF00010001FF00FFFF0000FF006F
:10D6C0000001000000FF0101000000000100010155
:10D6D000FF01FF00000100010001FFFF0000FFFF4C
:10D6E00000FF00000001000001FFFF000101010038
:10D6F000000000010101FFFFFFFF00000001010128
:10D700000001FF0000000100010000010001FF0115
:10D7100001FF00FF00FF00FF000000000100FF010B
:10D720000001FF0101000001FFFF00000100FF00F8
:10D7300001010000FF01000000000001FF00FF01E7
:10D7400000FF0001FF0100FF000000FFFF0000FFDD
:10D75000000000FF000000000000010000010000C8
:10D7600001FF000100000101FF00FF01010000FFB7
:10D770000101000000010100FF01000001FF0000A5
:10D7800000000000FF000000FFFFFFFF010001009C
:10D790000001FF0001000000FF00FFFF010100FF8A
:10D7A0000100FFFF010001FF010101010100000074
:10D7B00000FF00010001FF00000001000001010165
:10D7C000FF0000FF000100000100000100FF010058
:10D7D00001000100FF0000000000FFFF0000010049
:10D7E000000000FF01FF00FFFF010000000000013A
:10D7F00000FFFF00000000FF0000000001FFFF002D
:10D80000FF000000FF01000000010000FF01010017
:10D81000000100010000010100FF0000FF00010104
:10D82000010100FF000101FF00FF01FF00000001F6
:10D8300001FF01000001FF0000FF0000FF000000E9
:10D8400001000100010001010001FF00000101FFD2
:10D8500001FFFFFF0001FF000100FF0000000000CA
:10D860000001010001FF0100010000FFFF0000FFB7
:10D870000101010001000100FF00000001FF0101A2
:10D88000FF01FF0000FF000000000000FF00FF019B
:10D890000000000000FF010100FF00000000010087
:10D8A00000FF01FF000000FFFF00FF00000100007B
:10D8B000FF0001FF0100010100FF01010000010163
:10D8C0000001FF0000FF000100010100FF00010155
:10D8D0000101FF000101FFFF00000000FFFF000049
:10D8E000000100000000FF0000FF0101FFFF000039
:10D8F000FF01010000010000FF0000000101000025
:10D90000FFFF00FF01FF01000000000000FF01FF1A
:10D91000000100010000000100FFFFFF000000FF08
:10D92000FF01010001FFFF00FF0100FF0001FF01F7
:10D930000101010100010000010100000000FF01E0
:10D940000001000000000100010000FF0001FF00D5
:10D95000FF010000FF000100FF00010100000001C5
:10D96000000000000000000101000100FF01FF00B5
:10D97000FF0000FF000100010001010001FFFF00A6
:10D98000000100000000FF00000001000001000095
:10D99000FF01010100FF0001000000000001000183
:10D9A00001FF0100000101FF0001FF010101FFFF74
:10D9B00000FFFF0000FF00FFFF00000001FF00006C
:10D9C00001FF00FF0100010000000101FFFFFF0057
:10D9D0000000000101FF000000FF00010000FF0146
:10D9E000000000010001FF00FF0000000101FF0135
:10D9F0000000000000010000FFFF0001FF00000028
:10DA000000FF00FF00000000000001FFFF00FF0119
:10DA10000001FFFF0101000001FFFFFFFF01010006
:10DA20000100000100000100FF00FF01FF00FF00F6
:10DA300001000100000101010000000101000001DE
:10DA400000FF010000FFFF000000FF000101FF01D7
:10DA500000FFFF01000001000000010000000001C4
:10DA60000100FF000000000100FF000101010001B2
:10DA7000FF00000001FF0101010000FF0100FF00A5
:10DA80000000010001FF00010001000000FF010192
:10DA900000FF01FFFFFF0000010000010100000086
:10DAA000FF01000101000000FF01FF010100000172
:10DAB0000100010000FF00000000FF000100FF0066
:10DAC00000000001FF0000FF0000FF010101010054
:10DAD00001FF010000000100FF00010100FFFF0045
:10DAE00001FF0000010101FF01000000FF01000132
:10DAF000010100FF000100000000FF000001010023
:10DB000000010000FFFFFF01FF000101FF00000016
:10DB100001000100FF010001000000000100000001
:10DB20000001FF00010001000001000000010001F0
:10DB300001FFFFFF00FF010000FF0100010000FFE7
:10DB400000FF00010100000000FFFF010000FF01D5
:10DB5000000101FF010100010000FF0001010101BE
:10DB6000FFFF01FFFF01FF01010101FF01FFFFFFB7
:10DB70000101FFFF010101010101FF0101FF01009E
:10DB80000001FFFF0100FFFF01000101010101FF92
:10DB9000FF010101FFFF00FFFF0001FF01FFFFFF89
:10DBA000FF00FF01FF01FF010001FFFF0101FF0175
:10DBB000FF0101010001010001FF01FFFFFF010161
:10DBC000010101FF01FF0101FFFF01FFFF0101FF53
:10DBD000FFFF01FF0001010100FF01010101FF0141
:10DBE000000100FFFF0001FF0101FF010101010130
:10DBF00001FFFF01FF01010000010101FFFF000122
:10DC0000FFFFFFFFFF01FF0001FF01FF01FFFFFF1B
:10DC1000010101FFFF010101FFFFFF01FF01FF0003
:10DC2000FF01FFFF000101FF01FF0100FF010101F2
:10DC300001010101010101FFFF01FFFF0101FF01DE
:10DC400001000101FF01FF01FFFF01FFFF010101D1
:10DC5000FFFFFF00FF010101FF00010000FFFFFFC8
:10DC60000101FF01FFFF00FF0101000101010101AE
:10DC7000FFFF010101FF0101FFFFFF01FF01FFFFA6
:10DC8000000101FFFFFF01FF010001FFFFFFFFFF98
:10DC90000100010101FFFF01FF01FFFF01FF010181
:10DCA000FF0101010100FF00FF0101000001FF0170
:10DCB0000101FF0101FF0100FF0100FFFF01FFFF64
:10DCC000FF010101000101FF00FFFF01FF0101FF52
:10DCD000FF00010100000101FF0101FFFFFFFFFF45
:10DCE000010101010101FF0001FFFF01FF0101FF2F
:10DCF000FF01FF010101FFFF01010101010101FF1E
:10DD00000101010001FF01FF00FF00FF0101FFFF12
:10DD1000FF0100FFFFFF010100FF01FF01FF010103
:10DD2000FFFF010100FFFF000101FF0000FFFF01F5
:10DD300001FF0101FF01FFFF0101010101FFFFFFE1
:10DD4000010101FF01FF0001FF01FF0100010101CD
:10DD50000101FF010101FF010101FF0100FFFFFFC0
:10DD6000FFFFFF0101FF0101FF0100FFFFFFFF01B6
:10DD7000FF01FF00010001FF010101FFFF01FF01A1
:10DD80000100010101FFFF0101FF0001010000FF8F
:10DD9000FF0101FFFF010101FF01FFFFFFFFFFFF87
:10DDA00000010101FF0101010101FFFF01FF01016C
:10DDB000FFFFFF01FF01FFFFFF01FF0100FF01FF68
:10DDC000FF00010001FF0101FF01010001FF01FF50
:10DDD000FF000101010101FF010101010101010138
:10DDE000010101FFFFFF01FF0101FFFF0101000031
:10DDF000FF01FF0100FF01FF00FF0101FFFF010123
:10DE000001FF01010100FFFF000101FF01FF01FF10
:10DE100000FFFFFF0101FF00FFFFFFFF0101010104
:10DE2000FF01FF000100FF01FF0101FF0101FFFFF2
:10DE300001FF0400000404040404040404000000BE
:10DE400060DE00000890010218050000800D00004F
:10DE500040E0000020950102AC260000BEC2000098
:10DE6000560026B8030145900050084202C2030044
:10DE70001515C0C1C2C3C4C5C6C7C8C9CACBCCCD9D
:10DE8000CECF000101013C0180030509020302021B
:10DE9000010133020365090203014202571400190C
:10DEA000412717901D0706050403020100F2979809
:10DEB000DDC89D5CB81CC0DEA7DB615BCA01020047
:10DEC0000352404805100406010001522D2C280081
:10DED00004007C007B0105020308FF5B0F01006565
:10DEE000F901417B0707010160002000881333E03E
:10DEF000536420ACFF501B0D070E080E080E080ED1
:10DF0000080C030D050B050D070D070D070D070187
:10DF1000012E010402004003FFFF7F00FFFF7F0886
:10DF200016FFFFFF00FFFFFF3A010001000A00019A
:10DF30000106401E400512051200051504020102EB
:10DF4000030102400402010303020C0E0900087AD7
:10DF50000232413428002A820303455006C570016D
:10DF60004013E620700140144C07001000D6FF005B
:10DF7000B000500B4202820345FFFF0F20320442E3
:10DF800008320104551000010A50B40003010020BA
:10DF90000050074601012800049901020100FFFF1B
:10DFA000FFFF37609001022FCC0051151EC135BF15
:10DFB00080F3E2BDC0B464BF871699BDAD178DBFB5
:10DFC000941799BD33A876BFC4780DBD2BC162BA32
:10DFD0000CB0AFBEA9F6E9BAFC567BBE07254CBB18
:10DFE000EC8823BE5DC0CBBB0CCE20BD7BA095BC16
:10DFF000D40F3A3E2D5EACBD5913073F6401004279
:10E000004209440300063201451001400FC20E428E
:10E0100001520332804201C20702100352014590AF
:10E020000140184204023D0545A001401942060284
:10E030003D07454001400D82010000000000000046
:020000040000FA
:10E38000A5A54B4D0000001000000002AAAA5A7F6C
:10E3900080E3000000000000020000000000000018
:10E3A000000000000000000000000000000000006D
:10E3B000000000000000000000000000000000005D
:10E3C00018E40000000000000A56656E646F7209D0
:10E3D0003A204D4B53454D490A43686970093A202C
:10E3E0004D4B383030300A44617465093A2041752C
:10E3F0006720203820323032340A56657273696FD4
:10E400006E093A2056302E362E32000000000000F1
:08E41000000000000000000004
:04000005000000C136
:00000001FF
